:020000040800F2
:1000000000000220F92701085192000853920008CD
:10001000559200085792000859920008000000000D
:100020000000000000000000000000005B920008DB
:100030005D920008000000005F92000861920008D5
:100040003D2801083D2801083D2801083D280108F8
:100050003D2801083D2801083D2801083D280108E8
:100060003D2801083D2801083D280108C175000808
:100070003D2801083D2801083D2801083D280108C8
:100080003D2801083D2801083D2801083D280108B8
:100090003D2801083D2801083D28010881940008F9
:1000A0003D2801083D2801083D2801083D28010898
:1000B0005D9400083D2801083D2801083D280108FD
:1000C0003D2801083D2801083D2801083D28010878
:1000D0003D2801083D280108959500083D280108A4
:1000E0003D2801083D280108659200083D280108C7
:1000F0003D2801083D2801083D2801083D28010848
:100100003D2801083D2801083D2801083D28010837
:100110003D2801083D2801083D2801083D28010827
:100120003D2801083D2801083D2801083D28010817
:100130003D2801083D2801083D2801083D28010807
:100140003D2801083D2801083D2801089592000836
:100150003D2801083D2801083D2801083D280108E7
:100160003D2801083D2801083D2801083D280108D7
:100170003D2801083D2801083D2801083D280108C7
:080180003D2801083D2801089B
:100188002CEB050800000020B00D0020B00D002069
:10019800483F002008B5074B186808F0F7FF0DF036
:1001A800BBFA054B054806221A70BDE8084001F065
:1001B8009EBA00BFB0280020382800201011002067
:1001C80008B5034801F093FA024B00221A7008BDE3
:1001D800081A00203828002008B5054B0122002005
:1001E8001A7005F06FFC0348BDE8084001F07FBABB
:1001F800C82E0020D41600202DE9F041144C2046CA
:1002080003F0BFFD00201349134A03F071FB1349A3
:10021800134A0746002003F06BFB1249124A0646B0
:10022800002003F065FBD22105463A4623460A2002
:1002380003F076FCD22132462346FA2003F070FC04
:100248005A20D2212A462346BDE8F04103F068BC73
:10025800E8140020D6D70508C9010008DFD705082B
:10026800E1010008E7D705089D01000808B5054B1E
:10027800012200201A7005F025FC0348BDE808405B
:1002880001F035BAC82E0020D416002008B503485E
:1002980001F02DFA024B00221A7008BD081A00203E
:1002A8003828002008B5054B07221A700DF034FADB
:1002B8000348BDE8084001F01ABA00BF38280020FA
:1002C800E81400202DE9F041144C204603F059FDB4
:1002D80000201349134A03F00BFB1349134A07463E
:1002E800002003F005FB1249124A0646002003F0DD
:1002F800FFFAD22105463A4623460A2003F010FCAD
:10030800D221324623465A2003F00AFCAA20D221E1
:100318002A462346BDE8F04103F002BC1011002034
:10032800D6D7050895020008F0D70508AD020008E1
:10033800F9D7050875020008014801F0D8B900BFCF
:10034800FC12002010B5094C204603F01AFD0020CD
:100358000749084A03F0CCFAD221024623464FF453
:100368008270BDE8104003F0DBBB00BF1C18002002
:1003780002D805084103000870B50C4C0C4D2068E4
:100388004FF6E076314602F0F7FD2068294602F084
:10039800A1FD6068314602F0EFFD6068294602F071
:1003A80099FDBDE8704003F025BF00BFB00D0020E7
:1003B800DFDD050838B52B4CFFF7DEFF002005F020
:1003C80081FB237A23B90A203221274A05F088FCC9
:1003D800637A23B90A206421244A05F081FC214C60
:1003E800A37A23B90A209621214A05F079FCA37A39
:1003F8001C4DFBB16B7AEBB12B7ADBB100232B726E
:100408006B72AB721B4B286801221A704FF6E071B1
:1004180002F0B2FD2868184902F05CFD68681749C7
:1004280002F058FD0BF0A3F903F0E4FE144803F0C2
:1004380025FF0DE00B4C4FF47841206802F09CFD3D
:100448002068104902F046FD60680F4902F042FD3D
:10045800FFF792FF00200BF04DF90C48BDE838403B
:1004680001F045B9B00D002009D8050817D80508CE
:1004780026D805083828002034D80508E0DD050806
:100488008096980048D80508E2DD0508081A00207B
:1004980008B500200BF02EF90248BDE8084001F02D
:1004A80026B900BF081A002038B5FFF765FF0DF020
:1004B8004BF93C213F220023DF2005F0F3FB4FF4EA
:1004C80080600DF0A5FE124C3E223C21DF20002367
:1004D80005F0E8FB012323720E4B4FF6E075186810
:1004E80008F054FE2068294602F046FD20680A49B3
:1004F80002F0F0FC6068294602F03EFD606807499A
:1005080002F0E8FC03F076FE054B00221A7038BDB5
:10051800B00D0020B02800205AD805086DD805086D
:100528003828002038B5FFF727FF0DF00DF96E21A8
:100538003F220023DF2005F0B5FB4FF486400DF085
:1005480067FE124C3E226E21DF20002305F0AAFB35
:10055800012363720E4B4FF6E075186808F016FE1B
:100568002068294602F008FD20680A4902F0B2FC1A
:100578006068294602F000FD6068074902F0AAFC9D
:1005880003F038FE054B00221A7038BDB00D00206C
:10059800B028002080D8050891D805083828002000
:1005A80010B5FFF7E9FE0DF0CFF8A0213F22002398
:1005B800DF2005F077FB4FF402400DF029FE114CC7
:1005C8003E22A021DF20002305F06CFB0123A3724B
:1005D8000D4B186808F0DAFD20684FF6E07102F05C
:1005E800CBFC2068094902F075FC6068084902F0F4
:1005F80071FC03F0FFFD64200AF054FF054B002254
:100608001A7010BDB00D0020B0280020A2D805082F
:10061800E0DD0508382800202DE9F74F3A4D3B4E1C
:100628000024284603F0ADFB224623464FF6FF710F
:1006380037480094019402F063FC4FF6E0780427F1
:10064800F06041462246234632480097019402F062
:1006580057FC23463060414622462F4800970194B4
:1006680002F04EFC2D4970602D4A204603F040F9F7
:100678002C492D4A0746204603F03AF92B492C4AC3
:100688008046204603F034F92A492B4A8146204601
:1006980003F02EF929492A4A8346204603F028F90F
:1006A80021468246F2682B46204603F039FA5A2141
:1006B80032682B460A2003F033FA6E2172682B4603
:1006C8000A2003F02DFA9B213A462B46FA2003F024
:1006D80027FA692142462B46FA2003F021FA3721EE
:1006E8004A462B46FA2003F01BFAC82152462B46ED
:1006F800AA2003F015FAF020C8215A462B4603B069
:10070800BDE8F04F03F00CBA8C150020B00D0020A6
:10071800B6D80508BED80508D1D80508E0D8050818
:10072800A9050008E8D805082D050008D8D8050847
:10073800B1040008F0D8050899040008F7D805089E
:10074800BD03000838B50C4C4FF6E0752068294603
:1007580002F012FC2068094902F0BCFB60682946D7
:1007680002F00AFC6068064902F0B4FB03F042FD9F
:10077800BDE8384003F03EBDB00D0020BED80508E6
:10078800FED8050870B52DED028B9FED248A88B040
:100798000A26F0EE488A03E0B0EE608AF0EE418A5D
:1007A8000CF037FA8DED000ACDED010A9DE8030043
:1007B80004AB83E80300F0EE680AB0EE480A9DED4A
:1007C800041ADDED051A8DED028ACDED038A0BF0D2
:1007D800C3FFCDED010A8DED000A9DE8030002ADCF
:1007E80085E80300013E6C46DDED020A9DED031A23
:1007F800D2D19FED0B0A0CF003FA8DED000ACDED76
:10080800010A9DE8030085E80300DDED030A9DED7C
:10081800020A08B0BDEC028B70BD00BF00000000EA
:10082800CDCCCC3D2DE9F74F564D574CDFF86491B0
:10083800DFF864814FF6E07005F018F9286810F0C9
:10084800DFFE064668680F4610F0DAFE3246CDE94C
:1008580000013B464946204615F00CFD2246002380
:100868000520372105F03CFA2869484F484E10F01A
:10087800C7FE824668698B4610F0C2FE5246CDE933
:1008880000015B463946204615F0F4FC2246002359
:100898000520692105F024FA286B10F0B1FE824684
:1008A800686B8B4610F0ACFE5246CDE900015B4602
:1008B8004146204615F0DEFC002305209B212246F8
:1008C80005F00EFA31462A6C204615F0D3FC224674
:1008D80000239B21A22005F003FA4FF4FC6005F0E9
:1008E800C5F8A86810F08CFE8246E8688B4610F0C0
:1008F80087FE5246CDE900015B464946204615F081
:10090800B9FC224605205021002305F0E9F9A86921
:1009180010F076FE8246E8698B4610F071FE52466A
:10092800CDE900015B463946204615F0A3FC224676
:1009380000230520822105F0D3F9A86B10F060FE92
:100948008246E86B8B4610F05BFE5246CDE900010B
:100958005B464146204615F08DFC00230520B42156
:10096800224605F0BDF931466A6C204615F082FC36
:10097800A220B4212246002303B0BDE8F04F05F0C1
:10098800AFB900BFD43C0020C00D002023D9050812
:1009980046D9050811D9050835D9050808B5002034
:1009A80005F090F80A4B1B780B2B0BD8DFE803F007
:1009B8000A0A0A0A0A0A08060A0A0A0A054802E08E
:1009C800054800E00548BDE8084000F090BE00BFBB
:1009D80038280020E814002010110020081A0020F0
:1009E8002DE9F14F2D4C204603F0CBF900202C497E
:1009F8002C4A02F07DFF2C492C4A8146002002F047
:100A080077FF2B492B4A0746002002F071FF2A493D
:100A18002A4A0646002002F06BFF2949294A054662
:100A2800002002F065FF2849284A8046002002F08D
:100A38005FFF2749274A8246002002F059FFD2214A
:100A480083464A462346E62003F06AF828203A46B9
:100A58002346014603F064F84621324623462820FF
:100A680003F05EF864212A462346282003F058F84C
:100A7800822142462346282003F052F85246234654
:100A88002820A02103F04CF828205A46BE212346EE
:100A980001B0BDE8F04F03F043B800BFD416002002
:100AA8004BD90508A509000854D90508751200088E
:100AB8005FD905085112000869D905082D120008E8
:100AC80074D90508091200087FD90508E51100083E
:100AD80089D90508C1110008023810B50A2800F2A2
:100AE8003C83DFE810F00B000F006400D2008A019D
:100AF8002001170231023A03A102F502BDE81040B5
:100B08000AF0A2BE00204FF6E0710AF0FBFF632056
:100B18004FF6E0710AF0F6FFB3204FF4F0610AF0E7
:100B2800F1FFC7204FF6E0710AF0ECFF4FF6FF70B7
:100B380004F09CFFDC2100237D20D34A05F0D0F887
:100B48004EF29C7004F092FF052001210023CF4A49
:100B580005F0C6F8052052210023CD4A05F0C0F85B
:100B6800B62100230520CB4A05F0BAF84FF4F0600F
:100B780004F07CFF0121002340F21310C34A05F062
:100B8800AFF8002340F213105221C24A05F0A8F82A
:100B9800B621C14A40F21310002305F0A1F84EF225
:100BA8009C7004F063FF0520A221BC4A68E0002085
:100BB8004FF6E0710AF0A6FF31204FF6E0710AF017
:100BC800A1FF63204FF6E0710AF09CFF95204FF6D5
:100BD800E0710AF097FFC7204FF6E0710AF092FF24
:100BE8004EF29C7004F042FF052001210023AC4A1C
:100BF80005F076F8052020210023AA4A05F070F8B0
:100C0800052052210023A84A05F06AF8052084210E
:100C18000023A64A05F064F8B62105209D4A002362
:100C280005F05EF84FF4F06004F020FF012140F277
:100C3800131000239A4A05F053F840F213102021AC
:100C48009B4A002305F04CF840F213105221914AB8
:100C5800002305F045F840F213108421954A00233B
:100C680005F03EF8B621944A40F21310002305F02F
:100C780037F84FF6FF7004F0F9FE904A7D20DC212A
:100C88000023BDE8104005F02BB800204FF6E071B6
:100C98000AF038FF27204FF6E0710AF033FF4F20A3
:100CA8004FF6E0710AF02EFF77204FF6E0710AF058
:100CB80029FF9F204FF6E0710AF024FFC7204FF666
:100CC800E0710AF01FFF4EF29C7004F0CFFE052081
:100CD800012100236F4A05F003F80520162100239F
:100CE800774A04F0FDFF05203E210023754A04F0F1
:100CF800F7FF052066210023734A04F0F1FF8E21D7
:100D080000230520714A04F0EBFF0520704AB62144
:100D1800002304F0E5FF4FF6FF7004F0A7FE7D20E6
:100D2800DC216C4AACE700204FF6E0710AF0EAFEDD
:100D380031204FF6E0710AF0E5FE63204FF6E071CE
:100D48000AF0E0FE95204FF6E0710AF0DBFEC720BE
:100D58004FF6E0710AF0D6FE4EF29C7004F086FE63
:100D68000520012100235C4A04F0BAFF0520202158
:100D780000235A4A04F0B4FF052052210023584AA0
:100D880004F0AEFF052084210023564A04F0A8FF92
:100D9800B62105203F4A002304F0A2FF4FF4F0607B
:100DA80004F064FE012140F2131000234E4A04F0BF
:100DB80097FF40F2131020214C4A002304F090FFC3
:100DC80040F213105221334A002304F089FF40F205
:100DD80013108421464A002304F082FFB621454AB5
:100DE80040F21310002304F07BFF4FF6FF7004F06D
:100DF8003DFE7D20DC21404A42E700204FF6E071AD
:100E08000AF080FE31204FF6E0710AF07BFE632085
:100E18004FF6E0710AF076FE95204FF6E0710AF081
:100E280071FEC7204FF4FC610AF06CFE4EF29C7014
:100E380004F01CFE052001210023304A04F050FF75
:100E48000520202100232E4A04F04AFF05205221C4
:100E580000232C4A04F044FF8421002305202A4A59
:100E680004F03EFF4FF4F06004F000FEB6210520C8
:100E7800264A002304F034FF4FF6FF7004F0F6FD15
:100E88008720234ADC21FBE65FD9050893D90508AA
:100E98008ED9050860DF050892D90508C0D905086C
:100EA800ACD9050897D90508A7D905089CD905081C
:100EB800A1D90508A6D90508ABD9050869D9050837
:100EC800AFD90508B3D90508B7D90508BBD90508AE
:100ED800BFD90508C3D90508CFD90508D3D905084E
:100EE800D7D90508DAD90508E3D90508DFD90508EF
:100EF800DED90508E2D90508E7D90508F2D90508B9
:100F0800B8D90508B0D9050802DA050877E0050858
:100F180089D9050800204FF6E0710AF0F3FD632037
:100F28004FF4FC610AF0EEFD4FF6E071C7200AF0BD
:100F3800E9FD4FF6FF7004F099FD002004F098FEDB
:100F4800A520D721854A9BE6042004F091FE0020C5
:100F58004FF6E0710AF0D6FD31204FF6E0710AF045
:100F6800D1FD63204FF6E0710AF0CCFD95204FF6D5
:100F7800E0710AF0C7FDC7204FF6E0710AF0C2FD24
:100F88004EF29C7004F072FD052001210023744A82
:100F980004F0A6FE052020210023724A04F0A0FEDA
:100FA800052052210023704A04F09AFE052084216E
:100FB80000236E4A04F094FE0520B6216C4A0023F3
:100FC80004F08EFE4FF6E07004F050FD40F20B1076
:100FD8000121684A002304F083FE40F22B102021EF
:100FE800654A002304F07CFE40F223105221634A34
:100FF800002304F075FE40F21B108421604A002390
:1010080004F06EFEB6215F4A002340F2131004F08C
:1010180067FE4FF6FF7004F029FD002004F028FE5B
:101028006E20D221584A90E0042004F021FE0020CE
:101038004FF6E0710AF066FD27204FF6E0710AF0DE
:1010480061FD4F204FF6E0710AF05CFD77204FF606
:10105800E0710AF057FD9F204FF6E0710AF052FD4B
:10106800C7204FF6E0710AF04DFD4EF29C7004F077
:10107800FDFC052001210023444A04F031FE05202F
:1010880016210023424A04F02BFE05203E210023AE
:10109800404A04F025FE052066213F4A002304F05B
:1010A8001FFE05208E213D4A002304F019FEB621BB
:1010B8003B4A0023052004F013FE4FF6FF7004F0AE
:1010C800D5FC002004F0D4FD6420D221354A3CE050
:1010D800042004F0CDFD00204FF6E0710AF012FD67
:1010E80043204FF6E0710AF00DFD85204FF6E071C0
:1010F8000AF008FD4FF6E071C7200AF003FD4EF232
:101108009C7004F0B3FC05200121274A002304F059
:10111800E7FD05204521254A002304F0E1FD0520CF
:1011280087211F4A002304F0DBFDB621204A002353
:10113800052004F0D5FD4FF6FF7004F097FC002061
:1011480004F096FD1B4A7D20D221002304F0C8FD3F
:101158000420BDE8104004F08BBD10BDF8DD050883
:10116800F6D9050802DA050801DA050804DA0508DF
:1011780008DA05080DDA0508ACD9050814DA0508F7
:1011880018DA05081DDA050823DA050829DA05083A
:10119800DFD90508E4D905082EDA050831DA05088B
:1011A800C0D9050834DA05083DDA0508F2D905087A
:1011B80060DF0508D4DE050810B5064C064806238E
:1011C800237000F094FA2078FFF786FCBDE8104001
:1011D8000CF0ECBFC82E00206419002010B5064C96
:1011E80006480723237000F082FA2078FFF774FC82
:1011F800BDE810400CF0DABFC82E002064190020AA
:1012080010B5064C06480523237000F070FA2078C4
:10121800FFF762FCBDE810400CF0C8BFC82E0020E4
:101228006419002010B5064C06480423237000F00A
:101238005EFA2078FFF750FCBDE810400CF0B6BF0E
:10124800C82E00206419002010B5064C0648032358
:10125800237000F04CFA2078FFF73EFCBDE8104000
:101268000CF0A4BFC82E00206419002010B5064C4D
:1012780006480223237000F03AFA2078FFF72CFC86
:10128800BDE810400CF092BFC82E00206419002061
:1012980070477047704770470E4A002310B51370A7
:1012A8000D4A0E4C13700AF08DFC05F0A5FB0AF0F0
:1012B80064FA0AF081FC20684FF6E07101F05CFEE8
:1012C8002068074901F006FE02F094FFBDE81040CF
:1012D80002F090BF3C0F0020DF0E0020DC0D002044
:1012E80041DA05080E4A012310B513700D4A00248F
:1012F80014700D4A204613700AF0FCF9204604F0D9
:10130800E1FB0A4B03221A700AF036FD0BF01DFAB6
:10131800074B08481C70BDE8104000F0E8B900BF52
:10132800C82E0020DF0E0020DD0E00203828002007
:10133800AC3A0020A013002038B50D4B0D4D002409
:101348001C700D4B28681C700C4B4FF6E0711C701C
:1013580001F012FE28680A4901F0BCFD02F04AFFBC
:10136800204604F0AFFB0748BDE8384000F0BFB99D
:101378003C0F0020DC0D0020DF0E00203828002064
:10138800E4DD0508081A002007B50E4B0E481A7848
:10139800D2F1010238BF00221A700C4B05221A70D4
:1013A80000F0A5F9022201238DE80C00B02060218D
:1013B800102232230DF082F803B05DF804EB02F03E
:1013C80019BF00BF3C0F0020581200203828002009
:1013D8002E4A002310B513702D4A13700CF0DEFC52
:1013E8000446002842D02B4C4FF6E071206801F0EB
:1013F800C3FD2068284901F06DFD60684FF6E07173
:1014080001F0BAFD6068254901F064FDA0684FF657
:10141800E07101F0B1FDA068214901F05BFD02F027
:10142800E9FE4FF47A600AF03DF820684FF6E07163
:1014380001F0A2FD20681B4901F04CFD60684FF6E1
:10144800E07101F099FD6068164901F043FDA0685C
:101458004FF6E07101F090FDA068124901F03AFDE5
:1014680002F0C8FEBDE8104002F0C4BE0CF054F90A
:10147800204604F027FB0C4B0C4804221A7000F09D
:1014880036F9BDE81040FFF75DB900BF3C0F0020FA
:10149800DF0E0020DC0D002051DA050865DA0508AA
:1014A80075DA0508E3DD0508382800208C150020CA
:1014B8002DE9F04F634DDFF8E89187B000244FF62F
:1014C800FF78284602F05DFC4146224623465E48E6
:1014D8000094019401F014FD4FF6E0760427039080
:1014E80031462246234659480097019401F008FDE9
:1014F80031462246234656480097019401F000FDE4
:1015080041462246234648460097019401F0F8FCDC
:10151800504E414630602246234648460097019483
:1015280001F0EEFC2346706041462246484600978B
:10153800019401F0E5FC4849B060484A204602F0B1
:10154800D7F94749474A0746204602F0D1F94649A4
:10155800464A8046204602F0CBF94549454A81462D
:10156800204602F0C5F94449444A8246204602F022
:10157800BFF943490490434A204602F0B9F920468E
:101588004149424A02F0B4F94149424A8346204659
:1015980002F0AEF94049414A84462046CDF808C0D9
:1015A80002F0A6F921460590039A2B46204602F040
:1015B800B7FA052132682B46A52002F0B1FA692155
:1015C80072682B46782002F0ABFA7D21B2682B4670
:1015D800782002F0A5FA1E213A462B46052002F093
:1015E8009FFA42462B464121052002F099FA6421D0
:1015F8004A462B46052002F093FA872152462B468D
:10160800052002F08DFAD2215A462B46602002F0BE
:1016180087FADDF808C0D22162462B46052002F081
:101628007FFAD221059A2B46B02002F079FA049A63
:101638004FF48070D2212B4607B0BDE8F04F02F07E
:101648006FBA00BF3016002085DA05088FDA050862
:101658009CDA0508DC0D0020A7DA050899120008B5
:10166800AFDA05089B120008B7DA05089D120008D2
:10167800BFDA05089F120008C7DA050841130008F9
:10168800CFDA0508A1120008D7DA0508D91300082F
:10169800DFDA050891130008E8DA0508ED120008FA
:1016A800E0DD050808B500F023FEFEF7A5FD00F013
:1016B8004FF800F06FF8FEF7AFFFFEF703FEFFF7F5
:1016C8008FF901F0E9FAFFF7F3FE00F0D5FFFEF716
:1016D80039FE01F03BF901F0DBF900F06DFB00F099
:1016E80081FD00F061FABDE8084000F02FBB10B59D
:1016F800044628B90F48104A104B532102F0A2FFA4
:101708000F4B1868844213D010B1C3690021984761
:10171800002004F0D7F9002004F0BEF94FF6FF705E
:1017280004F0A4F9E369204601219847044B1C60A2
:1017380010BD00BFF0DA0508641804080CDB0508C2
:10174800E80D00200048D2E7081A00200CF0EABA99
:1017580010B5084C204602F014FB00200649074A41
:1017680002F0C6F8D22102462346FA20BDE810400E
:1017780002F0D6B9C80F00202ADB05085517000863
:10178800024B034801221A70FFF7B1BF3828002026
:10179800301600202DE9F743374D384F384E0024D6
:1017A800284602F0EEFA2246234647F6FF713548EE
:1017B8000094019401F0A4FB4FF6FF78814641465E
:1017C8002246234638460094019401F099FB41468D
:1017D80030602246234638460094019401F090FB7D
:1017E800414670602246234638460094019401F031
:1017F80087FB2346B0604146224638460094019450
:1018080001F07EFB2049F060204A204602F070F883
:101818001F49204A0746204602F06AF821468046BA
:101828004A462B46204602F07BF93C2132682B467B
:10183800192002F075F95A2172682B46192002F016
:101848006FF97821B2682B46192002F069F99621C0
:10185800F2682B46192002F063F9D2213A462B464A
:10186800EC2002F05DF99C20D22142462B4603B0C1
:10187800BDE8F04302F054B9A0130020E0DD0508EC
:10188800EC0D00201CDB050829DB0508891700087A
:1018980032DB05085D1A000870B5474E474C3278B0
:1018A80047492DED028B142592B005FB02420C32FC
:1018B8000FA814F0DFFC33780D2B05FB03F504EBC0
:1018C800050332D8D3ED016A9B6807EE103A6359D5
:1018D800B8EEE68A06EE903ADFED3A7AF8EEC78A75
:1018E800B8EEE67A88EE278AC8EEA78AC7EE277A86
:1018F80017EE900A0FF084FE02460B4668463249FE
:1019080014F0B8FC18EE100A0FF07AFE02460B46E7
:1019180005A82E4914F0AEFC18EE900A0FF070FEE0
:1019280002460B460AA82A4929E093ED017A9B68EA
:1019380007EE903A635906EE903AF8EEE78AF8EE29
:10194800E67AB8EEC78A17EE900A0FF059FE0246FB
:101958000B4668461F4914F08DFC18EE100A0FF06C
:101968004FFE02460B4605A81B4914F083FC18EEEF
:10197800900A0FF045FE0B46184902460AA8184C73
:1019880014F078FC2068174901F0A4FA20680FA920
:1019980001F0A0FA6068694601F09CFAA06805A900
:1019A80001F098FAE0680AA901F094FA02F022FC22
:1019B80012B0BDEC028B70BDB628002000000020DC
:1019C8003BDB050800007A4446DB050857DB0508C1
:1019D80068DB050879DB05088ADB05089BDB050859
:1019E800EC0D0020E9DD050808B5124B124A1B78FA
:1019F8000D2B8CBF00210121117014225A430F496D
:101A080088588B184FF47A720D495043086059680A
:101A18004A430C490A609A680B4B1A6009F028FE81
:101A28000AF0CAF8094B0A4800221A70BDE80840B3
:101A3800FFF75DBEB6280020840F002000000020BC
:101A4800B8280020D82E0020AC2E002038280020EE
:101A5800081A0020C8E700BF4FF6FF7070474FF61E
:101A6800FF7070471FB5002947D04FF2DE7004F0B1
:101A780029F8002004F0FCF80F2003F0F7FF1F4CB2
:101A88001F4A412101230A2004F02AF9042004F006
:101A9800EFF8236828209621042B24DC0123194A17
:101AA80004F01EF903A90DF10E02206804F0A0FB52
:101AB8000F2003F0DBFFBDF80C00BDF80E10143842
:101AC8000F242822002380B2009403F0FFFFBDF802
:101AD8000E10BDF80C000094143989B22822012395
:101AE80003F0F4FF09E0084A012304F0F9F81E2086
:101AF800A521064A012304F0F3F81FBDFC0D0020C0
:101B0800ACDB0508BFDB0508DBDB0508F1DB0508F6
:101B180037B51E4C2368042B05462BDC01A80DF1B4
:101B2800060104F063FBBDF80630BDF8042018492F
:101B380004200CF019FE2368002B04DA1548164A15
:101B4800164B592105E0042B05DD1248124A144BA7
:101B58005A2102F077FD04EB8302BDF8041001332B
:101B68009180BDF806102360052BD18008D1201D77
:101B780004F0BEFB00230B482360FFF7B8FD03E029
:101B880028460121FFF76EFF3EBD00BFFC0D002077
:101B980008DC05084DDC0508761804086FDC050824
:101BA80086DC05087817002037B50B4C204602F074
:101BB800E8F80A4B0A49009300250120094A0A4B14
:101BC800019501F086FF294602462346284603B0C0
:101BD800BDE8304001F0A4BF441400206D1A00088D
:101BE800611A0008671A0008191B00084FF6FF70F1
:101BF80070474FF6FF70704730B54FF6E07087B00A
:101C080003F060FF002004F033F80F2003F02EFFEC
:101C180000212C4A2C4C01230A2004F061F80020F2
:101C280003F024FF042004F023F80A201921274A8E
:101C3800012304F055F82521254A01230A2004F040
:101C48004FF81F2003F012FF01230A203721214AF1
:101C580004F046F82378002B31D001231E2096216A
:101C68001D4A04F03DF862881C4902A814F002FBE2
:101C780001231E20A22102AA04F032F8A2881849E2
:101C880002A814F0F7FAAE2102AA01231E2004F0DC
:101C980027F80F2003F0EAFE6088A188143880B284
:101CA8000F2528220023009503F010FFA1886088E3
:101CB8000095143989B22822012303F007FF07B0E1
:101CC80030BD00BFB4DC0508140E0020C6DC0508D2
:101CD800E6DC050806DD050829DD05083BDD050805
:101CE80048DD050801B187E7704713B50DF1060116
:101CF80001A804F02FFA144B01221A705988BDF874
:101D08000420891A0E311C2919460AD89C88BDF866
:101D18000600201A0E301C2803D8996801319960F2
:101D280001E000238B60084B9968012905DD00223A
:101D38009A601A70FFF706FD05E05A80BDF8062084
:101D48009A80FFF759FF1CBD140E002037B50B4CC5
:101D5800204602F016F80A4B0A4900930025012094
:101D6800094A0A4B019501F0B4FE2946024623466A
:101D7800284603B0BDE8304001F0D2BE78170020F5
:101D8800ED1C0008F51B0008FB1B0008F31C0008ED
:101D980008B5064B00221A70054B186813F000FFAF
:101DA8000448BDE80840FFF7A2BC00BF382800205F
:101DB800A0380020081A00202DE9F04F514D524E4E
:101DC80085B00024284601F0DCFF2246234647F66A
:101DD800FF714E480094019401F092F84FF6FF7796
:101DE800039039462246234649480094019401F05D
:101DF80087F83946306022462346464800940194C5
:101E080001F07EF84FF001087060224623464FF635
:101E1800E0714148CDF80080019401F071F8234643
:101E2800B060394622463D48CDF80080019401F063
:101E380067F83B49F0603B4A204601F059FD3A49B2
:101E48003A4A0746204601F053FD3949394A804647
:101E5800204601F04DFD3849384A8146204601F0B8
:101E680047FD3749374A8246204601F041FD364949
:101E7800364A8346204601F03BFD21468446039AB4
:101E8800CDF808C02B46204601F04AFE3C213268B6
:101E98002B46142001F044FE3C2172682B46EC20AE
:101EA80001F03EFEB421B2682B460F2001F038FE47
:101EB800D2213A462B46E62001F032FE6421424602
:101EC8002B46052001F02CFE4A462B46052087218B
:101ED80001F026FE52462B460520D22101F020FEB5
:101EE800D2215A462B46502001F01AFEDDF808C0D0
:101EF8009B20D22162462B4605B0BDE8F04F01F089
:101F08000FBE00BF6C100020200E002055DD050814
:101F18005FDD050868DD0508DEDD0508E0DD05088C
:101F280029DB0508991D0008D8D80508811F000875
:101F3800E8D80508812000086BDD0508892100081C
:101F480073DD0508452100087BDD0508012100082F
:101F580008B50BF0F9FB4FF441400CF059F9044B6C
:101F6800186807F013F9034B09221A7008BD00BF5F
:101F7800B02800203828002010B50C4CFFF7E8FFE7
:101F88000B4A0023B420052103F0AAFEA0684FF6EF
:101F9800E07100F0F1FFA068064900F09BFF0BF02C
:101FA800D3FBBDE8104002F025B900BF200E002089
:101FB800E6DD050883DD0508264B2DE9F74318887B
:101FC800C00013F0E5FD054628B90520B421224AD2
:101FD8002B4603F085FE214BDFF878801D60002436
:101FE8000BF0B2FB26461E4FDFF8889023E009F07D
:101FF80097F93B68D9F8000045F8083C7B6845F834
:10200800043C184B1B68C01807F0C0F8164B18683A
:1020180009F048FAB8F8000094FBF0F080B24FF4E9
:10202800FC63009328210246322303F0ABFC04F53D
:102038009E7401360334B8F800300835B342D6DA56
:102048000A4B186807F0A2F8094B09221A70BDE874
:10205800FE8300BFA43C00209CDD0508A0380020BA
:102068006C3A00203428002064280020B028002082
:1020780038280020A838002010B5094CFFF79CFF2D
:10208800A0684FF6E07100F077FFA068054900F0FE
:1020980021FF0BF059FBBDE8104002F0ABB800BFC0
:1020A800200E0020AADD050810B5074C4FF6E07198
:1020B800A06800F061FFA068044900F00BFFBDE8CC
:1020C800104002F097B800BF200E0020C4DD0508BC
:1020D80010B5074C4FF6E071A06800F04DFFA068FE
:1020E800044900F0F7FEBDE8104002F083B800BFD5
:1020F800200E0020DADD050810B50C4C0B232370E8
:102108000B4B01221A70002002F0AAFF0948FFF7C2
:10211800EEFA2078FEF7E0FC074B032093ED000A67
:102128000BF021FBBDE81040D2E700BFC82E00200D
:10213800E00E002064190020D403002038B50C4DAF
:102148000C232B700B4B01241C70002002F088FF1D
:102158000948FFF7CCFA2878FEF7BEFC074B204663
:1021680093ED000A0BF0FFFABDE83840B0E700BF76
:10217800C82E0020E00E002064190020D40300209F
:1021880010B50C4C092323700B4B01221A70002048
:1021980002F066FF0948FFF7AAFA2078FEF79CFCD0
:1021A800074B022093ED000A0BF0DDFABDE8104062
:1021B8008EE700BFC82E0020E00E00206419002022
:1021C800D40300200BF070BE034A044800231370A8
:1021D800034A1370FFF78BBAAC3A0020081A0020A4
:1021E800382800202DE9F743384D394EDFF8FC80B8
:1021F8000024284601F0C5FD2246234647F6FF7114
:1022080034480094019400F07BFE4FF6FF77814636
:1022180039462246234630480094019400F070FE67
:10222800394630602246234640460094019400F027
:1022380067FE394670602246234640460094019462
:1022480000F05EFE2346B0603946224640460094C0
:10225800019400F055FE2149F060214A204601F022
:1022680047FB2049204A0746204601F041FB21460A
:1022780080464A462B46204601F052FC3C213268F3
:102288002B46282001F04CFC5A2172682B46192055
:1022980001F046FC7821B2682B46192001F040FC79
:1022A8009621F2682B46192001F03AFCD2213A46D1
:1022B8002B46EC2001F034FC0520D22142462B4667
:1022C80003B0BDE8F04301F02BBC00BFB4110020FF
:1022D800300E0020F4DD0508FCDD050829DB0508C3
:1022E800D121000807DE0508CD210008E0DD05083A
:1022F80010B50B4C204601F044FD00200146224653
:1023080000F05EFE00200749074A01F0F1FAD221E9
:10231800024623464FF48270BDE8104001F000BC2D
:10232800641900200FDE05085923000870B5C92478
:102338000AE0A8B200223146013502F021FDF02D55
:10234800F7D10134EF2C02D00025A6B2F1E770BD19
:1023580010B51A4C2378092B08D1194A0023137099
:10236800184A1370FFF7E2FF174823E00A2B0ED133
:10237800164B186813F014FC154A00231370114A01
:102388001370144A1370FFF7D1FF134812E00020AE
:1023980002F066FE114A00231360114A13800D4BA8
:1023A80002221A700F4B186806F0F0FE22780E4BC6
:1023B8000E481A70BDE81040FFF799B93828002078
:1023C800E00E0020DF0E00206C100020A038002056
:1023D800E10E0020AC3A0020B41100202C0F0020A0
:1023E8003A0F0020B02800205C280020FC120020B2
:1023F800034B01224FF4FC601A7003F037BB00BF97
:10240800DF0E002007B50A4A0023137004228DE866
:102418000C00C6201022232356210CF04FF8054B40
:1024280005480A221A7003B05DF804EBFFF75FB99C
:10243800DF0E002038280020B411002007B50A4A12
:102448000023137004228DE80C0097201022232308
:1024580056210CF033F8054B054809221A7003B0D1
:102468005DF804EBFFF743B9DF0E002038280020A1
:102478006C10002007B50B4B00221A7008220323AA
:102488008DE80C004920102223233D210CF016F87A
:10249800054B064801221A7003B05DF804EBFFF7FC
:1024A80026B900BFDF0E0020382800203016002093
:1024B80008B50A4B00201870094B1870094B082200
:1024C8001A70094B187003F0FDFA084B08480122EE
:1024D8001A70BDE80840FFF70AB900BF3C0F00209A
:1024E800DF0E002038280020C82E0020B838002031
:1024F800C80F002070B51F4C1F4E20684FF6E075BE
:10250800294600F039FD20681C4900F0E3FC6068AA
:10251800294600F031FD6068194900F0DBFCA0682D
:10252800294600F029FDA068164900F0D3FC01F007
:1025380061FE4FF47A6008F0B5FF2068294600F084
:102548001BFD2068314600F0C5FC6068294600F094
:1025580013FD6068314600F0BDFCA068294600F014
:102568000BFDA068314600F0B5FCBDE8704001F0F5
:1025780041BE00BF400E0020E3DD050851DA050822
:1025880065DA050875DA05080C4B10B500241C70CF
:102598000B4B01221A70204609F0ACF8204603F0D4
:1025A80091FA084B0B221A7009F0E6FB0AF0CDF8F5
:1025B8000548BDE81040FFF79AB800BFDF0E0020BD
:1025C800C82E002038280020D41600200F4A0023E7
:1025D80010B513700E4A13700BF0E0FB044628B1D7
:1025E800FFF788FFBDE8104001F004BE03F06AFA67
:1025F80009F0E8FA074B1C70074B07221A7009F01C
:10260800DBFA0648BDE81040FFF771B83C0F002020
:10261800DF0E0020C82E002038280020E8140020F3
:10262800104A002310B513700F4A13700BF0B6FB55
:10263800044628B1FFF75EFFBDE8104001F0DABD9F
:1026480003F040FA09F0BEFA06F0F8FD074B1C70DB
:10265800074B06221A7009F0AFFA0648BDE8104089
:10266800FFF745B83C0F0020DF0E0020C82E0020E1
:1026780038280020101100202DE9F04F674DDFF8B1
:10268800F09189B000244FF6FF78284601F079FBD5
:1026980041462246234662480094019400F030FCEB
:1026A8004FF6E076042703903146224623465D48DC
:1026B8000097019400F024FC3146049022462346FA
:1026C80059480097019400F01BFC414605902246AA
:1026D800234648460097019400F012FC534E4146A9
:1026E80030602246234648460097019400F008FCD3
:1026F800234670604146224648460097019400F000
:10270800FFFB4B49B0604B4A204601F0F1F84A49BB
:102718004A4A0746204601F0EBF84949494A8046AB
:10272800204601F0E5F84849484A8146204601F02C
:10273800DFF84749474A8246204601F0D9F846491A
:10274800464A8346204601F0D3F84549454A84461F
:102758002046CDF808C001F0CBF843490690434A1B
:10276800204601F0C5F821460790039A2B462046DB
:1027780001F0D6F92146049A2B46C82001F0D0F979
:102788000A21059A2B46C82001F0CAF9552132685A
:102798002B46782001F0C4F9692172682B4678200D
:1027A80001F0BEF9B2682B4678207D2101F0B8F916
:1027B8003A462B460520282101F0B2F9D22142469B
:1027C8002B46052001F0ACF9D2214A462B4656206B
:1027D80001F0A6F9D22152462B46A62001F0A0F915
:1027E800B4215A462B46052001F09AF9DDF808C0B5
:1027F800B42162462B46562001F092F9B421069A7C
:102808002B46A62001F08CF9079AF620D2212B46F8
:1028180009B0BDE8F04F01F083B900BF081A0020E5
:1028280014DE05088FDA05089CDA0508400E00203A
:102838001DDE05087D24000825DE05089125000811
:102848002EDE05082926000837DE0508D5250008EC
:1028580040DE0508B924000849DE050845240008BB
:1028680052DE05080D2400085BDE0508F923000880
:10287800E0DD050810B5064C4FF6FF71206800F042
:102888007BFB044B20681968BDE8104000F022BBB0
:102898004C0E00209402002008B5002003F012F925
:1028A800054B1868054B196800F014FB0448BDE88F
:1028B8000840FEF71CBF00BF4C0E0020900200200D
:1028C800301600200088A0F5C87080B2092808B525
:1028D80005D90848084A094B8C2101F0B3FE084B7A
:1028E8001880084BFF21197008F0E4FDBDE8084086
:1028F800C0E700BF62DE05088818040885DE050801
:10290800AC1A0020AE1A00200088A0F5967080B29C
:10291800092808B505D90848084A094B802101F05B
:1029280091FE084B1880084B0121197008F0C2FD70
:10293800BDE808409EE700BF62DE05089D18040850
:1029480085DE0508AC1A0020AE1A0020F7B5002471
:102958003348344D01F015FA224623464FF6FF71ED
:1029680031480094019400F0CBFA0426224623460D
:1029780007464FF6FF712D480096019400F0C0FA03
:102988002346286022464FF6FF7128480096019496
:1029980000F0B6FA26496860264A204600F0A8FFEB
:1029A800214606463A4620461D4B01F0B9F82A68EA
:1029B8001B4B2046282101F0B3F83246AA20D22129
:1029C800174B01F0ADF80F254FF4967440F2351609
:1029D80020461949194A00F08BFF01340246782134
:1029E80028460F4BA4B2233501F09AF8B442ADB291
:1029F800EED10F254FF4C87440F2991620461049BD
:102A0800104A00F075FF013402469B212846044B0A
:102A1800A4B2233501F084F8B442ADB2EED1FEBDC4
:102A2800C01800204C0E0020B6DE0508F1DD0508B0
:102A3800C2DE0508A1280008CBDE05081129000818
:102A4800CDDE0508CD28000808B5FFF713FF0020E4
:102A5800014608F02FFDBDE8084001F0CBBB00BFE0
:102A680007B5032308228DE80C00492010222323F0
:102A78003D210BF023FD044B044801221A7003B0DA
:102A88005DF804EBFEF733BE38280020301600202E
:102A98002DE9F743314E324F324D0024304601F0D4
:102AA80070F92246234647F6FF712F480094019497
:102AB80000F026FA4FF6FF78814641462246234623
:102AC80038460094019400F01BFA414628602246DB
:102AD800234638460094019400F012FA4146686093
:102AE8002246234638460094019400F009FA23460A
:102AF800A8604146224638460094019400F000FA46
:102B08001A49E8601A4A204600F0F2FE21460746B4
:102B18004A463346204601F003F83C212A683346EA
:102B2800192000F0FDFF5A216A683346192000F089
:102B3800F7FF7821AA683346192000F0F1FF9621A3
:102B4800EA683346192000F0EBFFEC20D2213A4620
:102B5800334603B0BDE8F04300F0E2BF581200204E
:102B6800E0DD0508540E0020CFDE050829DB050846
:102B7800692A00081C4B1A781C4B10B51A7009F00A
:102B880001F91B4B1B4A00241C6002202346CA2162
:102B980003F0A6F8204608F0ADFD174B1C80174B34
:102BA8001C70174B1B78023B052B1CD8DFE803F081
:102BB80003070B13170FBDE81040FEF757BBBDE81E
:102BC8001040FEF741BBBDE81040FEF72BBBBDE847
:102BD8001040FEF703BBBDE81040FEF711BBBDE88F
:102BE8001040FEF7E9BA10BD5C2800203828002004
:102BF8002C0F0020DFDD0508B4380020AC3A002097
:102C0800C82E002008B5084B186806F0BFFA002047
:102C180002F058FF09F0B0F8044B05480B221A706F
:102C2800BDE80840FEF763BDB02800203828002022
:102C3800D4160020114B10B500241C70104B1868D6
:102C480006F0A4FA204602F03DFF0E4B1B780B2B32
:102C58000ED8DFE803F006060D0D0D0D0A080D0D60
:102C68000D06094802E0094800E00948FEF73FFD63
:102C7800084B1C70BDE8104009F07EB8C82E002033
:102C8800B028002038280020081A0020E814002066
:102C980010110020AC3A00202DE9F041144C2046D8
:102CA80001F06FF800201349134A00F021FE134980
:102CB800134A0746002000F01BFE1249124A064636
:102CC800002000F015FED22105463A462346E620AC
:102CD80000F026FF4B2132462346642000F020FFF7
:102CE800642069212A462346BDE8F04100F018BF58
:102CF800FC1200204BD905083D2C0008D7DE05083A
:102D08000D2C0008E3DE05087D2B000808B508B186
:102D180043682BB90348044A044B9B2101F092FCF9
:102D2800586908BDF0DE0508B118040812DF050867
:102D380008B5FFF7EBFF8068123080B208BD08B510
:102D4800FFF7E4FF4068063080B208BD2DE9F84F70
:102D580004468846FFF7DAFF6689E589074606F1E3
:102D6800030905F10F0AB8F1000F1FD01F2002F068
:102D78007DFE2046FFF7DCFF83462046FFF7DFFF96
:102D8800294603465FFA8BF2F0B202F0AFFE042048
:102D980002F06EFF0B364FF6FF70033502F066FE49
:102DA800B0B2A9B23A68012302F09AFF3D69204601
:102DB80041464A465346A847BDE8F88F13B504462E
:102DC8000DF1060101A803F0C5F92046FFF79EFFA3
:102DD8006389BDF80410BDF80620C91AE389D21A20
:102DE8000339C3680F3A204698471CBDF7B5044617
:102DF80014200D4616461F4612F0CAFE089BC760EF
:102E08000361064B0649074A80E870000093019069
:102E1800054B002000F05DFEFEBD00BF552D0008EB
:102E2800472D0008392D0008C52D0008704708B542
:102E380008B143682BB90448044A054BAD2101F099
:102E480001FC586908BD00BF31DF0508C91804082E
:102E580012DF0508F8B505460E46FFF7E8FF836B55
:102E680004461BB128463146984700E018466F894A
:102E780094F83C30ED890EB9034310D0208E02F04F
:102E8800F5FD608E02F008FE94F8350002F0F0FEC1
:102E980094F8343038462946224602F021FF0023B0
:102EA80084F83C30F8BD08B5FFF7C1FF90F835004D
:102EB800BDE8084002F0F1BE38B5FFF7B8FF044698
:102EC80013F05EFA054694F8350002F0E1FE684317
:102ED80080B238BD38B50D46FFF7A9FF29462E2226
:102EE800044613F07DFA50B1204629462E2213F0ED
:102EF800C9FA002384F82E30012384F83C3038BD09
:102F08002DE9F743074640200E461546984612F02D
:102F18003FFE044628B91148114A124B4E2101F0D0
:102F280091FB114B114A12498DE818000020114BF2
:102F380000F0CFFD39468146FFF7CCFF9DF82830D9
:102F4800268684F835300B9B6586A363002384F8B6
:102F5800348084F83C304846BDE8FE8331DF0508FC
:102F6800E11804084FDF05085D2E0008AF2E0008A1
:102F7800C12E0008352E000810B50C46FFF757FF84
:102F88000123048680F83C3010BD00BF4FF4A070C8
:102F98007047C82070477047074B1B78022B07B54E
:102FA80008D1064B1B78022B04D001A80DF10601AD
:102FB80003F0D0F80EBD00BFAC3A0020C82E0020A8
:102FC80073B50A4B06460D4614460093002008497F
:102FD800084A094B019000F07CFD29460246234629
:102FE800304602B0BDE8704000F09ABD9F2F00083F
:102FF800952F00089B2F0008A12F000813B502ABDE
:1030080003E90600436843B1027C0124082A9C7046
:1030180004D11B692146984700E01C4620461CBD88
:1030280030B500282BD0058B002425E0036A1A7CD4
:10303800012A05D15B681A888A421BD1187F30BDE6
:10304800052A06D15B681A888A4213D193F82C00A6
:1030580030BD032A06D15B681A888A420AD193F8E0
:10306800250030BD062A05D15B681A888A4201D13D
:10307800D87A30BD01340430AC42D7D3002030BDFB
:1030880008B1817501207047F8B504460D46D0B1E6
:10309800E175D0F898309847012D0DD127460026C4
:1030A80006E0F86900F10802436906CA9847013644
:1030B800238B04379E42F4D3D4F89830204629460F
:1030C80098470120F8BDF8BDF8B5054608461746EB
:1030D8000E4613F055F9013FB84234BF04463C464A
:1030E8003CB128463146224613F0CCF900232B5533
:1030F800F8BD2C70F8BDF7B504460020009001908B
:1031080000296CD00E8B68E000F1080351F82330D9
:103118001D7C042D04D15D682D88954247D001306F
:1031280000F1080351F823301D7C012D04D15D689E
:103138002D8895423BD0013000F1080351F8233027
:103148001D7C052D04D15D682D8895422FD0013056
:1031580000F1080351F823301D7C032D04D15D686C
:103168002D88954223D0013000F1080351F823300F
:103178001D7C022D04D15D682D88954217D0013041
:1031880000F1080351F823301D7C072D04D15D6838
:103198002D8A95420BD0013000F1080351F82330F5
:1031A8001D7C062D08D15D682D88954203D103F159
:1031B8000801204615E0013000F1080351F82350BA
:1031C8002B7C082B09D16F683F88974204D105F101
:1031D800080120461A4605E00130B04294D3204643
:1031E8006946082212F084FF2046FEBDF8B5054660
:1031F8000F461646002830D04388032B2FD02020B6
:1032080012F0C6FC044600282BD040F80C5B394667
:103218000C22FFF759FF1820E66112F0B9FC0646A8
:10322800B8B102230374012363760F4B44606360D3
:103238000E4BA360002323766B8805EB83020133D2
:103248009BB2012B50606B800CD16A685268137670
:1032580008E0204612F0A4FC04E0064602E000263E
:1032680000E006463046F8BD2E980408CC940408C1
:1032780037B5456802AB03E906003DB3037C01247A
:10328800042B85F8314022D1688E02F0EFFB95F8C7
:10329800300002F0EDFC95F8343043B9BDF8020077
:1032A800BDF80610AA1C234602F01AFD0FE0012BF8
:1032B80003D1084840F2395104E0022B07D10548F0
:1032C80040F24151044A054B01F0BCF92C46204616
:1032D8003EBD00BF62DF0508A263040860DF050881
:1032E800F8B504460F46164610B3838A0A2B20D039
:1032F800202012F04DFC0546E8B14460102200F190
:1033080008003946FFF7E0FE4FF6FF73A08A2B80CE
:103318001F236B8000232B76831D013080B2012888
:10332800EE6144F82350A08207D1A3691876F8BD4E
:10333800F8BD0020F8BD0120F8BD0120F8BD2DE939
:10334800F3471D464B1C984282460C461746BDF86B
:1033580028600DDD95420BDC01320AF101035B1A8E
:10336800521BC8B2D2B29BB22946009602F0B6FBF5
:10337800AAF1020A3046C4EB0A0A02F077FB4FF0C2
:1033880000084FF001091FFA8AFA0BE0601C08EBED
:10339800050180B289B252460023009602F096FBDE
:1033A80009F101097B1B08F1010899451FFA88F802
:1033B800ECD3BDE8FC87F8B5C7B2144638461E46BC
:1033C8000D4602F095FB621E92B23846294602F07D
:1033D8008FFB304602F04AFB022606E0A21B92B29F
:1033E8003846294602F084FB0136A642F6D3F8BDDA
:1033F80073B504460E4600F11E00154600920023E0
:103408003C2280B21E3E02F061FBB1B220463C2253
:103418000123009502F05AFB7CBD73B504460E46A5
:103428000138154600920023032280B2013E02F0C3
:103438004DFBB1B2204603220123009502F046FB62
:103448007CBDF7B5089D2E7BEF7A1C463604AB7A17
:1034580006EB0726F618431A687B06EB00602D1862
:1034680000200190121B08462146009501F026FF16
:10347800FEBD30B5456885B004AB03E906007DB1F3
:1034880001242C736D68BDF80800BDF80A109DF87A
:103498000C209DF80E300095FFF7D3FF204600E082
:1034A800284605B030BD2DE9F04385B004AB03E9EB
:1034B80006004468BDF80860BDF80C70002C41D0C7
:1034C800012384F8263094F825300BB9A26800E06F
:1034D8006268FFB2BDF80A109DF80E3000923046BF
:1034E8003A46FFF7AEFF04F10C08022002F0C0FBD9
:1034F800404612F045FF054600B1451E0F3F002427
:10350800153E1FFA87F90DE002F0BCFB02F0C0FB84
:1035180004FB106189B248462022002302F0FAFB1E
:103528000134E4B2AC42EFD3002002F09FFAB8B203
:10353800B1B24246012302F0EDFB002002F098FBF5
:10354800012000E0204605B0BDE8F0832DE9F043F6
:1035580085B004AB03E906004568BDF80860BDF80E
:103568000C70002D3CD001236B762B7EBDF80A1021
:10357800012B0CBF6A68AA689DF80E300092FFB252
:103588003A463046FFF75DFF0C35022002F070FB2B
:10359800284612F0F5FE0E3F81460024163E1FFA1B
:1035A80087F80DE002F06EFB02F072FB04FB10617D
:1035B80089B240462022002302F0ACFB0134E4B279
:1035C8004C45EFD9002002F051FAB8B2B1B22A4600
:1035D800012302F09FFB002002F04AFB012000E0DB
:1035E800284605B0BDE8F0832DE9F04F85B00546C3
:1035F800DDF84090029148469046039312F0C0FED1
:10360800DDF838A0DDF83CB00646294600242F46F0
:1036180011E024B1B4420CBF5B46534600E0039B63
:1036280001F10805ADB200932846029A4346FFF718
:1036380008FF01342946B442EBDD002002F016FAF7
:10364800022002F015FB7D1D08F10508A8B21FFA3B
:1036580088F14A46012305B0BDE8F04F02F040BBAF
:1036680070B5406886B006AB03E9060000282ED086
:10367800012380F82D308668164BF21A534243EB2B
:10368800020390F82C205AB1002B134D134B144A07
:1036980008BF1D46134B00F11C0418BF13460AE06F
:1036A800002B0D4D0D4B0E4A18BF1D460D4B00F15A
:1036B8000C0408BF1346BDF81200BDF81410BDF87D
:1036C8001620009601950294FFF78EFF012006B0A0
:1036D80070BD00BF126D04084E690408F46E04083A
:1036E800306B0408D670040870B5446886B006AB21
:1036F80003E9060004B301236377A668104B227F11
:10370800F11A4B4243EB01030AB10BB904E01BB9B0
:1037180066680C4D0C4B01E00C4D0D4BBDF81200CA
:10372800BDF81410BDF8162000960C3401950294CB
:10373800FFF75AFF012000E0204606B070BD00BF29
:103748005E7804089A7404087C760408347A0408BD
:103758000A7C04082DE9F04385B004AB03E90600B0
:103768004468BDF80860BDF80A90BDF80C50BDF873
:103778000E80002C00F08C800123A374022067685F
:1037880002F076FA4FF6FF7002F086F9002002F098
:103798006DF9EDB25FFA88F8A6F1160189B23046E4
:1037A8002A4643460097FFF74CFE277A002F2ED172
:1037B800A28A234600E00137974204D29969097E1C
:1037C80004330029F7D002F05DFA02F061FAA9F19A
:1037D80016091FFA89F90E2101FB10914FF6FF72A5
:1037E80008F101085FFA88F389B2009248462A4630
:1037F800FFF7A5FD022002F03BFA1F2002F036F980
:10380800A38A002B38D0103DE8B2303E2CE0E368A4
:103818005C68A28A2346013A002700E001379742F4
:1038280004D29969097E04330029F7D002F02AFAF4
:1038380002F02EFA0E2101FB10914FF6FF7208F1EB
:1038480001085FFA88F389B2009248462A46FFF7D2
:1038580076FD022002F00CFA1F2002F007F9A38A75
:1038680053B1103DE8B21A3E0637B1B254F82720DA
:103878000123083202F04EFA002002F0F9F94FF65F
:10388800FF7002F009F91F2002F0F0F8012000E0B3
:10389800204605B0BDE8F0832DE9F0410546362005
:1038A800884614461F4612F073F90646E0B120F820
:1038B800025B41462E22FFF707FCBDF8183086F858
:1038C800344073861820012386F8307086F831302A
:1038D80012F05EF9044618B104234660037404E04C
:1038E800304612F05DF900E004462046BDE8F0815C
:1038F800F8B5064624200F46154612F049F9044645
:10390800D8B10F4B068083600E4B394643601022B6
:1039180000F10C00FFF7D8FB0126002318202562D0
:103928002377667712F034F9054610B144600674BF
:1039380004E0204612F034F900E005462846F8BDB8
:103948005E780408B8720408F8B506462C200F46BD
:10395800154612F01DF90446E8B120F80C6B3946FB
:103968001922FFF7B1FB0D4BA562A3600C4B6360F6
:10397800002384F825301820012384F8263012F01B
:1039880007F9054618B103234460037404E0204690
:1039980012F006F900E005462846F8BD6A910408C9
:1039A800088E040810B50446142012F0F1F820B16E
:1039B80000234380014B0480036110BDF5310008EA
:1039C80038B50546442012F0E3F80446C0B10E4B62
:1039D800058243600D4B0360012383740023037247
:1039E80083820B4B0364182012F0D2F8054618B1F5
:1039F80007234460037404E0204612F0D1F800E085
:103A08000546284638BD00BFFE890408F485040829
:103A1800E93200082DE9F04105463420884614466D
:103A28001F4612F0B5F8064620B3144B0580836094
:103A3800134B41464360102200F10C00FFF744FB92
:103A4800214606F11C001022FFF73EFB002386F8F2
:103A58002C3018200123376386F82D3012F098F89F
:103A6800044618B105234660037404E0304612F09A
:103A780097F800E004462046BDE8F081126D04087E
:103A88006C6704082DE9F041044614200D461646DB
:103A9800984612F07DF80746B8B1069B048003618A
:103AA8000023C37201234560068180F80A800373EE
:103AB800182012F06DF8044618B106234760037405
:103AC80004E0384612F06CF800E004462046BDE8F1
:103AD800F0812DE9F041044618200D461646984617
:103AE80012F056F80746B8B101238370069B04808C
:103AF8000361079B45608660C0F80C80436118200D
:103B080012F046F8044618B108234760037404E02D
:103B1800384612F045F800E004462046BDE8F0813A
:103B28002DE9F34198461B8B1D2B05460C4617467D
:103B38004FF0000000F2B480B5F5A07F009001902E
:103B480000F2AE80F02900F2AB80127CADF80610CE
:103B5800511EADF80250072900F28A80DFE801F013
:103B680045595E04456A14767B684E4A7A611A881C
:103B780093F834303A80013BDBB2012B7FD8ADF8A3
:103B88000240ADF806507AE005F11602ADF80020C3
:103B980004F11602ADF8042002AE434A16E9030008
:103BA8007A6107F1080282E8030003F10802013391
:103BB80048F82270A8F818307B681A8A187A3A8070
:103BC80000286CD1FFF7FCFE384943685960384932
:103BD800DF600126163D196002461E72A8B2E1B2E6
:103BE8004346FFF79DFF30465AE0012A0CBF314B90
:103BF800314B78687B6130F80C3B3B8012F0C0FB9E
:103C0800431CDB001A34ED18ADF80440ADF8005041
:103C180035E07B68294A1B687A6102E0284A7B689C
:103C28007A611B8814353B80ADF800501434ADF828
:103C3800044024E07B68234A7A611A883A801A890A
:103C48009B7AAD18ADF80050E418F0E77E681E4B7B
:103C58007B61338838463B8073689847013D451936
:103C6800ADF80050B36838469847013C0419DEE7C0
:103C78001648174A174B40F21A3100F0E3FC02AA23
:103C880012E9030007F1080383E80300B8F81830C5
:103C980003F10802013348F82270A8F8183001200F
:103CA800BDE8FC81793200085D370008EA81040824
:103CB800E07D0408F136000869360008553500082B
:103CC800AF3400087B3400080530000862DF0508BF
:103CD800B263040860DF0508F8B51646002834D03A
:103CE8001378002B2ED0028B002327E0046A257C52
:103CF800042D21D165682F888F421DD195F8313068
:103D080053B16F8E01F0D8FE04F10802688663692A
:103D1800204606CA98476F86A81C31462E22FFF710
:103D2800D3F995F831307BB104F108026369204674
:103D380006CA98470120F8BD013304309342D5D311
:103D48000020F8BD1846F8BD0120F8BD70B5B8B11F
:103D5800068B0446002310E0256A287C04280AD133
:103D68006D682888884206D11046A91C2E22FFF7C4
:103D7800ABF9012070BD01330434B342ECD3002009
:103D880070BD38B5044620B3134BC361134BC0F85C
:103D98009830134BC0F89C30124B00257822C0F89D
:103DA800A0308575C5750583294600F1200012F0FD
:103DB800E1F9D4F898302046294698470A4A1388EA
:103DC800312B07D8094941F82340013313800120DA
:103DD80038BD38BD284638BD913000088930000804
:103DE80029300008FF300008640E0020B01A0020B7
:103DF8002DE9F0410446002800F0B380078B024605
:103E08000025A8E0136A1E7C042E00F08780012E8E
:103E180023D1586803888B4240F09B8005F108073E
:103E280011F0BEFE54F827004FF00008C0F80480D7
:103E380011F0B6FE228B531E9D4208D00732238311
:103E480054F8221044F8271044F8228002E044F87D
:103E5800278025833046BDE8F081052E5ED0032EED
:103E68005CD0022E13D15B68186803888B4270D12E
:103E78004388013B9BB243800BB911F091FE05F1D9
:103E8800080654F82630586811F08AFE4EE0072ECE
:103E980021D15E68338A8B425BD1002706E0BB1DC7
:103EA800013756F8230011F07BFEFFB2B38ABB42FC
:103EB800F5D80027B78205F1080654F82630586867
:103EC80011F06EFE54F8260033E044F8267025837E
:103ED8000120BDE8F081062E1ED1586803888B4268
:103EE80037D105F1080611F05BFE54F826000027CB
:103EF800476011F055FE228B531E9D4209D00833AE
:103F0800013A54F82310228344F8261044F8237009
:103F1800DEE744F826701AE0082E1AD1586803889C
:103F28008B4216D111F03CFE05F1080654F8260024
:103F38000027476011F034FE228B531E9D42C4D0E7
:103F4800073254F8221044F8261044F822702383CC
:103F5800BEE701350432BD42FFF454AF0020BDE88E
:103F6800F081BDE8F08170B5044600282AD0068BA0
:103F7800751E083600EB86061EE056F8043D1A7CCE
:103F8800042A13D0012A11D0052A0FD0032A0DD0F4
:103F9800022A02D15B681B6809E0072A02D15B6824
:103FA800198A05E0062A01D0082A04D15B68198815
:103FB8002046FFF71DFF013D681CDED10023238347
:103FC800012070BD70BDF0B528B30023068B1A46DA
:103FD8001EE0046A257C072D18D16468258A8D4265
:103FE80014D1A78A002504EB83040DE004EB050C2B
:103FF8000435DCF818C09CF818C0BCF1010F03F1B7
:10400800010301D1D8B2F0BDBB42EFD30132043075
:10401800B242DED30020F0BD70B508B3048B002394
:104028001BE0026A157C072D15D15268158A8D424E
:1040380011D10023958A11461C46012007E013B9C7
:104048009669307601E08E69347601330431AB42EB
:10405800F5D3012070BD01330430A342E1D3002021
:1040680070BD2DE9F04128B30023078B1A461EE0E6
:10407800046A257C072D18D16468258A8D4214D1DD
:10408800B4F814C0002504EB83040CE06619043569
:10409800B66996F81880B8F1010F03D106F1080047
:1040A800BDE8F08101336345F0D301320430BA42F0
:1040B800DED30020BDE8F0812DE9F04700282FD09D
:1040C8000023B0F818C01D4627E0046A267C072E96
:1040D80021D16468268A8E421DD1B4F81480002646
:1040E80004EB830915E009EB0604A7693C7E012C63
:1040F8000DD192F800A0BAF1000F08D007F108001E
:1041080011461022FEF7E0FF2046BDE8F087013394
:1041180004364345E7D3013504306545D5D300203F
:10412800BDE8F087F0B5B0B1068B002510E0046A51
:10413800277C062F0AD1646827888F4206D12381FD
:104148009DF814306260A3720120F0BD013504307F
:10415800B542ECD30020F0BD10B500210446FEF7AF
:1041680093FF20460121BDE81040FEF78DBF38B50A
:1041780098B1048B024600230CE0106A05880432CB
:104188008D4206D100F10802436906CA984701200A
:1041980038BD0133A342F0D3002038BD10B50C461A
:1041A8000021FEF771FF20460121BDE81040FEF70F
:1041B8006BBF13B502AC04E90C00BDF802308342B2
:1041C80006D8BDF80030834234BF0020012000E04B
:1041D8000020BDF806308B4206D8BDF804308B426B
:1041E80034BF0021012100E00021002818BF084643
:1041F800C0B21CBD38B5114B114A1988002319E00B
:1042080052F8045FA87D012812D100240CE004F1C3
:10421800080355F82300037C082B03D143680021C9
:104228001B6998470134A4B22B8BA342EFD838BD41
:1042380001339BB28B42E3D138BD00BF640E00202E
:10424800AC1A0020704770B5094CA5787DB9094BA8
:104258001E78012E0BD16368013363606268064BD8
:104268009A4204D9284601F0C5FCA670656070BD65
:10427800640E00208401002040420F00054A90602F
:10428800134602E099680139996091680029F9D1CB
:10429800704700BF640E0020F0B585B001F058FFEC
:1042A800002800F04981002502A80DF10A01ADF8A7
:1042B8000850ADF80A5001F04DFF03A80DF10E01AA
:1042C800ADF80C50ADF80E5001F090FFBDF80C1091
:1042D800BDF808200091BDF80E10BDF80A30019114
:1042E8002C46964D964908200AF03EFAA8780128EF
:1042F80003D101F07FFCAC7019E1924B5B78012B84
:1043080040F01581AB78002B40F011816B60298853
:104318008D4A09E152F8046FB07D012840F002810E
:104328000025FAE005F10803BDF8080056F8234017
:10433800BDF80A1004F108030CCBFFF73AFF002878
:1043480000F0E980237C013B062B00F29F80DFE828
:1043580003F00429159D1F9D4C006668012304F194
:104368000805337795E806006369204698470023D7
:1043780033772046636995E8060086E0636893F81A
:10438800252012F1FF3218BF012283F8252077E09B
:10439800636893F82C2012F1FF3218BF012283F8CA
:1043A8002C206DE06268137E1568002B6ED16E8834
:1043B8002F462946184606E051F804EFDEF804E0D7
:1043C80001338EF81800B342F6D301231376002682
:1043D80007E057F8040F00F10802436906CA984736
:1043E80001366B889E42F4D350E0656820892E68B8
:1043F800A37B227B0096A0F1160189B2FFF721F872
:104408001420FFF73BFF2B7AC3B9AF8A29461A4617
:104418001E4609E0886990F818E00676BEF1010F9B
:1044280008BF134604310132BA42F3D301220BB953
:10443800AB6924E0053355F8233020E06368DB6876
:104448005A680023908A154619461F4609E0AE6946
:1044580096F818E03776BEF1010F08BF0B46043511
:1044680001318142F3D3411E8B4203D1053052F80A
:10447800203003E004D2073352F8233001221A76A1
:1044880004F1080206CA636920469847237C013B69
:10449800072B4CD8DFE803F00410074B0A0D123A3B
:1044A80063681B6A34E063689B6A2DE063681B6B72
:1044B8002AE063681B6927E0636824E063681A7A66
:1044C8007AB9988A1946013800E00132824204D24A
:1044D8008C69247E0431002CF7D0063253F8223040
:1044E80011E0DB685A68908A11460138002300E021
:1044F8000133834204D28C69247E0431002CF7D026
:10450800063352F82330DB69984710E06368DB68AC
:10451800204698470BE00135ADB2338BAB423FF6EE
:1045280001AF04E001339BB28B427FF4F3AE01F09C
:1045380055FE0F20FFF7A2FE05B0F0BD640E002067
:1045480088DF050884010020AC1A0020034B9A6814
:1045580012B19A68013A9A60704700BF640E002051
:104568002DE9F3470120DFF8D080DFF8D09001462D
:104578000BF094FC012400254FF480760227404676
:10458800694600968DF804708DF805408DF8065040
:104598008DF807400BF0DAF84046082122460BF068
:1045A80055F9244BDFF898801A6844F2A243B2FB0D
:1045B800F3FA0AF1FF3A204621461FFA8AFA0BF06D
:1045C8009DFCC8F804A048464146A8F80050A8F841
:1045D8000250A8F8085088F80A500CF02BF87023FD
:1045E800A8F80C300423A8F810300AF1FF3A632326
:1045F800642203FB0AF3B3FBF2F39BB2C8F814304E
:1046080008F10C014846A8F80E40A8F81870A8F858
:104618001A50A8F81C60A8F81E500CF029F9484652
:1046280021460CF09CF8484621460CF0A2FBBDE858
:10463800FC8700BF980200200000024000000140F3
:10464800740E002083B50E460746154910201C46F7
:1046580015460AF089F8102012490AF085F810204A
:1046680011490AF081F810200E490AF07DF800235C
:1046780010200E4901930AF077F8334610200C49B0
:104688003A460AF071F810200A492A460AF06CF8EE
:104698001020094922460AF067F8019B0133E7E731
:1046A800C2DF0508C7DF0508E7DF0508F7DF0508EB
:1046B80007E005081CE005082DE0050808B5164BBD
:1046C8001A6A01321A621A6A012A1A4603D0134872
:1046D80040F21E210FE05862194602E04B6A013B86
:1046E8004B62506A0C4B0028F8D11A6A012A06D08E
:1046F8000A4840F229210A4A0A4BFFF7A3FF1A6A1F
:10470800013A1A621B6A2BB10448054A064B40F26B
:104718002B21F2E708BD00BF740E00203EE005081B
:10472800909B040868E0050879E0050810B5084C76
:104738000221002220460BF07EF844F6FF70FFF7B6
:10474800BDFF204602210122BDE810400BF073B8DE
:10475800000402400C4B0D491A6844F2A243642835
:10476800B2FBF3F3D4BF20EAE0706420013B9BB2B4
:104778004B60013B58436422B0FBF2F080B24861C1
:1047880003480C310BF0F7BF98020020740E00208C
:104798000000014010B5134B93F828202AB11248A5
:1047A800124A134B40F209310EE0012283F8282007
:1047B80066234FF0C042013BDBB2108033B90A4890
:1047C8000A4A0C4B40F21331FFF73CFF1488A4B29D
:1047D8008442F0D1084B1980024B002283F828202C
:1047E80010BD00BF740E00203EE005089A9B040827
:1047F8008AE0050860DF05080000026010B5FFF7D1
:10480800AFFE6420FFF7A6FF21210720FFF7C2FFB4
:104818003220FFF753FF01210020FFF7BBFF3220B2
:10482800FFF74CFF23210720FFF7B4FF3220FFF7E3
:1048380045FF00211020FFF7ADFF41F28830FFF758
:104848003DFF33210720FFF7A5FF3220FFF736FF92
:10485800112046F63001FFF79DFF3220FFF72EFFAB
:104868004FF4C0610220FFF795FF3220FFF726FFC3
:10487800122046F6EB41FFF78DFF3220FFF71EFFAF
:1048880003204AF6A401FFF785FF3220FFF716FF41
:1048980000210C20FFF77EFF3220FFF70FFF0D20CD
:1048A80040F60C01FFF776FF3220FFF707FF0E20D6
:1048B8004FF42C51FFF76EFF3220FFF7FFFEB021B7
:1048C8001E20FFF767FF3220FFF7F8FE012042F6AF
:1048D8003F31FFF75FFF3220FFF7F0FE0520002190
:1048E800FFF758FF3220FFF7E9FE00210620FFF707
:1048F80051FF3220FFF7E2FE16204EF61C71FFF73B
:1049080049FF3220FFF7DAFE172040F20311FFF7C4
:1049180041FF3220FFF7D2FE00210B20FFF73AFFBC
:104928003220FFF7CBFE00210F20FFF733FF3220A4
:10493800FFF7C4FE41200021FFF72CFF3220FFF7CC
:10494800BDFE42200021FFF725FF3220FFF7B6FE0B
:1049580000214820FFF71EFF40F23F143220FFF7E6
:10496800ADFE21464920FFF715FF3220FFF7A6FECE
:1049780000214A20FFF70EFF3220FFF79FFE00219B
:104988004B20FFF707FF3220FFF798FE44204FF433
:104998006F41FFF7FFFE3220FFF790FE0021452010
:1049A800FFF7F8FE3220FFF789FE21464620FFF781
:1049B800F1FE3220FFF782FE302040F20771FFF748
:1049C800E9FE3220FFF77AFE31204FF40171FFF73C
:1049D800E1FE3220FFF772FE32204FF40171FFF73B
:1049E800D9FE40F202543220FFF768FE21463320F8
:1049F800FFF7D0FE3220FFF761FE342040F2075166
:104A0800FFF7C8FE3220FFF759FE35204FF4017139
:104A1800FFF7C0FE3220FFF751FE36204FF4017138
:104A2800FFF7B8FE3220FFF749FE21463720FFF78F
:104A3800B1FEA4F500743220FFF740FE21463A206B
:104A4800FFF7A8FE3220FFF739FE2F2041F2BE21E2
:104A5800FFF7A0FE3220FFF731FE21463B20FFF78B
:104A680099FE3220FFF72AFE00212320FFF792FE4D
:104A78003220FFF723FE00212420FFF78BFE32208F
:104A8800FFF71CFE25204FF40041FFF783FE32207C
:104A9800FFF714FE00214F20FFF77CFE3220FFF7BE
:104AA8000DFE4E200021FFF775FE3220BDE81040B4
:104AB80004E608B5124B93F829202AB11148124A86
:104AC800124B40F223310FE0012283F829202221E2
:104AD80066234FF0C042013BDBB2118033B909486D
:104AE800094A0B4B4FF44F71FFF7ACFD108880B2A9
:104AF8002228F0D1024B002283F8292008BD00BFEC
:104B0800740E00203EE00508A79B04088AE005080B
:104B180060DF050810B51E4B032826D8DFE800F033
:104B2800021A080E1C8841F2280246F628000AE0FC
:104B38001C8841F2080246F6080004E01C8841F28D
:104B4800300246F6300049F241318C4214BF01462A
:104B580011460BE0188846F6200249F24131884296
:104B680014BF11464FF4815100E000211B8848F61C
:104B78008912934205D049F22032934204D103208E
:104B880000E01120FFF706FEBDE8104091E700BFE6
:104B980086010020014B18800A208FE50000026082
:104BA8004FF0C043188003F500331A881A88188814
:104BB80080B270474FF0C04322221A8003F50033B9
:104BC80082B01A8892B2ADF806201B889BB2ADF865
:104BD8000630BDF8060080B202B07047072040F2E8
:104BE8007311D7E507200021D4E582B0044BADF856
:104BF8000600BDF8062092B25A8502B0704700BF81
:104C0800740E002082B0044BADF80600BDF80620F3
:104C180092B25A8002B0704786010020014B80B2E0
:104C280018807047000002604FF0C04380B21880BF
:104C38007047024B80B21880704700BF00000260C6
:104C48004FF0C04380B218807047024B80B2188082
:104C5800704700BF0000026082B0044B0190019AC7
:104C6800DA62DA6A002AFCD102B07047740E0020BA
:104C780070B54FF0C0452A242C800A4C060AC0B2F1
:104C880026802080100AD2B2208022802B222A80FF
:104C98000A0A2280C9B21A0ADBB221802280238044
:104CA80070BD00BF0000026010B50B4614460246F6
:104CB800FFF7DEFF4FF0C0432C22A0B21A80BDE8F8
:104CC800104067E7114B1B8848F68912934210B5CC
:104CD80004460BD049F22032934212D1C1F1EF01C0
:104CE800202089B2FFF756FD212006E0C1F1EF012F
:104CF8004E2089B2FFF74EFD4F202146BDE81040F7
:104D080048E502460B46BDE81040B1E786010020A1
:104D180008B5FFF7D7FF0F4B1B78012B4FF0C042A8
:104D28000D4B0FD12E2111801A881A881B8892B238
:104D380002F0FC0002F4784242EAC000C3F3C42344
:104D4800184308BD222111801A881A88188880B251
:104D580008BD00BF801B00200000026070B5074D31
:104D68000646012421463046FFF7D2FF0134A4B29B
:104D7800C82C25F8020FF5D170BD00BFAE3A00204F
:104D880010B5084B1B78012B144602D1BDE8104022
:104D98008AE7FFF797FFFFF78CFE2046BDE8104033
:104DA800F8E600BF801B002070B5074D06460124B9
:104DB8002146013435F8022F3046A4B2FFF7E0FF50
:104DC800C82CF5D170BD00BFAE3A002070B50546BD
:104DD8000E46FFF7C3FF0124214601342846324618
:104DE800A4B2FFF7CDFFC82CF6D170BD2DE9F04174
:104DF80004460D461646BDF81880032B39D8DFE85F
:104E080003F00B351927381980B229464246013775
:104E1800FFF7B6FFBFB200E00027B742F3D1BDE805
:104E2800F081E01B80B2294642460137FFF7A8FF10
:104E3800BFB200E00027B742F3D1BDE8F081E91B1B
:104E480089B2204642460137FFF79AFFBFB200E019
:104E58000027B742F3D1BDE8F081791989B220461D
:104E680042460137FFF78CFFBFB200E00027B74288
:104E7800F3D1BDE8F08170B5194B1A4A598E92F9F1
:104E8800004064180025A4B28AB0AC4208BF0124CF
:104E9800C62C28BFC62415700F264FF6FF721E8633
:104EA8005C865A8519202B46009221460A22FFF774
:104EB8009DFF21463046FFF72BFF224603460A494D
:104EC80002A811F0D7F902AA06A8084911F0D2F9E8
:104ED8003220D22106AA2B4600F002FF0AB070BD8C
:104EE800740E0020ED1B00209FE00508A7E00508D0
:104EF8002DE9F341BDF820500C4690461F461A464E
:104F0800002306460095FFF771FF611E41443046B5
:104F18003A46002389B20095FFF768FF30462146DC
:104F2800424601230095013EFFF760FFBF19B8B262
:104F3800214642460123089502B0BDE8F04155E7F5
:104F48002DE9F0410D46C5F1F008411E5E18C2EB8F
:104F58000802C5F1EF039BB292B2B6B29A422CBFD7
:104F6800904698469A4234BF11461946864234BF45
:104F78003746074640F23F13864238BF06469E42F0
:104F880028BF1E46174B1B8848F68912B8F1EF0F49
:104F980028BF4FF0EF089342044610D049F2203260
:104FA80093421AD15020FFF7F5FB51204146FFF7F5
:104FB800F1FB52203946FFF7EDFB53200AE041EAA6
:104FC800082189B24420FFF7E5FB45203946FFF761
:104FD800E1FB46203146FFF7DDFB20462946BDE8C8
:104FE800F0416FE68601002000200146F0224FF4D0
:104FF800A073A5E770B580B202FB03F489B292B240
:105008009BB2FFF79DFF0020FFF784FD0025064EA9
:1050180004E0708D80B2FFF7BDFD0135A542F8DBD5
:10502800BDE87040E0E700BF740E002070B54FF097
:10503800C0452A242C80094C060A26802080080AAC
:10504800208021802B212980110A218022801A0AA0
:10505800228023802C232B8070BD00BF00000260BB
:1050680070B5114B1B78012B044607D1002040F284
:105078003F110246EF23FFF7D9FF04E0FFF7B4FF23
:105088000020FFF747FDF02509E0013E2046B6B2B3
:10509800FFF780FD002EF8D1013DADB215B14FF4F8
:1050A800A076F2E770BD00BF801B00202DE9F04F0D
:1050B8001C463E4B87B01B78039183469DF84410ED
:1050C80010980591012B039B049092461FFA8BF0D0
:1050D8009AB208D1411E531E0919534489B29BB292
:1050E800FFF7A4FF09E01FFA8AF51146A3B22A4682
:1050F800FFF726FF0020FFF70DFD0027DDF80C80E5
:105108003E4640F23F1CA14639E0BBF1000F2EDBC2
:1051180065452CDC0398002829DBB8F1EF0F26DC65
:10512800220702D1002CC8BF01362149214000299D
:1051380003DA013961F00F010131059A0AB1C1F1B1
:105148000F01049830F8162003FA01F10A4012B250
:105158006AB118494A8D029392B2A8B21FFA88F12F
:10516800CDF804C0FFF70CFEDDF804C0029B013443
:1051780001354C45C9DB0136013708F101085745AF
:1051880003DA5D4600240123F3E7084B1B78012B63
:1051980008D1002040F23F110246EF2307B0BDE8D6
:1051A800F04F43E707B0BDE8F04F1DE7801B002034
:1051B8000F000080740E00202DE9F74F1F463B4B6F
:1051C800DDF830801B7816469DF83420012B044604
:1051D80001920D4680B28AB208D1411E531EC919E8
:1051E8009B1989B29BB2FFF721FF09E01FFA86FEDF
:1051F8001146BBB27246FFF7A3FE0020FFF78AFCF8
:105208004FF0000BDA463DE0002C30DB09EB0403DD
:1052180040F23F1293422ADC002D28DB0BEB0503FA
:10522800EF2B24DC19F00F0F04D1B9F1000FC8BF20
:105238000AF1010A1E4B09EA0303002B03DA013BBA
:1052480063F00F030133019A0AB1C3F10F0301227E
:1052580002FA03F338F81A2013401BB213B1154BA6
:10526800588D01E0144A508880B2FFF793FC09F189
:10527800010901E04FF00009B945C5DB0AF1010A4F
:105288000BF1010BB345F5DB084B1B78012B08D15B
:10529800002040F23F110246EF2303B0BDE8F04F73
:1052A800C4E603B0BDE8F04F9EE600BF801B0020B7
:1052B8000F000080740E0020860100202DE9F041C7
:1052C8001C4F069C3F789DF81C60012F02FB03F5DC
:1052D80080B28FB209D1411ECB1899B27B1E9A18A1
:1052E80093B23A46FFF7A2FE07E092B29BB2394664
:1052F800FFF726FE0020FFF70DFC002709E034F831
:10530800020B1EB1030A43EA002080B2FFF742FCF9
:105318000137AF42F3DB074B1B78012B07D1002085
:1053280040F23F110246EF23BDE8F0417EE6BDE8BA
:10533800F04159E6801B00202DE9F0431F2093B06F
:10534800FFF78EFE4FF47840FFF78AFE4FF6E075C0
:105358004FF4FC60FFF784FE2846FFF781FE00202B
:10536800514CFFF77DFE00204FF6FF79014664227D
:105378000346A4F82A90CDF80090FFF737FD0020E7
:105388000A2164220346CDF80090FFF72FFD002084
:105398000146642201234FF4784765850095FFF79D
:1053A80025FD7720EF21C82200234FF4FC6667858E
:1053B8000097FFF71BFDBD213222012340F23F1069
:1053C80066850096FFF712FDA0203222002378217F
:1053D80067850097FFF70AFDA02078213222012374
:1053E8004FF01F0866850096FFF700FDA020782182
:1053F80032220223A4F82A80CDF80080FFF7F6FCB9
:10540800A02078213222032365850095FFF7EEFC62
:10541800264B2749A3F8028002AD3C22284610F00B
:1054280067FEEB20C3210522302300950025A4F850
:105438002A900195FFF7C0FE32210A2096220B46DA
:1054480067850097FFF754FD32213C2096220B46D2
:1054580066850096FFF74CFD32210B4696226E209A
:10546800A4F82A80CDF80080FFF742FDFFF7BAFBC9
:10547800FFF7B4FB3220FFF76DF92846FFF76AF90A
:105488006420FFF767F90B4B03F110028DE8240045
:1054980028465A681B682946FFF710FF1195119B8B
:1054A80001331193FBE700BF740E00208601002032
:1054B800BC9B040850C001082DE9F14FFFF750F8D4
:1054C8004FF0C0456420FFF745F90127FFF72EF993
:1054D8004FF028096D48FFF7F1F82F800520A5F84F
:1054E800009003F01BFACF232B80694B0026832200
:1054F8001E801A8030221A80ED222A804FF064081C
:105508000322A3F800801A8012221A8081221A80AE
:10551800E8222A8085221A8079221F801A80CB22CD
:105528002A8039221A804FF0340C02242C21F722C9
:1055380019801E80A3F800C01C802A8020221A80AF
:10554800EA222A80C0221E80C1211E802A802622AB
:105558001A80298011211980C521298035211980B7
:105568003E211980C7212980BE2119803621298032
:105578003A205521A3F8009028801980B12129806C
:105588004FF0100BF2211E80A3F800B029800821EB
:1055980019802A80E0221F804FF01F092A801A22D2
:1055A800A3F800904FF0180A1A800F210A22A3F8D6
:1055B80000A01A80198006211980452119808721A9
:1055C80019803221198007211A804FF0E10E1980C5
:1055D8001C80052419801C801E80A5F800E04FF06F
:1055E800250E1E80A3F800E04FF0270EA3F800E078
:1055F8001C80A3F800B04FF0090BA3F800B04FF0DF
:10560800780B1880A3F800B04FF04D0BA3F800B04A
:105618001C800D24A3F800A01C8038241C8018804E
:105628002A20A3F80090EF2428802B201E801E80BB
:105638001E801C8028803F201E801E801F801880AE
:10564800B720A5F800C028801980B62129801A80C3
:1056580082221A801122A3F800E040461E802927E2
:105668002A8003F05BF940462F8003F057F9094878
:10567800FFF724F82C232F8030462B8040F23F116F
:105688003246234601B0BDE8F04FCFE4400D030099
:105698000000026040420F002DE9F041022098B05E
:1056A800012100240AF0FAFB0125022680481696FB
:1056B80016A98DF85D408DF85E408DF85F408DF835
:1056C8005C500AF043F8182029460AF0E7FB284600
:1056D80029460AF0FBFB21460C2276480AF0B6F868
:1056E8000C22744829460AF0B1F804210C227148AA
:1056F8000AF0ACF805210C226E480AF0A7F8072139
:105708000C226C480AF0A2F808210C2269480AF019
:105718009DF809210C2267480AF098F80A21654883
:105728000C220AF093F80B2162480C220AF08EF83A
:105738000E210C225F480AF089F80F210C225D48DF
:105748000AF084F807210C225B480AF07FF8082148
:105758000C2259480AF07AF809210C2256480AF016
:1057680075F80A210C2254480AF070F80B210C2213
:1057780051480AF06BF80C210A464F480AF066F8BF
:105788000D210C224C480AF061F80E210C224A48DF
:105798000AF05CF80C2248480F210AF057F84CF63A
:1057A800B3734448169316A98DF85C608DF85E4073
:1057B8008DF85F408DF85D5009F0C8FF16A94FF6C7
:1057C80080733D4816938DF85C608DF85E408DF8C7
:1057D8005F408DF85D5009F0B9FF40F6B830FEF72C
:1057E8006DFFFEF7A3FF40F6B830FEF767FF0F2303
:1057F80011934FF4805310270DF13C080993684624
:105808004FF4002310941294149415940094019466
:105818000294039704940694079408940A940594B0
:105828000B940C93CDF834800F95139509F007FD70
:105838000523684611930F961094129414941594A6
:10584800CDF83880139509F0FAFC2946204609F06E
:1058580076FD40F6B830FEF731FF2046FFF7A0F995
:1058680004461649164E3846224608F07DFF41F296
:1058780089239C4248F68918124F01D044450ED11D
:10588800FEF7BCFF00233B70A6F8008010200E49ED
:1058980048F6891241F2892308F066FF05E0FFF710
:1058A8000BFE49F241333D70338018B0BDE8F081FA
:1058B80000040240000C024000100240ACE0050861
:1058C80086010020801B0020C3E005084FF0C0437C
:1058D80036221A8003F50033012814BF68204820B7
:1058E8001880704770B5244B01228CB01A700024C0
:1058F8000AE0A9B21F2230460135FFF741FA642DAC
:10590800F7D10134642C02D00025A6B2F1E7322089
:10591800014602460346FFF7ABF94FF0C0432E227B
:105928001A8003F5003300201A881C881D88A4B249
:1059380000F09CF8ADB20023224600930F492B4695
:1059480003A810F097FC00230A20C82103AA00F03E
:10595800C7F904F0FC0204F4784444EAC20242EABB
:10596800D522074903A810F085FC0A20DC2103AAE8
:10597800002300F0B5F9FEE7801B002002E10508CE
:105988001AE105082DE9F04F40F23F19484534BFA8
:1059980004464C46EF2B34BF98464FF0EF084A4573
:1059A80038BF9146EF2934BF0D46EF25C4EB090AED
:1059B800C5EB080785B0BAF1000FB8BFCAF1000AF5
:1059C800002FB8BF7F424FF6FF734C452CBF1A46D5
:1059D80001221FFA8AFA454538BF0123BFB2029354
:1059E8000FFA8AF63BB29E42BDF838B0019202DD4A
:1059F800C6F34F0607E0022693FBF6F67642B6B2E8
:105A080001E01E4603E00FFA8AF35B420393144A4F
:105A18001378022B204629465A4602D1FDF7FDFC91
:105A280001E0FFF7ADF94C4501D1454514D0039A83
:105A380033B2934205DD019AF31BA4189BB2A4B2BA
:105A480000E0334636B23AB29642DADA029A534462
:105A5800AD189BB2ADB2D4E705B0BDE8F08F00BF7A
:105A6800C82E002000487047881B002082B0064BD3
:105A7800ADF80600BDF8062092B21A80188880B2E8
:105A880002B0FFF7B2B800BF841B0020014B188892
:105A980080B27047841B002082B0064BADF8060028
:105AA800BDF8062092B21A80188880B202B0FFF7BB
:105AB800A9B800BF861B0020014B188880B2704728
:105AC800861B0020FFF7CCBAFFF73ABA10B5BDF82D
:105AD80008400294BDE81040FFF788B910B5BDF83A
:105AE80008400294BDE81040FFF702BAFFF782BAF7
:105AF8002DE9F04F4FEA420800253D4C85B082461B
:105B08008B46C8F1030817462E461FFA87F909EB9A
:105B18000B0C228805EB0A031FFA8CFC9BB261462A
:105B2800184692B2CDF804C00293FFF729F9C9EBE1
:105B38000B0292B20392029B22880399184692B2F2
:105B4800FFF71EF9DDF804C02288C5EB0A039BB2F3
:105B58006146184692B20293FFF712F9029B228817
:105B68000399184692B2FFF70BF905EB0B0292B2B4
:105B7800039209EB0A03228803999BB2184692B252
:105B88000293FFF7FDF8029B2288C5EB0B0C1FFA66
:105B98008CFC1846614692B2CDF804C0C9EB0A09DC
:105BA800FFF7EEF8228803991FFA89F992B248465E
:105BB800FFF7E6F82288DDF804C092B2484661464D
:105BC800FFF7DEF8B8F1000F04DA08EB860808F1F1
:105BD800060805E0F31B08F10A0808EB8308013FF3
:105BE80001360135BE42ADB28FD905B0BDE8F08FA0
:105BF800841B002008B9FEF7F5BF012801D1FEF784
:105C0800EDBF7047704700200146F0224FF4A073A3
:105C1800FFF796B9704708B505280CD8DFE800F0FB
:105C2800121403050709094808BD094808BD0948B1
:105C380008BD094808BD0948094A0A4B40F2411104
:105C4800FEF700FD084808BD084808BD740100209B
:105C5800640100205C0100205401002025E10508B2
:105C6800F89B040860DF05087C0100206C01002017
:105C780010B50446FFF7CFFF014B18601C7110BD2B
:105C88008C010020014B1879704700BF8C0100205F
:105C980008B5FFF7C0FF808808BD08B5FFF7BBFF50
:105CA800C08808BDF7B51F460B4B0C4E1D6814463F
:105CB800EA882B68203C5443A4B2AE1B03EB44048F
:105CC80018BF0126AB888DE8500017B1FFF7EEF931
:105CD80001E0FFF771FAFEBD8C0100207C01002075
:105CE8002DE9F0410F46984615460446084E08E04F
:105CF800204643463946FFF7D5FF33689B88E418AA
:105D0800A4B215F8012B002AF2D1BDE8F08100BF3A
:105D18008C01002010B5044608462146BDE8104015
:105D2800DEE7094B70B5044618790E461546FFF7AD
:105D3800B4FFC6F1F001091A89B220462A460023A9
:105D4800BDE87040CCE700BF8C010020704700BF61
:105D5800044B1A680AB9044A1A601A6810181860BD
:105D680010467047A80E0020483F00204FF0FF3033
:105D7800704708B50248034A034B3721FEF762FC17
:105D880044E105080E9C040860DF050801207047FF
:105D980010B504460A4802210AF006FB0028F9D08B
:105DA800074821460AF0C9FA054801210AF0FCFA19
:105DB8000028F9D00248BDE810400AF0BBBA00BF7D
:105DC8000038004010B5194802210AF0EDFA002801
:105DD800F9D0164800210AF0B0FA144801210AF057
:105DE800E3FA0028F9D011480AF0A4FA0402A4B290
:105DF800002301E001339BB2002BFBD00B480221AA
:105E08000AF0D2FA0028F9D0084800210AF095FAD9
:105E1800064801210AF0C8FA0028F9D003480AF018
:105E280089FA2043C0F3CB0010BD00BF0038004002
:105E38002DE9F0478AB00AAF0A2001210AF02EF8AE
:105E48004FF4604347F8143D474EDFF824A101247E
:105E580000254FF00208304639468DF81A508DF863
:105E680018808DF819808DF81B4009F06FFC3046BA
:105E78000D21052209F0EAFC30460E21052209F021
:105E8800E5FC052230460F2109F0E0FC21464FF4DD
:105E980080400AF027F850460AF002F94FF482735E
:105EA800ADF802304FF40073ADF80A303823ADF87E
:105EB8000C30504607236946ADF81030ADF8005055
:105EC800ADF80450ADF80650ADF80850ADF80E50D6
:105ED8000AF018F9504621460AF0AFF9A9468DF89C
:105EE8001A5030464FF48055394605958DF81840BC
:105EF8008DF819808DF81B4009F028FC304629469A
:105F080009F095FC4025394618488DF818908DF809
:105F180019808DF81A908DF81B40059509F016FC2C
:105F280021464FF4804009F0E9FF062103200AF0DA
:105F380073FA0C2307A88DF8213007958DF8209067
:105F48008DF8224009F0F6F817238DF8243009A8B7
:105F58000F238DF825308DF826308DF8274002F074
:105F6800FBFE0AB0BDE8F08700040240000C0240C6
:105F780000380040014B1878704700BFAC0E002075
:105F8800024B5A889B8802800B807047AC0E002019
:105F9800014B00221A707047AC0E0020F0B593B088
:105FA80068460021482210F0E5F86D460024644850
:105FB8004FF4805109F03DFC002301E001339BB20E
:105FC800002BFBD09020FFF7E3FE002301E0013314
:105FD8009BB2002BFBD0FFF7F5FE4FF4805107462C
:105FE800574809F024FC002301E001339BB2002B41
:105FF800FBD053484FF4805109F01BFC002301E00B
:1060080001339BB2002BFBD0D020FFF7C1FE002349
:1060180001E001339BB2002BFBD0FFF7D3FE4FF416
:1060280080510646464809F002FC45F8047B0134D5
:106038002E6244484021E4B209F0E7FB10B9092C6C
:10604800B5D101E0092C78D19DE80C00D218029B4B
:1060580003980699D218049BC018059BC018079B83
:10606800CB180899032490FBF4F092FBF4F25B1828
:1060780093FBF4F3151AC11A9C1A002DB8BF6D4290
:106088000029B8BF4942002CB8BF6442502D03DD37
:10609800502909DD502C50DC8D4205DAAC424FF016
:1060A800020405DB111806E08C424FF0020401DA05
:1060B800D11800E0C1180A9B099A0C980F9DD218B4
:1060C8000B9BD2180D9BC0180E9BC018109BEB1889
:1060D800119D91FBF4F1032492FBF4F290FBF4F090
:1060E8005B1993FBF4F3161AC41A9D1A002EB8BF55
:1060F8007642002CB8BF6442002DB8BF6D42502EC6
:1061080089B203DD502C09DD502D16DCA64205DAD4
:10611800B5424FF0020405DB131806E0A5424FF024
:10612800020401DAD31800E0C318074A93FBF4F31A
:106138009BB2938001235180137013B0F0BD00BF50
:1061480000040240000C0240AC0E002000000000D9
:10615800FFF710BFF7B505460C4601A80DF106017B
:10616800FFF70EFF1B4BBDF80660BDF8040093E86F
:106178000600724301FB002299685218164992FBE7
:10618800F1F207EE102AF8EEC77A40F23F17FCEE5C
:10619800E77A17EE902A92B2B2F5207F28BF3A46E6
:1061A8002A801D69DA685B696E4302FB0060C018CB
:1061B80090FBF1F107EE101AF8EEC77AFCEEE77AD9
:1061C80017EE903A9BB2B3F5F07F28BFEF232380F8
:1061D800FEBD00BFB40E002040420F00FFF7D8BE3E
:1061E800014B187E704700BFB40E0020FFF7C8BEF1
:1061F800042808B505D90748074A084B7D21FEF74A
:1062080021FA054B03EB8000038B0B80438B138033
:1062180008BD00BF65E10508149C040883E1050872
:1062280008B5082001F0F6F942F69643C31A584219
:1062380040EB030008BD10B50A2001F013FA0C4C1E
:1062480020600E2001F00EFA6060122001F00AFAB8
:10625800A060162001F006FAE0601A2001F002FAA8
:1062680020611E2001F0FEF901236061237610BD34
:10627800B40E002010B5FFF7DBFD01F0A9FA0446C3
:1062880001F0B2FA074903462246202008F06CFACA
:10629800FFF7C6FF28B101F0B5FA10B9BDE8104004
:1062A800C9E710BDBFE1050810B5104C0A202168E8
:1062B80001F0BFF961680E2001F0BBF9A168122056
:1062C80001F0B7F9E168162001F0B3F921691A2045
:1062D80001F0AFF961691E2001F0ABF9082042F620
:1062E8009641BDE8104001F087B900BFB40E002008
:1062F8002DE9F04F0346A7B0B0F800C01C89868886
:10630800DF885D89CDF810C0B249B0F802C0B3F893
:106318000C90B3F80E80CDF824C00FFA84FB30B28D
:1063280001220FFA87FE0BEB000C0A7629B20FFA4E
:1063380089FACDF888C001EB0E0C0FFA88F2CDF877
:1063480090C00AEB0B0CCDF830C002EB010CCDF875
:1063580058C0B3F810C05B8ACDF800C00FFA8CFCA7
:1063680006910CEB00010A9102930CEB0A011BB297
:10637800239103EB0E010E9199182591049900FAC7
:1063880081F0584450446044DDF824C006990EFA60
:106398008CFEDDF810C01FFA80FB1CFB0CF08E444D
:1063A80016FB0600964414FB0400009A19FB09002A
:1063B8009E4412FB02001FFA8EFA0BF0FFF8DDF87C
:1063C80024C0029ACDE912011CFB0CF017FB070050
:1063D80015FB050018FB080012FB02000BF0EEF895
:1063E800DDF824C0029ACDE9140104991CFB01F3DD
:1063F80017FB063615FB0466009B18FB096612FBA3
:1064080003600BF0DBF8DDE91423CDE90001DDE9D9
:1064180012010BF049F904460D46DDE90001024678
:106428000B460BF041F902460B46204629460AF076
:1064380087FFCDE9180158460BF0D0F8CDE91001D7
:10644800DDE91023DDE900010BF02EF9CDE90601A5
:1064580050460BF0C3F8804689464246DDE91201F2
:106468004B460BF021F9DDE91023CDE91C01DDE9EC
:1064780014010BF019F9002206460F46564BDDE9C8
:1064880018010BF011F9424604460D464B46DDE96A
:1064980006010BF009F902460B460AF053FF0246C3
:1064A8000B46204629460AF04DFF424604460D4653
:1064B8004B46DDE91C010BF0F7F802460B46204677
:1064C80029460AF03DFFDDE9102304460D46304613
:1064D80039460BF0E9F802460B46204629460AF0F1
:1064E8002FFFDDF828C0CDE902014FEA8C10DDF856
:1064F80030C000EB0C20DDF810C0A0241CFB040009
:106508000BF05CF8DDF838C0CDE90A014FEA8C10D1
:10651800DDF858C000EB0C20DDF824C01CFB04009B
:106528000BF04CF8CDE90C0150460BF047F8DDE9CB
:106538001023CDE91601DDE90C010BF0B5F8424650
:10654800CDE91E014B46DDE90A010BF0ADF84246E4
:10655800CDE920014B46DDE900010BF0A5F83246F4
:106568003B460AF0EDFECDE90E0158460BF026F841
:10657800DDE91C23CDE91A01DDE906010AF0E0FE98
:10658800DDF88CC0C024CDE9060104FB0CF0DDF871
:1065980088C0302505FB0C00DDF810C078261CFBF0
:1065A80006000BF00BF8DDF894C0824604FB0CF0F3
:1065B800DDF890C005FB0C00DDF824C01CFB0600CC
:1065C8008B460AF0FBFFDDE9102306460F460BF069
:1065D8006BF803E0B40E0020000014404246CDE9F9
:1065E80004014B46504659460BF05EF8DDE914238A
:1065F80080468946DDE90A010BF056F8DDE90023FB
:1066080004460D46DDE90C010BF04EF802460B4638
:10661800204629460AF094FE0022A14B0BF044F8CC
:10662800DDE9202304460D46DDE91E010AF088FE57
:1066380002460B46DDE916010BF036F802460B461A
:10664800204629460AF07EFE002204460D46954B58
:10665800DDE90E010BF028F802460B4620462946D4
:106668000AF070FEDDE902230BF048F988A3D3E9AC
:1066780000230BF019F80BF0B1FA8B490860DDE93B
:106688001223DDE90C010BF00FF8DDE900230446C5
:106698000D46DDE90A010BF007F802460B462046D5
:1066A80029460AF04DFE00227D4B0AF0FDFFDDE988
:1066B8001E2304460D46DDE920010AF041FE02468C
:1066C8000B46DDE91A010AF0EFFF02460B462046A9
:1066D80029460AF037FE002204460D46714BDDE9D3
:1066E80006010AF0E1FF02460B46204629460AF059
:1066F80029FEDDE902230BF001F965A3D3E90023A4
:106708000AF0D2FF0BF06AFA674A5060DDE90E23FF
:10671800DDE90A010AF0C8FFDDE9062304460D4653
:10672800DDE90C010AF0C0FF02460B462046294667
:106738000AF008FE002204460D465A4BDDE918010E
:106748000AF0B2FF02460B46204629460AF0FAFD37
:10675800DDE902230BF0D2F84DA3D3E900230AF0B8
:10676800A3FF0BF03BFA504B59469860DDE9142320
:1067780050460AF099FFDDE9002304460D463046ED
:1067880039460AF091FF02460B46204629460AF090
:10679800D7FD0022424B0AF087FF424604460D46C9
:1067A8004B46DDE904010AF0CBFD02460B46DDE964
:1067B80016010AF079FF02460B46204629460AF0E0
:1067C800C1FD35A3D3E9002304460D46DDE90E01DA
:1067D8000AF06AFF02460B46204629460AF0B2FD37
:1067E800DDE902230BF08AF829A3D3E900230AF094
:1067F8005BFF0BF0F3F9DFF8B0C0DDE91223CCF84A
:106808000C00394630460AF04FFFDDE90023044604
:106818000D46504659460AF047FF02460B462046A9
:1068280029460AF08DFD00221D4B0AF03DFFDDE9E7
:10683800042304460D46404649460AF081FD0246B7
:106848000B46DDE91A010AF02FFF02460B462046E7
:1068580029460AF077FD10A3D3E9002304460D4624
:10686800DDE906010AF020FF02460B4620462946CC
:106878000AF068FDDDE902230BF040F804A3D3E930
:1068880000230AF011FF0BF0A9F9074908610DE090
:106898000000000080842E410000000000C08240FB
:1068A8000000144000008940B40E0020DDE90E23EA
:1068B800504659460AF0F8FEDDE9062304460D461F
:1068C800304639460AF0F0FE02460B462046294675
:1068D8000AF038FD11A3D3E9002304460D46DDE98B
:1068E80018010AF0E1FE02460B46204629460AF046
:1068F80029FDDDE902230BF001F80AA3D3E90023FF
:106908000AF0D2FE0BF06AF9034A506127B0BDE8DD
:10691800F04FC9E4AFF30080B40E0020000000007F
:1069280000C082400000000080842E41AFF3008048
:10693800064B074A596811601969064A1160D969F6
:10694800054A11609A6A054B1A6070479401002045
:10695800B8280020D82E0020AC2E00206428002063
:10696800014B1878704700BFD00E0020032808B5E7
:1069780005D90548054A064B7321FDF763FE0C232C
:106988005843044B185808BDFAE10508409C040810
:1069980014E2050894010020032808B505D9064823
:1069A800064A074B7821FDF74DFE064B0C2202FBE9
:1069B8000030406808BD00BFFAE10508509C040893
:1069C80014E2050894010020034B044A1B780C21AB
:1069D80001FB032398687047D00E00209401002023
:1069E800034B044A1B780C2000FB03239960704773
:1069F800D00E002094010020144B1B78012B10B5F9
:106A0800134B144C0ED11968C82000F012FE2168EF
:106A1800CC2000F00EFE104BD020196800F009FEC3
:106A2800D4200DE01968D82000F003FE2168DC208E
:106A380000F0FFFD084BE020196800F0FAFDE420A3
:106A4800064B1968BDE8104000F0F3BD840F002024
:106A5800B8280020D82E0020AC2E00206428002062
:106A6800144B1B78012B10B5134C0FD1C82000F024
:106A7800F9FD2060CC2000F0F5FD104B1860D02007
:106A880000F0F0FD0E4B1860D4200EE0D82000F086
:106A9800E9FD2060DC2000F0E5FD084B1860E020EF
:106AA80000F0E0FD064B1860E42000F0DBFD054B2C
:106AB800186010BD840F0020B8280020D82E0020B0
:106AC800AC2E00206428002008B504F045FE10B163
:106AD800BDE80840C4E7BDE8084029E70148FAF7DF
:106AE80006BE00BFC01800200148FAF700BE00BF6C
:106AF800C01800200148FAF7FABD00BFC0180020EE
:106B08000148FAF7F4BD00BFC0180020032808B5F3
:106B180005D91648164A174B4F21FDF793FD164B1A
:106B28001870164B1870164B012202281A70154B54
:106B38000FD0032813D0904205D0134A12681A6068
:106B4800BDE80840CAE7114A12681A60BDE8084063
:106B5800CAE70F4A12681A60BDE80840CAE70D4A3A
:106B680012681A60BDE80840CAE700BFFAE10508E4
:106B7800619C04083EE20508D00E0020AF280020E2
:106B8800DC0E0020940200208C02002088020020E5
:106B98008402002080020020064B07495960C0216A
:106BA800002219721E211A70D9601A745A611A7655
:106BB800DA617047B41B002040787D0110B50321CD
:106BC800FF22C02001F0B0FB1F4C10212060802262
:106BD800C02001F0A9FB112120608022C02001F013
:106BE800A3FB122120608022C02001F09DFB13210D
:106BF80020608022C02001F097FB142120608022B1
:106C0800C02001F091FB152120608022C02001F0F6
:106C18008BFB802220601621C02001F085FB2060BC
:106C2800C0201721802201F07FFB2060074CC02084
:106C3800227AB72101F078FB00232374636123765D
:106C4800E3610123237010BD90280020B41B0020AD
:106C580038B5C0200321FF2201F066FB0B4D00244C
:106C68002B19615D5A78C020023401F05DFBC82CF5
:106C7800F6D1B121AC22C02001F056FBC02003217F
:106C8800002201F051FB002038BD00BF759C0408AC
:106C98002DE9F34706460F4692461D461AB90C1FC2
:106CA800E401914635E005EE902A06EE903AB8EEFA
:106CB800657AF8EE667AFC01C7EE277AA4F50074C7
:106CC8009FED5C7A67EE877A17EE900A0AF098FCD7
:106CD80041EC100B0CF06CFD59EC108B494640460A
:106CE8000AF0A4FF24184FEACA100AF067FCCDE99D
:106CF800000128460AF062FC4B4642460AF0D4FCE2
:106D080002460B46DDE900010AF01AFB0AF08EFF85
:106D18008146002E14BF4FF022084FF01A08C5F321
:106D280007224146C02001F0FFFA08F10101EAB24A
:106D3800C02001F0F9FAC4F3014208F10201C020B1
:106D480001F0F2FAC4F3072208F10301C02001F0B0
:106D5800EBFAE2B208F10401C02001F0E5FAC9F348
:106D6800034305F4702243EA123208F10501C020FA
:106D780001F0DAFA08F10601C9F30722C02001F090
:106D8800D3FA08F107015FFA89F2C02001F0CCFAC2
:106D9800C020B121A02201F0C7FA07EE107A264CD4
:106DA800F8EEC77A0EBBD4ED015A06EE90AAB8EEFB
:106DB800657A05EE905AB8EE666AF8EE656A0123C0
:106DC800C6EE266A237477EEA67A67EE277A17EE60
:106DD800900A0AF015FC41EC100B0CF0E9FC51ECA0
:106DE800100B0AF023FF606120E005EE90AAD4EDB5
:106DF800016AB8EE656A05EE905AB8EE667AF8EE62
:106E0800656A0123C6EE266A237677EEA67A67EED0
:106E1800277A17EE900A0AF0F3FB41EC100B0CF0FE
:106E2800C7FC51EC100B0AF001FFE0610020BDE83F
:106E3800FC8700BF00000043B41B00200022012390
:106E480026E7012838B50D4604D002280CBF3C249B
:106E58002C2400E034242146C02001F0DFFA05F09C
:106E6800070200F00F0040EA02122146C020BDE8E8
:106E7800384001F059BA2DE9F3470A9C1D460746E8
:106E88008A461646524B01E06D0864089C42FBD8BE
:106E98002DB906F10076043EF601A94634E006EE67
:106EA800905AB8EE667A06EE904AF8EE667AF601DF
:106EB800C7EE277AA6F500769FED467A67EE877AC1
:106EC80017EE900A0AF09CFB41EC100B0CF070FCDA
:106ED80059EC108B494640460AF0A8FE3618E801DE
:106EE8000AF06CFBCDE9000120460AF067FB4B462F
:106EF80042460AF0D9FB02460B46DDE900010AF0DA
:106F08001FFA0AF093FE8146022F9BBF324BDB1912
:106F18004FF0000893F8C880C4F307224146C02008
:106F280001F002FA08F10101E2B2C9B2C02001F091
:106F3800FBF908F10201C9B2C6F30142C02001F011
:106F4800F3F908F10301C9B2C6F30722C02001F022
:106F5800EBF908F10401C9B2F2B2C02001F0E4F97A
:106F680004F47024C9F3034308F1050143EA143219
:106F7800C9B2C02001F0D8F908F10601C9B2C9F3B5
:106F88000722C02008F1070801F0CEF95FFA89F25C
:106F98005FFA88F1C02001F0C7F9BAF1010F0CBF00
:106FA8002F220F220DB942F04002012F06D002D342
:106FB800022F0AD105E0C020102104E0C0201121D1
:106FC80001E0C020122101F0AFF90020BDE8FC87E4
:106FD800FFFF0F0000000043759C040807B501235C
:106FE80000930023FFF747FF0EBD00280CBFFF22C8
:106FF800002208B5C020032101F096F9002008BD41
:1070080008B5C020B121AC2201F08EF9002008BDDE
:1070180008B50420012108F041FF4FF480700121D8
:10702800BDE8084008F06ABF07B5022300930323B0
:107038008DF804300348002369468DF8073008F0BE
:1070480085FB0EBD0008024030B5124D8BB0002400
:1070580006A8069407940894099407F045FD00943F
:107068008DF804408DF80540029403940494284652
:10707800012469468DF8144007F007FD28460B21C6
:107088002246062307F07CFD2846214607F046FDE8
:107098000BB030BD0020014010B50021044601228C
:1070A800302001F041F9C0B9012001F037FC002C73
:1070B800B8BF4034E4B210212246302001F034F940
:1070C800012001F02BFC30201121224601F02CF97F
:1070D8000120BDE8104001F021BC10BD10B5002111
:1070E80004460122302001F01FF9C0B9012001F047
:1070F80015FC002CB8BF4034E4B2122122463020DF
:1071080001F012F9012001F009FC30201321224678
:1071180001F00AF90120BDE8104001F0FFBB10BDE5
:1071280038B5012205460C463020002101F0FCF854
:10713800F0B9012001F0F2FB25EAE5725F2AA8BF49
:107148005F223B21D2B2302001F0EEF8012001F09D
:10715800E5FB24EAE4725F2AA8BF5F22D2B230209E
:107168003C2101F0E1F80120BDE8384001F0D6BB30
:1071780038BD302810B504460ADC10F17F0F02DB59
:10718800002802DB05E06FF07E0404F5807400E05F
:107198003024002130200A4601F0C6F8A8B90120A1
:1071A800E4B201F0BBFB41212246302001F0BCF8DB
:1071B800012001F0B3FB30204221224601F0B4F84F
:1071C8000120BDE8104001F0A9BB10BD282810B56A
:1071D800044609DC10F1180F02DB002802DB04E08A
:1071E8006FF017047F3400E02824002130200A467D
:1071F80001F09AF8A8B90120E4B201F08FFB5321FD
:107208002246302001F090F8012001F087FB302061
:107218005421224601F088F80120BDE8104001F011
:107228007DBB10BD08B530200021012201F07CF89B
:1072380060B9012001F072FB30203321402201F0B7
:1072480073F80120BDE8084001F068BB08BD10B51F
:1072580030200021012201F067F8044660B90120BE
:1072680001F05CFB30203321224601F05DF801205B
:10727800BDE8104001F052BB10BD10B53020002110
:10728800012201F051F80446A0B9012001F046FBA3
:1072980034212246302001F047F8012001F03EFB5E
:1072A80030203721224601F03FF80120BDE8104088
:1072B80001F034BB10BD4020EEE640200EE708B5D3
:1072C80000210122302001F02FF8012001F026FBD7
:1072D80030203421024601F027F8012001F01EFB7E
:1072E80030203721024601F01FF80120BDE8084090
:1072F80001F014BB08B500210122302001F014F878
:10730800012001F00BFB302034210C2201F00CF895
:107318000120BDE8084001F001BB000000000000AA
:107328002DE9F04F984B994A1968994B002914BFD9
:1073380091469946974B2DED048BC3F80090964BD8
:107348000025002287B01A80AA46AB46A8465AE014
:10735800A2004046CDF804C002920AF051F907464F
:10736800584601F100460AF04BF902460B463846EA
:10737800314609F0E5FF39F9243007EE103AF8EE06
:10738800C77A064617EE900A0F460AF039F9024600
:107398000B463046394609F0D5FF0AF067FC074628
:1073A80050460AF02DF90446284601F100460AF035
:1073B80027F9CDE90401DDE904232046314609F027
:1073C800BFFF029A09EB02030446B3F9023007EE45
:1073D800103AF8EEC77A0D4617EE900A0AF010F93F
:1073E80002460B462046294609F0ACFF0AF03EFC4F
:1073F800DDF804C0684A0CF1010CC3465546A2F8F2
:1074080000C08246B846644BB3F800C00FFA8CF44B
:10741800B32C9DDD58460AF0F3F8CDE90201404649
:107428000AF0EEF8002206460F465C4BDDE9020141
:107438000AF03AF902460B463046394609F082FF0F
:107448000022574B0AF05AFA0AF010FC4CA3D3E971
:10745800002309EE900ADDE902010AF025F900226D
:107468004F4B0AF04BFA0AF001FC09EE100A2846C5
:107478000AF0C6F8044650460D460AF0C1F8002244
:1074880006460F4620462946444B0AF00DF90246A7
:107498000B463046394609F055FF0022404B0AF0AA
:1074A8002DFA0AF0E3FB36A3D3E9002308EE900A8D
:1074B800294620460AF0F8F80022394B0AF01EFA4D
:1074C8000AF0D4FB08EE100A69EE287A58EE297AF9
:1074D80017EE900A0AF094F868EE097A48EEA97A4D
:1074E800044617EE900A0D460AF08AF845EC104B50
:1074F80041EC110B0CF060FA51EC100B0AF0B6FBE2
:1075080028EE088A08EEA88A07EE100A254B264CB2
:10751800F1EE477AC3ED007A18EE100A0AF070F817
:1075280041EC100B0CF056FB29EE099A51EC100BAC
:1075380009EEA99A0AF09AFB206019EE100A0AF0DF
:107548005FF841EC100B0CF045FB51EC100B0AF006
:107558008DFBD4ED007A07EE100A87EE877A134B7D
:107568001860134BFDEEE77A83ED007A114BC3EDFB
:10757800007A07B0BDEC048BBDE8F08FAFF3008054
:10758800912B50E67AB6EB3FDC1B002062250020E9
:10759800C21F0020D81B0020E41B00200000E03F91
:1075A80000005940E02E0020FC2E0020F02E002084
:1075B800E82E0020E01B002010B5084C204607F0FC
:1075C80012FD074B1860FFF7ABFE064B0649012278
:1075D80020461A80BDE8104007F086BD10600240C2
:1075E800DC1B0020D20E002020800010014B186800
:1075F800704700BFE01B002038B505460C46013532
:10760800C1F3072101F098F9A8B2E1B201F094F9A9
:1076180000B238BD38B5044600F0C8FF013405464D
:10762800A0B200F0C3FFEDB2C0B240EA052000B23C
:1076380038BD37B50B0E8DF804300B0C8DF80530BE
:107648000B0A8DF806308DF80710002400E0284654
:1076580001AB451CE15C013401F06EF9042CADB2BC
:10766800F5D13EBD37B5002400E02846451C00F0A2
:107678009DFF01ABADB2E0540134042CF5D19DF867
:1076880005009DF80430000440EA03609DF80730C7
:1076980018439DF8063040EA03203EBD37B5002365
:1076A8000193002400E02846451C00F07FFF01AB51
:1076B800ADB2E0540134042CF5D19DED010A3EBD74
:1076C8007047000038B50446642001F027F9257892
:1076D8006068AD00EDB2257008F09DF8237A40FA95
:1076E80003F000F003000543104B257005F00F056B
:1076F8005A5D6378D218D2B2D3B20132D2B2022A1A
:10770800637001D80022A2705BB2012B03DD012354
:10771800A3700023637094F90130013303DAFF2367
:10772800A3700023637094F9020038BD409D0408DB
:10773800F7B504200121234F08F0B0FB02AD012169
:107748004FF48040012408F0D9FB00264FF4B073B1
:107758003846694645F8083D8DF804608DF80740BD
:1077680007F0F4FF1020214608F098FB78236946BB
:10777800154800938DF804608DF8074007F0E6FF80
:107788000420214608F08AFB21464FF4804008F087
:10779800B5FB1C233846694600938DF804608DF8C4
:1077A800074007F0D3FF0220214608F077FBB023FB
:1077B80006488DF8046069468DF80740009307F085
:1077C800C5FFFEBD00080240001002400004024050
:1077D800802108B5034808F018F8D0F1010038BF37
:1077E800002008BD0004024008B54FF48071044829
:1077F80008F00BF8D0F1010038BF002008BD00BF29
:107808000008024008B5FFF7E3FF08B1FFF7ECFFF7
:10781800C0B208BD70B500283AD01E4B1A7880183F
:107828001D4AC0B292F90020187040B282421B4A29
:1078380002DD11780139197093F9001092F90020CE
:1078480091FBF2F402FB14141549E4B21C700A8887
:10785800144B1A80144B154A18881080144A92F950
:10786800000064B2013094FBF0F200FB1240114CAE
:107878002688114C258800FB065008800F49088887
:107888000F49098802FB00121A800E4B01221A7058
:1078980070BD00BF863C0020B93800209538002014
:1078A800B63C0020DA380020843C00208C3A0020C6
:1078B800B83C0020E83900201C3D0020483D00204D
:1078C8006A3A002094380020F0B5264A264C002356
:1078D8001370264A25681678254A12680FE0D45C8A
:1078E8002F197F7817F0040F07D0302C02D12023EE
:1078F800135431E01B4A137003E00133DBB29E429C
:10790800EDDA184B1B788342194B16D9A9B11A68BE
:10791800164C3121115430210BE01A681518125CED
:107928002E2A19D0303AD2B2092A88BF29700130DC
:10793800C0B222788242F0DA0EE01B681A5C79B194
:107948002E2A0DD05118C9B2392903D82F2998BF2A
:10795800302100E039211954BDE8F040FCF74ABC59
:10796800F0BD00BFD40E0020CC0400203C3E002017
:10797800A83C002010B5642000F0D0FF7E48FFF737
:10798800A1FE7E4B1B7804460A2B00F2D280DFE86A
:1079980013F00B000B00D000710071003400870059
:1079A800D00087009000AA00FFF71EFF10B1F9F77A
:1079B80073FCBEE0724B1888724B1B88C01A724B5E
:1079C8001B8890FBF3F0714B1A88714B1B88D31AF4
:1079D800704A128893FBF2F3DBB2C0B2032B00F2B9
:1079E800A580DFE803F0020406086B4A3FE06B4A13
:1079F8003DE06B4A3BE06B4A39E0FFF7F5FED8B152
:107A080000210A2268480FF085FD684B00211860A4
:107A18000A2267480FF07EFD664B18600420FEF7C7
:107A280027F996200521644A0023FEF759F900201A
:107A3800FEF71EF906F024FC514B1888514B1B88A1
:107A4800C01A514B1B8890FBF3F0504B1A88504BCF
:107A58001B88D31A4F4A128893FBF2F3DBB2C0B2E9
:107A680013B1012B62D101E04F4A00E0504A534B59
:107A78001A605BE000285CD0514B1A7806DD0132B1
:107A8800D2B20F2A1A7008D9102205E0013AD2B2F0
:107A9800102A1A7001D900221A70F9F7FDFE48E081
:107AA800002846D0474B93F90020002A41D118708E
:107AB8003FE0FFF799FEA0B1002143480FF076FCA4
:107AC800424B042083ED000AFEF7D2F8B4200521CA
:107AD8003F4A0023FEF704F9FAF7E6FA0020FEF71A
:107AE800C7F8394A16E0FFF77FFE90B10021394800
:107AF8000FF05CFC384B042083ED000AFEF7B8F861
:107B080096200521324A0023FEF7EAF80020FEF706
:107B1800AFF8304A294B1A60194B1888194B1B8843
:107B2800C01A194B1B8890FBF3F0C0B22146FFF72F
:107B3800CBFE2A48FFF7C6FD104B1B78013B0A2BEA
:107B480019D8DFE803F015181818150A0A180606D8
:107B58000A00234B1B78022B0AD10028214B01D1A4
:107B6800187010BD02DD01221A7010BDFF22FBE75C
:107B7800BDE810404EE610BDC401002038280020A2
:107B8800B63C00201C3D0020E8390020843C002041
:107B98006A3A0020483D00207C280020A4280020C4
:107BA800BA2E002068280020243D002078020020FA
:107BB800983C00207402002086E20508A83C0020BA
:107BC800B6280020B43C0020AC380020D4030020A4
:107BD80096E20508D0380020D0030020D00100200C
:107BE800AC3A0020ED1B002010B58CB01E490F22C6
:107BF80068460EF07DFA1D490F2204A80EF078FAA7
:107C08001B490F2208A80EF073FA00210822302021
:107C180000F08AFB012000F081FE002404AB1DF86F
:107C28000420E15C302000F07FFB0134012000F0EB
:107C380075FE0F2CF2D100210922302000F074FBD0
:107C4800012000F06BFE002408AB1DF80420E15C65
:107C5800302000F069FB0134012000F05FFE0F2C9A
:107C6800F2D10CB010BD00BF529D0408619D0408FC
:107C7800709D040810B58CB01E490F2268460EF09E
:107C880037FA1D490F2204A80EF032FA1B490F22B9
:107C980008A80EF02DFA00210822302000F044FB3D
:107CA800012000F03BFE002404AB1DF80420E15C39
:107CB800302000F039FB0134012000F02FFE0F2C9A
:107CC800F2D100210922302000F02EFB012000F023
:107CD80025FE002408AB1DF80420E15C302000F0EC
:107CE80023FB0134012000F019FE0F2CF2D10CB057
:107CF80010BD00BF7F9D04088E9D04089D9D04084B
:107D080010B58CB01E490F2268460EF0F1F91D49D6
:107D18000F2204A80EF0ECF91B490F2208A80EF058
:107D2800E7F900210822302000F0FEFA012000F0D7
:107D3800F5FD002404AB1DF80420E15C302000F0C0
:107D4800F3FA0134012000F0E9FD0F2CF2D10021F3
:107D58000922302000F0E8FA012000F0DFFD0024BD
:107D680008AB1DF80420E15C302000F0DDFA013496
:107D7800012000F0D3FD0F2CF2D10CB010BD00BFD4
:107D8800AC9D0408BB9D0408CA9D040807B50220E1
:107D9800012108F083F8012300938DF804300223B1
:107DA8008DF805300448002369468DF806308DF8B3
:107DB800073007F0CBFC0EBD0004024010B5084C9C
:107DC80001210022204607F036FD40F2FF4000F076
:107DD800A5FD012120460A46BDE8104007F02BBD4D
:107DE8000004024008B5FFF7E9FF00210A463020E9
:107DF80000F09AFA012000F091FD01210A46302096
:107E080000F092FA012000F089FD002101223020C3
:107E180000F08AFA012000F081FD012108223020BB
:107E280000F082FA012000F079FD022101223020C1
:107E380000F07AFA012000F071FD00210A46302096
:107E480000F072FA012000F069FD1B21CD223020DC
:107E580000F06AFA012000F061FD042103223020BD
:107E680000F062FA012000F059FD062109223020B5
:107E780000F05AFA012000F051FD072108223020B5
:107E880000F052FA012000F049FD0821702230204C
:107E980000F04AFA012000F041FD1E213020B022F6
:107EA80000F042FA012000F039FD0521912230202E
:107EB80000F03AFA012000F031FD0D2103223020B4
:107EC80000F032FA012000F029FD0E2100223020B6
:107ED80000F02AFA012000F021FD14218022302030
:107EE80000F022FA012000F019FD0B218822302031
:107EF80000F01AFA012000F011FD0C218222302036
:107F080000F012FA012000F009FD12218822302029
:107F180000F00AFA012000F001FD13218C22302024
:107F280000F002FA012000F0F9FC00210A46302096
:107F380000F0FAF9012000F0F1FC3D210222302086
:107F480000F0F2F9012000F0E9FCFFF74DFEFFF721
:107F580091FEFFF7D5FE30200021012200F0E4F960
:107F6800012000F0DBFC3D216422302000F0DCF928
:107F7800012000F0D3FC03210022302000F0D4F9C6
:107F8800012000F0CBFC04210022302000F0CCF9C5
:107F9800012000F0C3FC00210122302000F0C4F9C8
:107FA800012000F0BBFC0C210822302000F0BCF9B5
:107FB800012000F0B3FC0D210822302000F0B4F9B4
:107FC800012000F0ABFC0E210822302000F0ACF9B3
:107FD800012000F0A3FC0F210822302000F0A4F9B2
:107FE800012000F09BFC00210A46302000F09CF99B
:107FF800012000F093FC02224021302000F094F987
:10800800012000F08BFC30204121002200F08CF987
:10801800012000F083FC3F21D422302000F084F9B5
:10802800012000F07BFC00210122302000F07CF9C7
:10803800012000F073FC10210F22302000F074F9A9
:10804800012000F06BFC11210F22302000F06CF9A8
:10805800012000F063FC12210022302000F064F9B6
:10806800012000F05BFC13210022302000F05CF9B5
:10807800012000F053FC09213C22302000F054F983
:10808800012000F04BFC00210122302000F04CF9C7
:10809800012000F043FC30203421024600F044F96E
:1080A800012000F03BFC30203721024600F03CF96B
:1080B800012000F033FC36210322302000F034F98F
:1080C800012000F02BFC39210322302000F02CF98C
:1080D800012000F023FC3B213C22302000F024F951
:1080E800012000F01BFC3C210A46302000F01CF95E
:1080F800012000F013FC00210A46302000F014F99A
:10810800012000F00BFC5121C022302000F00CF9B6
:10811800012000F003FC52213020002200F004F975
:108128000120BDE8084000F0F9BB00BF2DE9F04F81
:10813800454E464D93B001214FF4001007F0AEFEB6
:10814800304606F051FE4FF0C0630293404B039354
:10815800404B002404934FF4B4794FF400334FF4A8
:1081680080684FF400674FF4005A4FF4807B304624
:1081780002A90C9301930997CDF8189005940794D8
:10818800CDF82080CDF828A0CDF82CB00D9406F0BD
:10819800B7FE22463046304906F00DFF3046012131
:1081A80006F013FF01210A464FF0402008F0E4F8DA
:1081B800284606F019FE294A019B0392284A0C9387
:1081C80004922846402202A9059209970294CDF804
:1081D80018900794CDF82080CDF828A0CDF82CB0C1
:1081E8000D9406F08DFE224628461E4906F0E3FE51
:1081F8002846012106F0E9FE42F210770122022109
:10820800194808F0B9F8384600F088FB30460121D3
:1082180006F0B1FE0121284606F0ADFE384600F012
:108228007DFB0B238DF8443011A801238DF84540C0
:108238008DF846408DF8473000F08EFD384600F046
:108248006DFB13B0BDE8F08F1060024088600240FB
:108258000C40004062250020C21F00200C3C00405A
:1082680092220020F21C0020003C0040024810210D
:10827800012206F0F7BE00BF1060024013B50220CD
:10828800012107F00BFE4FF410730E4C00930223EC
:108298008DF804308DF8053001238DF8063020461E
:1082A800002369468DF8073007F050FA204606216A
:1082B800042207F0CBFA20460921042207F0C6FA67
:1082C8001CBD00BF0004024030B5154D85B001212A
:1082D8004FF4001007F006FE284607F0CDFA0023F9
:1082E800ADF804304BF6FF73ADF806303323ADF824
:1082F80008304FF48063ADF80A304FF48043ADF88E
:108308000C3004AC074B2846012144F8103D07F017
:1083180055FB2846694607F0DDFA05B030BD00BFB9
:1083280000540040801A060073B54FF496130646B1
:108338000D461446019304E0019B5A1E0192002B3E
:1083480057D031484FF4003107F050FC0028F3D1E2
:108358002D48012107F03EFB4FF48053019304E0C0
:10836800019B5A1E0192002B45D02748274907F048
:1083780028FC0028F4D024483146002207F042FBAC
:108388004FF48053019304E0019B5A1E0192002B85
:1083980033D01D481E4907F014FC0028F4D01A48B1
:1083A800294607F0B2FB4FF48053019303E0019B89
:1083B8005A1E01921BB31448164907F002FC002804
:1083C800F5D01148214607F0A0FB4FF4961301930E
:1083D80003E0019B5A1E01929BB10B480E4907F01E
:1083E80005FC0028F5D00848012107F0FFFA002015
:1083F80008E0012006E0022004E0032002E0042057
:1084080000E005207CBD00BF0054004001000300CF
:1084180082000700800007000400001037B54FF401
:10842800961304460D46019305E0019B5A1E0192DE
:10843800002B00F09B8056484FF4003107F0D6FB24
:108448000028F2D15248012107F0C4FA4FF48053B2
:10845800019305E0019B5A1E0192002B00F08880D1
:108468004B484C4907F0ADFB0028F3D0484821465B
:10847800002207F0C7FA4FF48053019304E0019BF0
:108488005A1E0192002B75D04148434907F099FBC9
:108498000028F4D03E48294607F037FB4FF48053B4
:1084A800019304E0019B5A1E0192002B64D03848C6
:1084B8003A4907F09BFB0028F4D03548012107F022
:1084C80089FA4FF48053019304E0019B5A1E0192EC
:1084D800002B53D02E482F4907F073FB0028F4D007
:1084E8002B482146012207F08DFA4FF4805301935F
:1084F80004E0019B5A1E0192002B41D0244C2849CC
:10850800204607F073FB0028F3D02046002107F02F
:1085180081FA20460121238B07F068FA4FF4805333
:10852800019304E0019B5A1E0192002B2AD018489F
:108538001C4907F05BFB0028F4D0154807F0E7FA60
:108548004FF480530193124A03E0019B591E019195
:10855800D3B113889B05F8D4012104460C4807F0D1
:1085680059FA0B48104907F05BFB0EE001240CE0B8
:1085780002240AE0032408E0042406E0052404E0B9
:10858800062402E0072400E0082420463EBD00BF80
:10859800005400400100030082000700040000109E
:1085A80002000010400000100004001013B54FF442
:1085B80096130446019305E0019B5A1E0192002B75
:1085C80000F0AF8060484FF4003107F00FFB00283F
:1085D800F2D15D48012107F0FDF94FF48053019372
:1085E80005E0019B5A1E0192002B00F09C80564822
:1085F800564907F0E6FA0028F3D05348A021002294
:1086080007F000FA4FF48053019305E0019B5A1ECE
:108618000192002B00F089804B484D4907F0D1FAB0
:108628000028F3D0210A484807F06FFA4FF4805326
:10863800019304E0019B5A1E0192002B77D0424817
:10864800444907F0D3FA0028F4D0E1B23E4807F0D5
:108658005CFA4FF48053019304E0019B5A1E019287
:10866800002B66D038483B4907F0C0FA0028F4D000
:108678003548012107F0AEF94FF48053019304E027
:10868800019B5A1E0192002B55D02F482F4907F005
:1086980098FA0028F4D02C48A121012207F0B2F959
:1086A8004FF48053019304E0019B5A1E0192002B62
:1086B80043D0254C2849204607F098FA0028F3D0E3
:1086C8002046002107F0A6F920460121238B07F058
:1086D8008DF94FF48053019304E0019B5A1E0192D7
:1086E800002B2CD018481D4907F080FA0028F4D038
:1086F800154807F00CFA4FF480530193124A03E02F
:10870800019B591E0191E3B113889905F8D4012101
:1087180004460D4807F07EF90B48114907F080FA26
:1087280010E001240EE002240CE003240AE00424F3
:1087380008E0052406E0062404E0072402E00824F3
:1087480000E0092420461CBD00540040010003003D
:108758008200070004000010020000104000001012
:108768000004001013B54FF496130446019305E076
:10877800019B5A1E0192002B00F0AF8060484FF415
:10878800003107F033FA0028F2D15D48012107F0E3
:1087980021F94FF48053019305E0019B5A1E019281
:1087A800002B00F09C805648564907F00AFA00282A
:1087B800F3D05348A021002207F024F94FF4805346
:1087C800019305E0019B5A1E0192002B00F089805D
:1087D8004B484D4907F0F5F90028F3D0210A4848DD
:1087E80007F093F94FF48053019304E0019B5A1E5C
:1087F8000192002B77D04248444907F0F7F9002846
:10880800F4D0E1B23E4807F080F94FF48053019369
:1088180004E0019B5A1E0192002B66D038483B4960
:1088280007F0E4F90028F4D03548012107F0D2F820
:108838004FF48053019304E0019B5A1E0192002BD0
:1088480055D02F482F4907F0BCF90028F4D02C4800
:10885800A121012207F0D6F84FF48053019304E0D8
:10886800019B5A1E0192002B43D0254C28492046D3
:1088780007F0BCF90028F3D02046002107F0CAF819
:1088880020460121238B07F0B1F84FF48053019360
:1088980004E0019B5A1E0192002B2CD018481D4958
:1088A80007F0A4F90028F4D0154807F030F94FF480
:1088B80080530193124A03E0019B591E0191E3B1D1
:1088C80013889C05F8D4012104460D4807F0A2F846
:1088D8000B48114907F0A4F910E001240EE0022426
:1088E8000CE003240AE0042408E0052406E006243A
:1088F80004E0072402E0082400E0092420461CBD07
:10890800005400400100030082000700040000102A
:1089180002000010400000100004001082B0002384
:1089280004E0019B01330193009B01330093009BFA
:108938008342F6D302B0704737B54FF480530446EC
:108948000D46019304E0019B5A1E0192002B6DD045
:108958003C484FF4003107F049F90028F3D1394871
:10896800012107F037F84FF48053019304E0019B8D
:108978005A1E0192002B5BD03248334907F021F987
:108988000028F4D02F48A021002207F03BF84FF42C
:108998008053019304E0019B5A1E0192002B49D099
:1089A80028482A4907F00DF90028F4D0210A25485B
:1089B80007F0ABF84FF48053019304E0019B5A1E73
:1089C8000192002B38D01F48214907F0FAF80028F7
:1089D800F4D0E1B21B4807F098F84FF480530193A4
:1089E80003E0019B5A1E019243B31648184907F049
:1089F800E8F80028F5D01348294607F086F84FF420
:108A08009613019303E0019B5A1E0192C3B10D48CE
:108A1800104907F0EBF80028F5D00A48012106F0C4
:108A2800E5FF0D48FFF77AFF00200AE0012008E083
:108A3800022006E0032004E0042002E0052000E014
:108A480006203EBD005400400100030082000700DC
:108A58008000070004000010A0860100F7B54FF45D
:108A6800805304460D461646019304E0019B5A1EA6
:108A78000192002B74D040484FF4003107F0B6F84B
:108A88000028F3D13C48012106F0A4FF4FF480539D
:108A9800019304E0019B5A1E0192002B62D03648D4
:108AA800364907F08EF80028F4D03348A021002278
:108AB80006F0A8FF4FF48053019304E0019B5A1E6F
:108AC8000192002B50D02C482D4907F07AF8002845
:108AD800F4D0210A284807F018F84FF4805301937E
:108AE80004E0019B5A1E0192002B3FD022482549E1
:108AF80007F067F80028F4D0E1B21F4807F005F83E
:108B08004FF48053019304E0019B5A1E0192002BFD
:108B18002ED019481B4907F054F80028F4D0002437
:108B28004FF4961710E0295D134806F0EEFF019701
:108B380003E0019B5A1E0192E3B10F48124907F066
:108B480055F80028F5D00134E3B2B342EBD30A4814
:108B5800012106F04BFF0D48FFF7E0FE00200AE078
:108B6800012008E0022006E0032004E0042002E0DF
:108B7800052000E00620FEBD00540040010003006F
:108B8800820007008000070004000010A086010092
:108B980013B50520012107F081F9184C4FF4E05373
:108BA800009302238DF804308DF805302046002309
:108BB80069468DF806308DF8073006F0C7FD204667
:108BC8000A21062206F042FE20460C21062206F063
:108BD8003DFE062220460B21A4F5006406F036FE71
:108BE8004FF4004320466946009306F0AFFD204647
:108BF8000F21062206F02AFE1CBD00BF0008024015
:108C08001FB50446FFF7C2F8FFF75EFBFFF7EAF867
:108C1800FFF7BEFF01214FF4004007F063F902940B
:108C28000F4C1023ADF80230204600236946ADF8FA
:108C38000430ADF80C30ADF80030ADF8063007F070
:108C480080FA69464FF0402007F04FFB204601218B
:108C580007F0FFFA4FF04020012107F0FAFA1FBD94
:108C6800003C004082B0002304E0019B01330193E3
:108C7800009B01330093009B8342F6D302B07047F8
:108C880007B50420012107F009F901214FF48040BC
:108C980007F034F94FF40073009300238DF8043083
:108CA8000348012369468DF8073006F04FFD0EBDD5
:108CB800000802400D4B07B51A680D484FF47A7347
:108CC800B2FBF3F20B4B013A5A600B4AF02182F8DF
:108CD800231000229A6007221A60084B084A009362
:108CE8000121084B02F024F80EBD00BF98020020B5
:108CF800BC28002010E000E000ED00E0B4030020F4
:108D08009803002000030020054B1A6812B11A6866
:108D1800013A1A60034B1A6801321A60704700BFA3
:108D2800782800209428002082B0044B0190019AF2
:108D38001A601A68002AFCD102B07047782800200F
:108D4800704700BF40F0BE60024B40F42020D8605E
:108D5800704700BF00ED00E0C37810B503B3164BB1
:108D68004278DB688478DB43C3F30223C3F1040150
:108D7800C9B202FA01F10F2242FA03F2C9B2224043
:108D88000A430E4B01781201CB18D2B283F80023A4
:108D980003780122590903F01F0302FA03F307E0DD
:108DA80003780122590903F01F0302FA03F3203163
:108DB800024A42F8213010BD00ED00E000E100E079
:108DC80021F0604121F07F01014B08439860704712
:108DD80000ED00E0044B1A6909B1104301E022EAF2
:108DE80000001861704700BF00ED00E0044B1A68EE
:108DF80004280CBF42F0040222F004021A607047F3
:108E080010E000E000000000034A044B1A60044A26
:108E1800044B1A60704700BF00A00C468828002049
:108E2800920A064074280020034B00221A60034A65
:108E3800034B1A60E8E700BFF42E002000A00C46A0
:108E48004028002007EE100A024BF8EEC77AC3ED5F
:108E5800007A70474028002038B510EE100A08F054
:108E6800CFFB0DA3D3E9002308F01EFC084B0446F2
:108E780018680D4608F0C4FB0B46024629462046F2
:108E880008F03CFD08F0F2FE024B186038BD00BF48
:108E98008828002074280020182D4454FB211940EC
:108EA800014B93ED000A7047E82E0020014B93ED2B
:108EB800000A7047E02E0020014B93ED000A70472E
:108EC800F82E0020014B93ED000A7047E42E002095
:108ED800014B93ED000A7047FC2E0020014B93EDE7
:108EE800000A7047F02E002010B5FDF767FE00203D
:108EF800012324210246FDF7CBFE114B1C780020EC
:108F0800012C05D10146FDF79CFF2046002104E015
:108F18000721FDF796FF01200721FDF792FF632245
:108F28001221C020FFF700FA02200121FDF789FF76
:108F3800FEF766F80120BDE81040FEF756B800BFFE
:108F4800840F00200D4B1B78062B05D10C4B0D4AC6
:108F5800196812688A181A600B4B1B78012B084B8A
:108F6800196805D1094A914207DD01321A60704734
:108F7800074A914201DD01321A6070473828002003
:108F8800B42E002034280020840F00207FD1F00860
:108F9800FF27ED080E4B1B78062B05D10D4B0E4A0B
:108FA800196812688A1A1A600C4B1B78012B094B36
:108FB80005D10B4A1968914208DC1A6070471A6893
:108FC800B2F57A2FDCBF4FF47A221A60704700BFDF
:108FD80038280020B42E002034280020840F0020D8
:108FE80020A107002DE9F04F8DB00C460A90644887
:108FF800B0FBF1F008F0E2FA41EC100B0AF0D8FBF4
:1090080051EC100B08F012FE10F0010F804618BF4B
:1090180000F1FF3804FB08F008F0D0FA52A3D3E9B6
:10902800002308F06BFC04460D4645EC104B0AF093
:10903800BFFB57EC106B204632463B46294608F0EA
:109048007FF9CDE902013946304608F0EFFD48A323
:10905800D3E900230B90DDE9020108F0A1FD002807
:1090680058D1012000264FF01509314607464FF028
:10907800000A4FF0000B03E030463946069E049F75
:10908800A7FB0A23541807FB0B333E4A43F100059C
:109098000023A242AB41CDE904453ED3A6FB0A23F7
:1090A800141806FB0B33374843F100050021A04292
:1090B800A941CDE9064530D3DDE902012EA3D3E964
:1090C8000023049C069D08F06BFD40BBDDE90223EC
:1090D80000202D4908F012FC82468B464BEC10AB61
:1090E8000AF066FB5046594653EC102B8DED080BE1
:1090F80008F026F9CDE90201DDE9080109F064F874
:1091080009F1FF395FFA89F982468B46B9F1000FF8
:10911800B2D104E00125002401E035463C460B9A13
:109128000A9BD1B25BB9184622462B46FDF7B0FD23
:109138000A980123009301464246034609E0224665
:109148002B460120FDF7A4FD012000900146424670
:109158000023FDF790FEFDF753FF01200DB0BDE899
:10916800F04FFDF742BF00BF0000000084D77741F1
:10917800956479E17FFDA53DBBBDD7D9DF7CDB3D9B
:1091880000E9A435FFFF0F000000F03F224A234BFF
:109198001278012A10B5186009D1214A904201DDE0
:1091A80001321A601F4A1B6893420DDC0AE01E4A0E
:1091B800904201DD01321A601B68B3F57A2F03DC97
:1091C8004FF47A22154B1A60144B184A1968184B39
:1091D800184C1B68CB189342236018DC0020FFF75B
:1091E80001FF01202168FFF7FDFE0B4B1C780020D2
:1091F800012C05D10146FDF724FE2046002104E09C
:109208000721FDF71EFE01200721FDF71AFE034B7B
:109218001A68094B1A6010BD840F0020B42E002074
:109228007FD1F00820A10700FF27ED0880D1F008C2
:10923800CC2E0020D42E0020A8380020014B18681E
:10924800A4E700BFB02800207047FEE7FEE7FEE76E
:10925800FEE770477047704702F01AB910B5094C1D
:10926800A37A4BB1084B1A6822F006021A6000F084
:1092780013F8204600F039FE4FF48020BDE8104076
:1092880005F0C0BFBC28002010ED00E0014800F048
:10929800FBBF00BFBC280020364BD3F8882042F41F
:1092A8007002C3F88820344B1A6842F001021A6031
:1092B80000229A60196821F0847121F480311960C4
:1092C8002E495960196882B021F480211960DA604A
:1092D800009201921A6842F480321A601A6802F405
:1092E80000320192009A01320092019A1AB9009A4A
:1092F800B2F5A06FF2D1204B1B6813F4003318BFEE
:1093080001230193019B012B2ED11B4B1A6C42F0B8
:1093180080521A641A4A116841F4804111609A68AF
:109328009A609A6842F400429A609A6842F4A0529D
:109338009A60144A5A601A6842F080721A60196872
:109348000D4A8901FBD5104B40F2056119609368FD
:1093580023F003039360936843F0020393609368D8
:1093680003F00C03082BFAD1024B4FF000629A600D
:1093780002B0704700ED00E00038024010300024D1
:109388000070004008544007003C0240184B194A3E
:10939800996801F00C01042903D0082903D0164B61
:1093A80019E0164B17E059685A6811F4800F59688C
:1093B80014BF124B104B02F03F02B3FBF2F30C4AFE
:1093C8005268C2F30142C1F38811013252004B4383
:1093D800B3FBF2F3074A1360054B9A68054BC2F3D7
:1093E80003129A181968127921FA02F21A60704762
:1093F80000380240980200200024F40000127A008D
:1094080037B51C230124002501A88DF804308DF8F8
:1094180005508DF806408DF80740FFF79DFC204663
:10942800214606F05FFD0A4941F287334B6040F25E
:109438004F130B800D814D804FF0804007F0FAF8F4
:109448004FF080402146224607F0B9FC3EBD00BFE0
:10945800002F002008B54FF08040012107F0C4FC20
:1094680040B14FF08040012107F0C9FCBDE8084039
:10947800FEF780BA08BD00BF08B5402005F0B4FE6D
:1094880030B1FCF78BFD4020BDE8084005F0BABEBE
:1094980008BD0000014608B5044807F06FFE034800
:1094A800402107F018FF0028F9D008BD004400400B
:1094B800F0B589B04FF4E1330120019300232B4C20
:1094C800ADF808301E460146ADF80A30ADF80C304C
:1094D800ADF810300C23ADF80E3006F0DFFC4FF479
:1094E8000030012106F0FEFC20680221072206F068
:1094F800ADF907226068032106F0A8F901250227C3
:1095080004232068059305A98DF81A608DF81B506F
:109518008DF818708DF8197006F018F9082360682E
:10952800059305A98DF8187006F010F9A06801A92F
:1095380007F07AFD2A4640F225510D4807F0B2FEA1
:10954800262307A88DF81C308DF81D608DF81E6045
:109558008DF81F50FFF700FCA068294607F0E1FDD1
:10956800044A054B1A6009B0F0BD00BFAC020020E8
:10957800004400409D940008403E0020024B98683B
:10958800002107F0CEBD00BFAC02002010B5094C89
:1095980040F22551204607F0A8FE50B1A288D2B269
:1095A800112A02D1044B01211970044B19884A4031
:1095B8001A8010BD00440040E50E0020F00E002087
:1095C8007047704773B50120014606F067FC264CCA
:1095D8004FF4D8530093022303268DF80430204615
:1095E800002369468DF806308DF807308DF8056040
:1095F80006F0ACF8204608210A2206F027F9204692
:1096080009210A2206F022F920460B210A2206F037
:109618001DF90A2220460C2106F018F901254FF4FD
:1096280080632046694600938DF806508DF80750F0
:109638008DF8056006F08AF80A210A46204606F0E9
:1096480005F929464FF4804006F058FC8020294649
:1096580006F030FC4FF08050294606F07FFC284683
:1096680005F0D0FD7CBD00BF0000024007B54FF4F7
:10967800C060FFF767FB43238DF804300322012302
:1096880001A88DF805308DF806208DF80730FFF712
:1096980063FB0EBD782358430723B0FBF3F0002388
:1096A80001338342FCD970474FF47A735843F1E78A
:1096B80037B50023104C019305460320FFF7EAFF56
:1096C800EB681A69013C019213D0019A002AF4DA76
:1096D800019A42F001020192019A1A61064A196937
:1096E800013A019102D00199C907F8D40320FFF784
:1096F800D1FF00203EBD00BF410D030010B5C47866
:1097080074B900EB820003339B10D0F8D0002246D6
:1097180003E051F8044C0132046004319A42F8D154
:10972800002010BD033230B59210D0F8D0400B465F
:10973800002003E02568013043F8045C04339042BC
:10974800F8D101EB800030BD0122F0B50023827012
:1097580040220129C37082800CD10823037004239E
:1097680043704FF4A073C38002230372C1724FF099
:10977800A04309E041B90C230370062343704FF45A
:10978800A063C3801F4BC17203F500620261C3600E
:109798004678044601461A46002508E002F5106C92
:1097A80002F530620A65C1F814C001353A46043141
:1097B800B54202F12007F1D303F58062426103F557
:1097C8008862C0F8CC20067803F5A065014600221F
:1097D80003E0C1F88C50013220350431B242F8D38D
:1097E8001946002202E0C4F8CC1001320434B24217
:1097F80001F58051F7D303F56063C0F80C31002000
:10980800F0BD00BF0000044038B5037AC2680025E7
:10981800012B044625D1936B417A65F3104309B1B6
:1098280043F480139363D36823F4800323F0500335
:1098380043F010036FF3C3036FF3C7136FF3514380
:109848006FF3D343D3602046FFF732FFE378012B51
:109858003ED1052363F34405E36845F020059D6088
:1098680036E0D36843F04003D360FFF721FF237A43
:10987800627A032B14BF4FF434134FF43C130AB12C
:1098880043F48013E26814209363FFF70DFFE26846
:10989800217AD368032908BF43F48033D360237A3D
:1098A800032B15D1156B012363F39B656FF3D75514
:1098B8002D2345F0805563F316451563C820FFF73F
:1098C800F3FEE36845F400051D63C820FFF7ECFECE
:1098D800E378012B07D1E3689D68052262F344050C
:1098E80045F020059D60002038BDC3689A6842F0A5
:1098F80001029A6000207047C3689A6822F001024A
:109908009A600020704707B500230193019B43F03C
:1099180020030193019B61F38A130193019BC268A1
:109928001361064B1169013B019102D00199880628
:10993800F8D40320FFF7AEFE00200EBD410D030052
:1099480007B500230193019B43F010030193019B8A
:10995800C2681361064B1169013B019102D001995C
:10996800C906F8D40320FFF795FE00200EBD00BFFE
:10997800410D030008B5C268D36801296FF35D7310
:109988006FF39E7302D143F0005302E009B943F02C
:1099980080433220D360FFF787FE002008BDC368EC
:1099A800586900F001007047C3685B6913F0010F44
:1099B80014BF002001207047C368586900F00100F7
:1099C8007047C3685A69986910407047C3685868F7
:1099D800704703691A6861F301021A607047C26828
:1099E800002393614FF0FF335361536053610B4B76
:1099F8009361C3789169002B14BF4FF400634FF44F
:109A0800016343F4701343F4405343F0080321EA1D
:109A180003010B4393610020704700BF00080080DA
:109A2800F8B5D0F80C3100221A60036915461A6897
:109A380065F3CC221A60C37A012B04461BD103219B
:109A4800FFF7C7FFE36880214FF4800261F30F023C
:109A580059629A62C02262F30F0561F31F454FF401
:109A6800A072C3F8045162F30F056FF31F45C3F8E2
:109A78000851C3F80C5110212046FFF744FF204637
:109A8800FFF75EFF226900234FF0FF311361204684
:109A980053611E469161FF25D361214610E082691A
:109AA8001768C7F3076707F08007FFB2002F14BFD6
:109AB8004FF0904700271760013316610430956016
:109AC80062789342EBD300231D46FF2010E04A6DD5
:109AD8001668C6F3076606F08006F6B2002E14BFB5
:109AE8004FF09046002616600133156104319060EE
:109AF80062789342EBD323691A6942F480721A613F
:109B0800E278012A04D1054A402161F359421A63D7
:109B18002046FFF764FF0020F8BD00BF03010100E5
:109B280003699B68C3F34103013B022B9ABF024AB6
:109B3800D05C0320704700BF10DE040810B503692D
:109B480081699C680A68C4F34100022802D06FF357
:109B58000A0202E0032060F30A020A605A6842F42B
:109B680080725A60002010BD30B54D780B78002205
:109B7800012D00EB830405D105FA03F3A46963F30F
:109B88000F0205E0012505FA03F3646D63F31F4234
:109B98002368C3F3072505F08005EDB26DB98D681C
:109BA80065F30A03CD78C98865F3934361F3995344
:109BB80043F0805343F4004323600369D9690A439F
:109BC800DA61002030BD30B54D780B780024012DC6
:109BD800224600EB830105D105FA03F3896963F393
:109BE8000F0205E0012505FA03F3496D63F31F42EF
:109BF80003696FF3CF340C60D96921EA0202DA6194
:109C0800002030BDF8B54F780B78012F00EB8303A7
:109C180049D19E694C69356833692A4664F3120351
:109C280014B967F3DC430BE08F68E419013CB4FB1B
:109C3800F7F7CC7867F3DC43012C08BF64F35E7355
:109C48003361C378012B06D10B780C6900EB8303D1
:109C58009B695C610CE0CB78012B09D04B693BB167
:109C680003690C785E6B012707FA04F434435C63DC
:109C7800CB78012B07D103699B68DB0554BF45F0FE
:109C8800005245F080520B7800EB830342F0044207
:109C98009B691A60CB78012B38D10A788B8AC968FE
:109CA800FFF72CFD32E05E6D4F6935688C683369CB
:109CB8002A462FB964F31203012464F3DC430AE053
:109CC8003F19013FB7FBF4F7BF05BF0D67F3DC434E
:109CD8007C4364F312033361C378012B05D10B78FD
:109CE8000C6900EB83035B6D5C61CB78012B06D1BB
:109CF8004B7913B145F0005201E045F080520B78E2
:109D080000EB830042F00442436D1A600020F8BD66
:109D180073B54D78012D3DD183694A691E681C6968
:109D28000094E4B242B962F306048DF800409DF84D
:109D3800024065F3C4040EE08D68AA4286BF4D61F7
:109D480065F3060462F306048DF800409DF80240AE
:109D5800012262F3C4048DF80240009A1A61C278A5
:109D6800012A05D10A780C6900EB820292695461D4
:109D780046F004421A60C378002B34D14B69002B9B
:109D880031D003690A78586B012101FA02F20243C3
:109D98005A6328E00B784E698C6800EB83035B6D8F
:109DA8001A681D690095EDB206B14C6164F30605A9
:109DB8009DF802408DF80050012565F3C4048DF824
:109DC8000240009C1C61C378012B05D10B780C69FB
:109DD80000EB83035B6D5C610B7800EB830042F062
:109DE8000442436D1A6000207CBD4B78012B0B7830
:109DF80000EB83000AD182691368C3F3076101F09D
:109E08008001C9B221B143F0804301E0426D13687B
:109E180043F400131360002070474B78012B0B7834
:109E2800C97800EB83000CBF8269426D0239136860
:109E3800C9B26FF35553012998BF43F0805313609B
:109E48000020704703699A69D8691040000C704770
:109E580000EB810102694B6D9B685069184070479F
:109E680003699869DB69184080B2704782B00023A3
:109E78000093C0238DF803300122002362F3C4034A
:109E88008DF8023018238DF80030009A436D1A615E
:109E9800C278012A06D100F5B96058611A684FF0F6
:109EA80080221A6002B07047D0F8143110B5044609
:109EB800D3B103699A68D20716D5827A42B1D0F82D
:109EC8000C21D0F80C116FF341026FF300020A6005
:109ED8005A6842F001025A600520FFF7E5FB236942
:109EE8005A6822F001025A6010BD837A63B103698F
:109EF8009B68D90708D5D0F80C31D0F80C216FF33E
:109F080041036FF3000313607047012310B500226B
:109F180080F8123104460346FF2104E05869816045
:109F2800186D01328160607804338242F6D3236968
:109F380000221A615A61DA614FF0FF329A612046B5
:109F4800FFF7FEFC20461021BDE81040DBE44B780B
:109F5800012B0B7800EB83000FD183691868C0F3DD
:109F6800074000F02003DBB2CBB900F00200C0B21A
:109F780000280CBF302020207047436D1868C0F3BC
:109F8800074000F02003DBB25BB900F00200C0B26A
:109F980000280CBF4FF440504FF400507047102079
:109FA80070474FF4805070474B78012B0B7810B5F1
:109FB80000EB83030AD19C69102A236802D1BDE80B
:109FC800104012E7202A0CD0302A0FE05C6DB2F561
:109FD800805F236802D143F400131BE0B2F5005FF1
:109FE80002D143F0006315E0B2F5405F0FD1C3F32F
:109FF800074202F02002D2B222B100234B71BDE821
:10A0080010400AE743F0806343F0802302E00AB976
:10A0180062F3CF33236010BDF8B50446FFF794FB15
:10A028000122002384F8122184F8133128271646C8
:10A03800194640250CE007FB03F000F58C70221848
:10A048002354D3805670D1709560D160516101332B
:10A0580062789342EFD300232826194640250CE066
:10A0680006FB03F000F55C7022182354D38051706E
:10A07800D1709560D1605161013362789342EFD31A
:10A088002046FFF739FC2046FFF7BEFB002120469B
:10A09800FFF770FC2046FFF7C3FC2046BDE8F840F8
:10A0A800FFF723BC70B5CDB20C464FF0280601F07F
:10A0B8007F0106FB010115F0800F14BF01F58C71BB
:10A0C80001F55C7104F07F04ED090C704D708A6035
:10A0D800CB7005B1CC80022B01D100230B71FFF7A7
:10A0E80043FD002070BD10B5CAB201F07F034FF0E8
:10A0F800280404FB030312F0800F14BF03F58C73CC
:10A1080003F55C7301F07F01D20919705A70194682
:10A11800FFF759FD002010BD38B501F07F05282450
:10A128006C4304F55C7401194B6100238B614B701F
:10A13800EBB20355CA60C478012C08BF0A6113B991
:10A14800FFF7E6FD01E0FFF75DFD002038BD70B5C3
:10A1580001F07F042825654305F58C754119012612
:10A16800E4B2CA600A6100224E7044558A614B61AC
:10A1780014B9FFF7CDFD01E0FFF744FD002070BDE5
:10A18800CAB212F0800F10B54FF0280306D001F0C4
:10A198007F0403FB040303F58C7303E003FB010353
:10A1A80003F55C73D209012401F07F0119709C70DA
:10A1B8005A701946FFF719FE002010BDCAB212F0F6
:10A1C800800F10B54FF0280306D001F07F0403FB81
:10A1D800040303F58C7303E003FB010303F55C73CD
:10A1E8000024D20901F07F0119709C705A70194639
:10A1F800FFF713FE204610BD08B50B0604D501F085
:10A208007F01FFF780FB01E0FFF79AFB002008BD04
:10A218000369002261F30A1219680A431A60704739
:10A2280003695A6803206FF341025A60FFF73CBA8A
:10A2380003695A68032042F002025A60FFF734BAF1
:10A2480011F0800F4FF0280306D001F07F0103FBC7
:10A25800010101F58C7103E003FB010101F55C715B
:10A26800FFF775BE11F0800F4FF0280306D001F0FC
:10A278007F0103FB010101F58C7103E003FB010180
:10A2880001F55C71FFF790BE2DE9F74F0446FFF723
:10A298008BFB002800F03F822046FFF792FB054623
:10A2A800002800F03882C0F3074000F00800C0B270
:10A2B800002861D02046FFF7C5FDA1468246274603
:10A2C8004FF00008DFF86CB32E4650E01AF0010F8B
:10A2D80046D05FFA88F2114620460092FFF7B8FD93
:10A2E80010F0010F0546009A20D07B6D01259D6076
:10A2F800E178A94207D11B69D9F87813C3F312038F
:10A30800CB1AC9F88833DBF8003020461B681146A1
:10A318009847E378012B09D1B8F1000F06D194F8DA
:10A328001131052B02D12046FFF7A0FD05F00203ED
:10A33800DBB213B17B6D02259D6005F00403DBB22F
:10A3480013B17B6D04259D6005F00805EDB23DB1A4
:10A35800DBF8003020469B6898477B6D08209860A2
:10A3680008F101084FEA5A0A043709F12809BAF135
:10A37800000FABD135460120C5F3074303F00403B2
:10A38800DBB2002B00F0AF802046FFF769FD2646C0
:10A3980083464FF0000801959FE01BF0010F00F085
:10A3A800978023695FFA88F919695D6B04EB890264
:10A3B80025FA09F59269ED019268EDB20D43154051
:10A3C800EA071CD55A6B012000FA08F122EA0102BB
:10A3D8005A63B369974A9860136805465B682046D4
:10A3E80049469847E378AB4209D1B8F1000F06D146
:10A3F80094F81131042B02D12046FFF737FD05F000
:10A408000403DBB213B1B36904259D6005F00803AA
:10A41800DBB213B1B36908259D6005F01003DBB208
:10A4280013B1B36910259D6005F02003DBB213B1A9
:10A43800B36920259D6005F04003DBB213B1B36911
:10A4480040259D6005F00203DBB213B1B369022514
:10A458009D6025F07F0515F0FF0F39D0282505FBF5
:10A46800084505F58C75C246AB696A69C3EB020CF1
:10A47800AB689C4528BF9C460CF1030CB3694FEAB6
:10A488009C0C9B696746A04614E0AA68E9681C1BF7
:10A49800944228BF1446A3B240464A46FFF72EF915
:10A4A800EB681B19EB60AB69E71C1C19AC61B3695D
:10A4B8009B69BF089BB2BB4205D9AC696B699C42DA
:10A4C80001D2002BE1D1B369802544469D60D04676
:10A4D80008F101084FEA5B0B0436BBF1000F7FF46B
:10A4E8005CAF019D012005F00203DBB213B1E36804
:10A4F80002225A61C5F3076303F08003DBB2CBB1D4
:10A50800A37A43B1D4F80C31D4F80C216FF341038A
:10A518006FF30003136023695A6822F001025A603E
:10A52800444B1B6820469B699847E3684FF00042FC
:10A538005A610120C5F3072303F00803DBB2F3B126
:10A548003C4B1B6820465B6998472369E2689B6817
:10A558004FF400615161A27A82B1DB070ED5D4F8BD
:10A568000C311A6842F001021A601A6842F00302BC
:10A578001A60314B1A6942F006021A61012005F08F
:10A588000803DBB243B12B4B1B682046DB689847B6
:10A59800E36808225A61012005F01003DBB2002BA2
:10A5A80033D0E3689A6922F010029A611F6A28265C
:10A5B80007F00F0306FB0346C7F34343022B06F5D8
:10A5C8005C7602D0062B1AD10EE047F6F0733B40BA
:10A5D800ABB1C7F30A172046F1683A46FFF7A2F86D
:10A5E800F368DB19F36007E004F5B9612046082237
:10A5F800FFF798F8C7F30A17B369DF19B761E3687B
:10A608009A6942F010029A610120C5F3072303F00A
:10A618001003DBB2002B39D023695A68002622F0D8
:10A6280001025A6031462046FFF76DF9234632464B
:10A63800FF2108E04803002000ED00E05869816030
:10A64800186D01328160607804338242F6D3236941
:10A6580001274FF0FF3267F30F069A6167F31F4631
:10A668000F22DE615A612F221A611A686FF30A12EB
:10A678001A602046FFF7FAFBE3684FF480525A61EC
:10A68800264B1B6820461B6998473846C5F30723A5
:10A6980003F02003DBB2EBB12046FFF74FFAE36883
:10A6A8002046DE68FFF73CFA032806D10023A37092
:10A6B8004FF40073A380092304E00123A37040230F
:10A6C800A380052363F38D26E3684FF40052DE6010
:10A6D80001205A61C5F3074303F01003DBB24BB105
:10A6E8000E4B1B682046DB699847E3684FF48012DD
:10A6F8005A610120C5F3074505F02005EDB255B1B3
:10A70800064B1B6820461B6A9847E3684FF4001203
:10A718005A610120FFE7BDE8FE8F00BF4803002013
:10A7280043230B8000487047B802002038B51F4B00
:10A738001A68511C052A196035D119790022012996
:10A748001A6030D09968B1F5006F08BF9A60174B4E
:10A758009968DC68A1421A4602D100221A7122E0E7
:10A7680086BFC1F500631361C1EB0404D0F8EC3572
:10A7780098BF14611569B3F839300C4C9D428AB200
:10A7880004D95918ED1AA160256104E06918A1607F
:10A798000021ABB22161054901240C7104498A18D2
:10A7A8008121FFF7D4FC002038BD00BFF40E002043
:10A7B8009F2F002038B528230A4D03FB01010A4BBF
:10A7C800B1F888131B69044628469847D4F8EC3535
:10A7D8002046B3F8403001212A46FFF79DFC0020AF
:10A7E80038BD00BF572F00203403002070B50B7808
:10A7F80013F0600506460C4625D0202D1FD1CD88C4
:10A80800B5B113F0800F487808D0214B21499B68D7
:10A818002A469847E2881F49304625E01E4B1D49C5
:10A8280058641E4B30465D612A4600F022FB1DE04D
:10A83800174B48789B6829462A46984725E000F038
:10A8480077FB022521E04B780A2B11D00B2B14D073
:10A85800062B1AD14B881B0A212B03D1CA883A2A06
:10A8680028BF3A220E49304600F0EAFA00250CE0EB
:10A878000C49012200F0E4FA07E08B781BB9074A7B
:10A888001D46936101E000F053FB284670BD00BFF0
:10A8980034030020972F0020B8020020F40E002077
:10A8A800CA0200200C0F002010B581210446FFF7D2
:10A8B8001AFC01212046FFF716FC82212046FFF7EB
:10A8C80012FC024B5B689847002010BD340300203F
:10A8D80038B5D0F8EC350446B3F839208121022385
:10A8E800FFF7E0FBD4F8EC350121B3F8402020460F
:10A8F8000223FFF7D7FB8221082203232046FFF714
:10A90800D1FB094B022200251A715D71074B1B68A8
:10A918009847D4F8EC35064AB3F840302046012170
:10A92800FFF7FAFB284638BD7803002034030020DF
:10A93800572F002010B5074C606CFF2807D0064B36
:10A94800064A9B68064952699847FF2363640020BA
:10A9580010BD00BFB802002034030020F40E002010
:10A96800972F002038B510490B79012B19D10C69A4
:10A978000CB90C7115E0D0F8EC358D68B3F83930A6
:10A988009C42AAB203D95D198D60E41A03E0A3B210
:10A998002C198C6000240C61044952188121FFF79E
:10A9A800D6FB002038BD00BFF40E00209F2F0020EA
:10A9B80000207047002070470023F0B5084A094E70
:10A9C8001D4609E01468C75C375501340133B4F5F6
:10A9D800006F146008BF15608B42F3D10020F0BDF2
:10A9E800000F00209F2F0020104B114AD3F800C001
:10A9F80000232DE9F0410F4F16461D460DE014685F
:10AA080010F8038007F804800134802C08BF2C4616
:10AA180014603468644505D001338B42EFD10020BF
:10AA2800BDE8F0810220BDE8F08100BF2038002099
:10AA380034380020A037002021280FD1084B1A688D
:10AA48000A701A68120A4A705A888A70DA78CA70C4
:10AA58001A790A715A794A719B798B71002070476B
:10AA68002C03002007B502AB012103F8010D18469D
:10AA7800FFF7A2FF0EBD002100E00131435C002B6F
:10AA8800FBD199E798E70B4B0B491A680968914283
:10AA98000BD00A498A5C02701A680132802A1A604F
:10AAA80005D100221A60012070470020704701205C
:10AAB800704700BF2038002034380020A03700201D
:10AAC800204B1A68204B1B689A42F0B509D135E033
:10AAD8000133802B08BF00239A4203D11A4B1A6016
:10AAE8002CE01A4CE15C0029F2D00A29F0D00D299B
:10AAF800EED0154C1549134D23600E460023CF1890
:10AB08002268BA5CC254226801339F18802F08BF9C
:10AB180053422F689A18974210D0B25C1AB10A2A89
:10AB280001D00D2AEBD10022C254074A11685918E6
:10AB38007F29116003D98039116000E0002318468D
:10AB4800F0BD00BF3438002020380020A037002096
:10AB5800704700BFD0F8E43510B51B690446984724
:10AB6800032384F81231002010BD08B5042380F8AF
:10AB78001231D0F8E435DB689847002008BD08B5E5
:10AB8800D0F8E035DB6903B19847002008BD08B567
:10AB9800D0F8E0351B6A9847002008BD08B5D0F802
:10ABA800E0355B6A9847002008BD002110B54022B7
:10ABB80004460B46FFF776FA802140220023204600
:10ABC800FFF770FA012384F81231D4F8E435A0783D
:10ABD8005B689847002010BD13B56946044600F02D
:10ABE80085F99DF8001001F01F03012B07D0022BF7
:10ABF8000AD073B92046694600F026FA0FE02046CD
:10AC0800694600F007FA0AE02046694600F0A2F912
:10AC180005E021F07F01C9B22046FFF7B1FA002014
:10AC28001CBD38B5044600293DD190F81131022BDE
:10AC380042D1D0F83421D0F820319A4211D9C178C4
:10AC4800D21A0129C0F8342104D1D0F82411CB1824
:10AC5800C0F8243192B22046D4F8241100F000F94B
:10AC68002AE0D0F83821B2FBF3F503FB152565B9C6
:10AC78009A420AD3D0F83C319A4206D229462A464B
:10AC880000F0EEF8C4F83C5116E0D4F8E035DB6883
:10AC98002BB194F81221032A01D120469847204667
:10ACA80000F00FF908E0D0F8E0355B6923B190F8BF
:10ACB8001221032A00D19847002038BD10B5044658
:10ACC80059BB90F81131032B30D1D0F88C23D0F830
:10ACD80078339A4214D9C178D21A0129C0F88C2342
:10ACE80004D1D0F87C13C918C0F87C139A4228BF45
:10ACF8001A4692B22046D4F87C1300F0CAF815E040
:10AD0800D0F8E0351B6923B190F81221032A00D14D
:10AD18009847204600F0C6F808E0D0F8E0359B696F
:10AD280023B190F81221032A00D19847002010BDC2
:10AD38002DE9F041069F0446164698460D46FEF753
:10AD480041FC20462946C4F8E085C4F8E475C4F8F7
:10AD5800E865FFF761F9D4F8E4351B6898472046A1
:10AD6800BDE8F041FEF782BC00207047D0F8E0351E
:10AD780010B504461B689847D4F8E4359B68984793
:10AD8800002010BD08B5D0F8E0355B689847002072
:10AD980008BD000012230B8000487047780300208C
:10ADA80004230B80004870478A03002010B5044C28
:10ADB80004480A46214600F075FA204610BD00BF37
:10ADC800383800204AE305080A4608B5024803490E
:10ADD80000F068FA014808BD5DE30508383800202E
:10ADE8000A4608B50248034900F05CFA014808BD64
:10ADF8006BE305083838002008B50A4608B9044846
:10AE080000E00448044900F04DFA034808BD00BFBB
:10AE180076E3050883E305083838002008B50A46B4
:10AE280008B9044800E00448044900F03BFA034824
:10AE380008BD00BF90E30508B1E3050838380020D5
:10AE480010B513460C46C0F83821C0F83421022248
:10AE580080F8112100212246FFF779F9002010BD62
:10AE680010B50C46134600212246FFF770F9002062
:10AE780010BD10B513460C46C0F89023C0F88C23BB
:10AE8800032280F8112100212246FFF745F900200E
:10AE980010BD10B50C46134600212246FFF73CF9B9
:10AEA800002010BD0021042310B50A46044680F88E
:10AEB80011310B46FFF74BF92046FEF7D7FF00206C
:10AEC80010BD0021052310B50A46044680F811314B
:10AED8000B46FFF721F92046FEF7C8FF002010BDFA
:10AEE800282303FB0100B0F88803704790F8C835A1
:10AEF8000B7090F8C9354B7090F8CB2590F8CA358F
:10AF080003EB02234B8090F8CD2590F8CC3503EB6A
:10AF180002238B8090F8CF2590F8CE3503EB0223DF
:10AF28009BB2CB80C0F83C31012380F811317047C7
:10AF380010B591F90030002B044601DBCB880BB922
:10AF4800802100E00021FFF71BF92046BDE81040F2
:10AF5800FEF78CBF38B50D4604466B780979012B8E
:10AF680010D027D3032B51D190F81231022B28D0BF
:10AF7800032B47D16B889BB991B1802910D0FFF77B
:10AF8800FFF80DE090F81231022B1AD0032B39D1BB
:10AF98006B88002B3AD149B1802907D0FFF70EF909
:10AFA800D4F8E03520469B68294698472046FFF7A5
:10AFB80079FF2BE090F81231022B02D0032B21D11C
:10AFC80006E019B3802921D02046FFF7D9F81DE003
:10AFD80011F0800F4FF0280306D001F07F0103FB2A
:10AFE800010393F81A2103E003FB010191F872238E
:10AFF800074B02B101221A60204605490222FFF7D9
:10B008001FFF03E020462946FFF792FF002038BDC6
:10B01800100F002038B590F81231032B04460D4666
:10B028000CD10B79012B09D8D0F8E0359B689847EB
:10B03800EB883BB92046FFF735FF03E02046294659
:10B04800FFF776FF002038BD73B54B7804460D46F0
:10B05800092B00F21C81DFE813F0D10008011A0166
:10B06800E4001A0172000A001A01C00092004B881D
:10B078001A0A013A062A00F20A81DFE812F00700EC
:10B088001A0027000801080108010801D4F8E8356A
:10B09800A0781B680DF106019847EB88402B014604
:10B0A80003D094F81231012B3AD10823ADF80630B9
:10B0B80036E0D4F8E035A0789B6A0DF10601984790
:10B0C800022343700146C4F8EC0529E0DBB2052BE6
:10B0D80000F2DD80DFE803F003080D12171CD4F836
:10B0E800E835A0785B6817E0D4F8E835A0789B6865
:10B0F80012E0D4F8E835A078DB680DE0D4F8E8353C
:10B10800A0781B6908E0D4F8E835A0785B6903E00B
:10B11800D4F8E835A0789B690DF1060198470146F7
:10B12800BDF80630002B00F0B680EA88002A00F04F
:10B13800B2809A4228BF1A46ADF806205CE08B8898
:10B14800002B40F0A480CB88002B40F0A08094F81E
:10B1580012214B88032A00F09A8003F07F052046CD
:10B1680084F813512946FFF753F82046FFF79AFE53
:10B178000DB1022300E0012384F812318BE08978B5
:10B18800464E0129317100F2828094F81231022B67
:10B1980002D0032B7BD108E0002962D001210323D0
:10B1A80084F8101184F8123113E041B9022384F8AD
:10B1B800123184F810112046FFF7E4FD51E094F8AD
:10B1C8001011012920464DD0FFF7DCFD317984F8B4
:10B1D80010112046FFF7CAFD43E0CA88012A56D15C
:10B1E80094F81231022B02D0032B50D102E02046F2
:10B1F8002B4913E004F5887120460FE094F81231CA
:10B20800023B012B43D8D4F814312449002B0CBF3E
:10B218000123032341F80C3F20460122FFF710FECB
:10B2280039E04B88012B29D0022B34D18B8813F0BD
:10B23800FF0F30D121691B0A013B4A68042B0FD844
:10B24800DFE803F0030507090B00012306E00223EA
:10B2580004E0032302E0042300E0052363F306125D
:10B268004A602046FFF71EFE15E094F81231023BB3
:10B27800012B0CD84B88012B0DD10023C4F81431B5
:10B28800D4F8E03520469B6829469847E9E72046E8
:10B298002946FFF74DFE00207CBD00BF100F00209F
:10B2A800180F002030B5C8B10023DDB20133C4182F
:10B2B80014F8014C002CF8D16B1C5B0013800B7048
:10B2C80003234B70022305E0CA545A1CD2B202333E
:10B2D8008C54DBB210F8012B002AF5D130BD00BF29
:10B2E8007047704770477047704770477047000055
:10B2F80008B5FCF76DFA094B5A78187002435A7072
:10B308001AB19A7801329A7030B99B78034A012BA6
:10B3180002D900235370937008BD00BF200F00208E
:10B328002DE9F84F394B1A78394B2DED028B22B99C
:10B338001A68802392FBF3F300E01B68354A5361D7
:10B34800354B1A8892B2002AFBD0334B00221A8060
:10B35800FDF7A6FD10EE105AFDF7A8FD284610EEE1
:10B36800104A06F04DF980462046894606F048F90D
:10B3780041EC100B41EC180B08F0C2F957EC106BBC
:10B38800B0EE480AF0EE680A08F0BAFA32463B46D0
:10B39800404649465BEC10AB06F086F906F066FCC1
:10B3A8009FED1E8A07EE100ADFED1D7A57EE087A28
:10B3B800184C52465B46C4ED007A4046494606F0B2
:10B3C80073F906F053FC07EE900A27EE888A84ED9D
:10B3D800018AFDF77DFD84ED020AFDF77FFD84ED0E
:10B3E800030AFCF703F90F4B62691B68D31A0E4A6C
:10B3F80007EE100A1268F8EEC77A93FBF2F3C4ED71
:10B40800047A2383BDEC028BBDE8F88F840F0020FB
:10B41800B42E00206C3A0020D20E00200000F0422A
:10B4280000008C42B02800203428002007B50420F2
:10B43800012104F033FD4FF46043009301238DF89C
:10B44800043002238DF805300448002369468DF83E
:10B4580006308DF8073004F079F90EBD0008024077
:10B46800084B1A684FF47A73B2FBF3F2064B013AB1
:10B478005A60064AF02182F8231000229A600722B7
:10B488001A6070479802002010E000E000ED00E02C
:10B49800034B5A6812B15A68013A5A60704700BFA4
:10B4A800200F0020024B58605A68002AFCD17047D0
:10B4B800200F002030B585B004460D4601A85C4930
:10B4C8000A220AF015FE5B4B1B78032B10D8DFE825
:10B4D80003F00205080B01A8574907E001A85749DE
:10B4E80004E001A8564901E0564901A80AF0EAFE1D
:10B4F80004AA131913F80C3C5D19EDB22F2D01D8CD
:10B508000A3502E0392D01D90A3DEDB204AB1C1908
:10B518004FF6FF7004F80C5CFAF7A8FA0020FAF767
:10B52800A7FB0DF103050F24204623345A210023DD
:10B5380015F8012FA4B2FAF7B5FBB4F5A57FF3D13E
:10B5480064205A212C220023FAF7ACFB0023CD20DB
:10B558005A212C22FAF7A6FB0020FAF787FA354B76
:10B568001B78032B62D8DFE803F002284B5601A9A9
:10B5780031480AF0A7FE0A2200212F480BF0CAFF23
:10B58800314A324B12781860012A06D1304A90426B
:10B5980001DC01321A602F4A06E0B0F5FA5FBCBF41
:10B5A8004FF4FA521A602C4A1B689342C4BF274BC7
:10B5B8001A602A4B1A682A4B20E001A91F480AF092
:10B5C80081FE0A2200211D480BF0A4FF1E4A254BCC
:10B5D80012781860012A06D11D4A904201DC013216
:10B5E8001A601C4A06E0B0F5FA5FBCBF4FF4FA5285
:10B5F8001A60194A1B68934218DD1A4B1A6015E045
:10B6080001A90F480AF05EFE0D4800210A220BF03E
:10B6180081FF154B09E001A90A480AF053FE0948C1
:10B6280000210A220BF076FF104B186005B030BDE0
:10B63800D2E30508AF2800207C280020A428002099
:10B64800BA2E002068280020840F0020B828002087
:10B658001FA1070080D1F00850DA1100B02800209F
:10B66800B42E0020D82E0020AC2E00206428002004
:10B6780010B50D4B0D4C1A680D4821460AF0FAFD1D
:10B688000C4B0D481A6821460AF0F4FD0B4B0C4888
:10B698001A6821460AF0EEFD0A4B0B481A68214643
:10B6A800BDE810400AF0E6BDB828002046D90508D4
:10B6B8007C280020D82E0020A4280020AC2E0020B2
:10B6C800BA2E002064280020682800209FED010A77
:10B6D800704700BF000000009FED010A704700BFDF
:10B6E800000000009FED010A704700BF0000000045
:10B6F8007047704718B1012801D1034B00E0034B94
:10B708001868FDF743BD00BFA0280020B02800201E
:10B7180010B9034B18687047024B1868704700BF90
:10B72800B8280020B028002010B9034B18687047CB
:10B73800024B1868704700BFD82E0020A0280020B0
:10B7480008B54FF49570FBF765FF40F26523C31AFF
:10B75800584240EB030008BD08B5C620FBF75AFF66
:10B7680040F28D13C21A504240EB020008BD4FF45C
:10B77800957040F26521FBF73FBFC62040F28D115E
:10B78800FBF73ABFDCE760EEA00AB7EE007AF0EE0E
:10B79800606A70EE077A40EE006A47EEA70A36EE56
:10B7A800C77A08B5C7EE200A10EE900A05F028FF00
:10B7B8000022084B05F078FF0022074B05F0C2FD78
:10B7C80006F054FA07EE900AFDEEE77A17EE900AB3
:10B7D8009F3008BD000059400000E03F38B52DED0E
:10B7E800028BF7EE008AB0EE608A70EE288A10EEBF
:10B7F800900A28EE088A05F003FF08EEA88A0022BE
:10B808000F4B05F051FF044618EE100A0D4605F0DF
:10B81800F7FE02460B462046294606F06FF800223E
:10B82800084B05F08FFD06F021FA07EE900AFDEEB1
:10B83800E77A17EE900A7730BDEC028B38BD00BF6F
:10B84800000069400000E03F2DE9F04F884F2DEDE2
:10B85800068B97E80F0091B00CAC103784E80F0006
:10B868000FCF05AE0FC697E807004FF6FF7386E8BF
:10B8780007009F2077216422F7F79DFDA0207721FC
:10B8880064224FF6FF73F7F796FD9E207721642216
:10B898004FF6FF73F7F78FFD9F20762164224FF64E
:10B8A800FF73F7F788FD4FF6FF73782164229F2016
:10B8B800F7F781FD0020F9F798F99F207721652295
:10B8C800FAF716F90C349F2077216422FAF710F959
:10B8D8000DF12C0A0394F7EE009A4FF00F0B00E0DD
:10B8E8004D460AF1040AF7EE008A9AED009A002400
:10B8F800B0EE68AA01E0B846354618EE900A05F0A1
:10B908007FFE59A3D3E9002305F0CEFE06F0AEF979
:10B9180008EE900A38EEE98AB0EE490AF0EE480AD5
:10B92800FFF731FFB0EE490AF0EE480A0646FFF786
:10B9380055FFB2B2074683B22CB9104619460F22FA
:10B94800F9F71EFA06E0A8B21FFA88F1CDF800B0A0
:10B95800FAF718F80134B4F5967FCCD13D46F7EEE6
:10B96800008A002401E045464E4618EE900A05F08C
:10B9780047FE3DA3D3E9002305F096FE06F076F9CD
:10B9880008EE900A39EEE88AB0EE490AF0EE480A65
:10B99800FFF7F9FEB0EE490AF0EE480A8146FFF7D4
:10B9A8001DFF1FFA89F2804683B22CB9104619464A
:10B9B8000F22F9F7E5F905E0B0B2A9B2CDF800B069
:10B9C800F9F7E0FF0134B4F5967FCCD1039B9A4593
:10B9D80086D104AD0DF12C0B4FF0000A01E0B846FA
:10B9E800B146043595ED009AF7EE008A002401E08F
:10B9F800B846B14618EE900A05F002FE1AA3D3E93C
:10BA0800002305F051FE06F031F908EE900A38EEF1
:10BA1800CA8AF0EE490AB0EE480AFFF7B4FEB0EE63
:10BA2800480AF0EE490A0646FFF7D8FEB2B20746C2
:10BA380083B22CB9104619462246F9F7A1F907E056
:10BA48001FFA89F01FFA88F1CDF800A0F9F79AFFDC
:10BA58000134B4F5C87FCBD15D45C0D111B0BDEC80
:10BA6800068BBDE8F08F00BF295C8FC2F528F03F38
:10BA780014DE0408121A06EE902A081AB8EEE67ABE
:10BA880006EE900AF8EEE67A08B5C7EE277A17EEC2
:10BA9800900A05F0B5FD07A3D3E9002305F004FEDD
:10BAA8000022034B05F04EFC06F098F808BD00BFD5
:10BAB8000000E03F0000000000F073408A1A06EE24
:10BAC800902A081AB8EEE67A06EE900AF8EEE67AB8
:10BAD80008B5C7EE277A17EE900A05F091FD07A37F
:10BAE800D3E9002305F0E0FD0022034B05F02AFC12
:10BAF80006F074F808BD00BF0000E03F0000000039
:10BB080000E0684070B506460D460024610704D57C
:10BB1800A0B231462A46F9F733F90134B4F5A07FCB
:10BB2800F4D170BD70B506460D460024600704D5F3
:10BB3800A1B230462A46F9F723F90134C82CF5D1C9
:10BB480070BD114B11481B781149124A0068012B2E
:10BB5800114B09D1126808601A60104B1A68104B13
:10BB68001A60104B1A680CE01268D2011A600B4B6D
:10BB78001A680B4BD2011A600A4B1A68C001086098
:10BB8800D201094B1A607047840F0020B8280020A2
:10BB9800B0280020D82E0020A0280020AC2E00209D
:10BBA800342800208C280020CC2E0020014B186857
:10BBB800FDF7ECBAB028002008B5FFF7C2FFBDE8D2
:10BBC8000840F3E770B500210A222748274D284E80
:10BBD800284C0BF09FFC00210A22286026480BF015
:10BBE80099FC00210A22306024480BF093FC0021C4
:10BBF8000A22206022480BF08DFC224B3268186024
:10BC08002B682149D31A06EE903A2368B8EEE67AF3
:10BC180006EE903AF8EEE67AC7EE277AFCEEE77A77
:10BC280017EE903A9AB20B80531C07EE903AB8EE92
:10BC3800E77ADFED167A67EE277A154BFCEEE76AAE
:10BC480016EE901A8AB206EE902AB8EEE67A1980B5
:10BC580077EEC77AF5EEC07AF1EE10FA01DD01321F
:10BC68001A80BDE87040A7E77C280020B82800208B
:10BC7800D82E0020AC2E0020A4280020BA2E0020A8
:10BC88006828002064280020A43C00200000803D93
:10BC9800343D00200022F0B51346202603254FF03E
:10BCA8002C0C00E02646303EF6B217460132092E2B
:10BCB80010F8014B0AD897FBF5F605FB16772FB954
:10BCC800CE1801F803C07470023301E0CC5401337C
:10BCD800092AE7D12022CA54CB1848225A707A225E
:10BCE8009A700022DA70F0BDF0B51F46144B1E782A
:10BCF800012E8DB005460C4620D0A6F1030CDCF1D0
:10BD0800000646EB0C06CEB90E4908A80AF0B2FAAE
:10BD180008A86946FFF7BEFF0B496A4604A80AF05F
:10BD2800A9FABDF84800F9F7A1FE3846F9F7B4FEBC
:10BD38002846214604AA3346F9F7D2FF0DB0F0BDD4
:10BD48003828002046D90508A7E0050810B50121C4
:10BD58000446F9F73BF8014B1C8110BD200F002069
:10BD680008B50021C620FBF747FC4FF49570002169
:10BD7800BDE80840FBF740BC014B9F221A81704781
:10BD8800200F002000200146C82240F23F13F9F797
:10BD980031B907B50DF10700FEF775FE9DF80700EC
:10BDA8000EBD08B5FFF7F5FF0028FBD108BD30B57B
:10BDB800044687B010EE100A0D4605F021FC024635
:10BDC8000B4601A805490AF055FA2046294601AA5A
:10BDD8000023F9F785FF07B030BD00BFDCE3050895
:10BDE80008B5084802F014FF0648022102F0E1FFF6
:10BDF8000028F9D0034802F037FF07EE900AB8EEA2
:10BE0800670A08BD0020014010B52DED028B9FED9B
:10BE1800098A1924FFF7E4FF013CE4B238EE008AEE
:10BE2800002CF7D19FED040A28EE000ABDEC028B26
:10BE380010BD00BF00000000ACC868392DE9F04F04
:10BE48002DED068B8E4B8F4C8F495D695F68C1B0B5
:10BE58000646324638A893ED038AD3ED04AAD3EDFB
:10BE6800028A93ED00AA93ED069A0AF003FAA068F5
:10BE780005F0C6FB02460B4628A884490AF0FAF9E1
:10BE8800E06805F0BDFB02460B462CA880490AF085
:10BE9800F1F91AEE900A05F0B3FBCDE90801DDE9E6
:10BEA80008237C4930A80AF0E5F9284605F0A8FBE4
:10BEB800CDE90401DDE90423774934A80AF0DAF969
:10BEC80018EE900A05F09CFB8046894642464B4690
:10BED800724910A80AF0CEF918EE100A05F090FB86
:10BEE80082468B4652465B466D4914A80AF0C2F951
:10BEF8001AEE100A05F084FBCDE90A01DDE90A23F0
:10BF0800684918A80AF0B6F9384605F079FB54A331
:10BF1800D3E90023CDE9060105F0C6FB02460B462E
:10BF28001CA861490AF0A6F949EC118B4BEC10AB3F
:10BF380007F042FD4AA3D3E9002351EC100B05F0AA
:10BF4800B3FB02460B4624A858490AF093F919EEA8
:10BF5800100A05F055FB02460B4620A854490AF082
:10BF680089F9D4ED047AFDEEE77A0CA817EE902A49
:10BF780050490AF07FF9B5EEC08AF1EE10FADFED0C
:10BF88004E9A37D5304605F029FB37A3D3E900236D
:10BF980005F08AFBF1EE487A044617EE900A0D4642
:10BFA80005F02EFB02460B462046294605F07CFB91
:10BFB80002460B462EA1D1E9000105F09FFC05F0D1
:10BFC80055FE9FED3E7A07EE900AF4EEC77AF1EE41
:10BFD80010FAC6BFC7EEA97A394C3A4CF4EEE97AA2
:10BFE800F1EE10FA38DD9FED347A374D374CC7EE55
:10BFF800877A76E020A3D3E900235046594605F016
:10C0080053FB044630460D4605F0E8FA16A3D3E97B
:10C01800002305F049FB02460B462046294605F059
:10C028006DFC05F023FE07EE900AB7EE007AF4EEF9
:10C03800C77AF1EE10FA46BF67EEA97A244C254C70
:10C04800F4EEE97AF1EE10FA4ADD9FED1B7A224D03
:10C05800224CC7EE877A44E01B4D42E0AFF30080E4
:10C068006666666666A64C401F85EB51B81E194089
:10C07800000000A2941A6D420000000080842E4146
:10C08800543C00206C3A0020FCE3050806E405084F
:10C0980011E405081CE4050826E4050830E4050851
:10C0A8003CE4050848E4050853E405085EE405088F
:10C0B80069E4050875E4050800007A440024744919
:10C0C800EDE30508EAE305088EE30508F6E305084D
:10C0D800F3E30508F0E3050884E20508F9E3050839
:10C0E800954D17EE900A05F08BFA2A46CDE9000126
:10C0F8003CA8924902940AF0BDF8914B1A68914BFA
:10C108001B689642CCBF002201229E428E4BD8BFAC
:10C118000022DA608D4B1B78082B40F09C800220AF
:10C12800F9F7A6FD4FF6FF70F9F7B6FC1F20F9F7EF
:10C138009DFC19210023864A2D20F9F7D1FD4FF6E1
:10C14800FF70F9F7A9FC00200024F9F78FFC0F20F5
:10C15800B42132464FF6FF730094FFF7C5FD0F2058
:10C168006E2128AA2346F9F7BBFDB0206E210DEBFE
:10C1780000022346F9F7B4FD0F20382118AA2346F8
:10C18800F9F7AEFDB02038211CAA2346F9F7A8FD1F
:10C198000F205C2130AA2346F9F7A2FDB0205C21CC
:10C1A80034AA2346F9F79CFD0F204A2110AA2346FA
:10C1B800F9F796FDB0204A2114AA2346F9F790FD15
:10C1C8000F209B2120AA2346F9F78AFD0F208421FE
:10C1D8003CAA2346F9F784FDB020842124AA2346EB
:10C1E800F9F77EFD5B4B1B68B3F57A7FCCBF4FF444
:10C1F800FC604FF47840F9F74FFC0023A0209B2106
:10C208000CAAF9F76DFD544B1B78012B08D14FF49C
:10C21800FC60F9F741FC4FF48C7002214F4A07E0AB
:10C228004FF6E070F9F738FC4D4A4FF48C70022154
:10C238000023F9F755FD0020F9F72EFC4FF4FC60B8
:10C24800F9F714FCFFF7E0FD0F20DC21FFF7AFFD45
:10C258001F20F9F721FC3D4B1B789A1FD2B2012A07
:10C2680002D90B2B40F025823E4B1B78023B052B55
:10C2780000F21F82DFE813F006007E00E2003B01B7
:10C28800DE015801DFED387A2AEE27AA1AEE100AE5
:10C2980005F0B6F99DED060B8046894607F030FAA1
:10C2A800404653EC102B494605F0FEF91EA3D3E98E
:10C2B800002305F047F805F091FC9DED060B0446B8
:10C2C80007F01EFB404653EC102B494605F0ECF9ED
:10C2D80002460B4616A1D1E9000105F031F805F038
:10C2E8007DFC4FF6E0730093054600230520DC2112
:10C2F8003246FFF7F9FC144BDB6853B11B4B188827
:10C308001B4B4FF4784719880097A2B2ABB2F9F7E4
:10C3180039FB164B1C60164B4FF6E0701D60F9F7A1
:10C32800A5FBC6E1AFF300800000000000E0634019
:10C338000000000000C05D4084E2050882E40508B2
:10C34800D82E0020B8280020200F002038280020F0
:10C358008FE40508E01B0020840F0020AEE40508E8
:10C36800B2E40508C82E00200000C842A03A002008
:10C37800403D0020A04B1868A04B9FEDA19A19687A
:10C388003246FFF777FBF4EE498AF1EE10FAC8BFA0
:10C39800F0EE498AF5EE408ADFED9A7AF1EE10FA6E
:10C3A80048BFF0EE678AF4EEC98AF1EE10FA044647
:10C3B8001ED8F4EEE78AF1EE10FA19DBFDEEE88AF2
:10C3C800002018EE902A4FF4FA71FFF777FB8E4B96
:10C3D800DB68054653B18D4B18888D4B4FF6FF77B8
:10C3E80019880097A2B2ABB2F9F7CCFA884B1D6056
:10C3F800B4EE498ADFED827AF1EE10FAC8BFB0EEEA
:10C40800678ADFED847AB4EE678AF1EE10FA48BFE6
:10C41800B0EE678AB4EEC98AF1EE10FA00F24981EB
:10C42800B4EEE78AF1EE10FAC0F24381BDEEC88A95
:10C43800794818EE102A4FF4FA71AEE06E4B18687E
:10C448006E4B32461968FFF715FBF5EEC0AAF1EE00
:10C4580010FA044627DDDDE9080159A3D3E90023D2
:10C4680005F094FBF8B158A3D3E90023DDE90801EE
:10C4780005F01AF90B4602466849002004F060FFEF
:10C4880005F0ACFB604BDB68054653B15F4B188881
:10C498005F4B4FF6FF7719880097A2B2ABB2F9F756
:10C4A80071FA5B4B1D60DDE9040149A3D3E9002360
:10C4B80005F08AFB002800F0FC80DDE9040140A3B8
:10C4C800D3E9002305F062FB002800F0F28042A3C4
:10C4D800D3E90023DDE9040105F0E6F802460B463E
:10C4E80000204F4904F02CFF05F078FB57E0424B41
:10C4F8001868424B32461968FFF7BCFA38A3D3E9EB
:10C5080000230446DDE90A0105F05EFB50B19DED0C
:10C518000A0B07F0D9FA002251EC100B414B05F039
:10C52800C3F8B1E0C825B2E02FA3D3E90023DDE9C1
:10C53800060105F0B9F82EA3D3E9002305F0DEF9CA
:10C5480005F094FB2C4B08EE100A18682B4B32466A
:10C558001968FFF78FFADFED347A4AEE677A2A4BCB
:10C56800FDEEE77ADB6817EE905A044625EAE57592
:10C5780053B1264B1888264B4FF6FF77198800973A
:10C58800A2B2ABB2F9F7FEF9BDEEC88A204B18EE9D
:10C59800102A1D606FF0B300B421FFF78FFA1A4B11
:10C5A800DB68054653B1194B1888204B4FF4FC67DC
:10C5B80019880097A2B2ABB2F9F7E4F91B4B75E002
:10C5C8009A9999999999B93F0000000000409F40B5
:10C5D8009A9999999999B9BF0000000000408F4035
:10C5E80089B5F81400E3693F000000000080764038
:10C5F8001F85EB51B81E1940B8280020D82E0020FE
:10C608000000FA4300000000200F0020A03A00209C
:10C61800403D00200000FAC30CFEFFFF0000694007
:10C6280000005940000054C00000484398380020DA
:10C638000000C8425FED027AB4EE679AF1EE10FA94
:10C64800C8BFB0EE679AB4EEE79AF1EE10FA30D8A8
:10C65800214B1868214B32461968FFF70BFA04463C
:10C6680019EE100A04F0CCFF41EC100B07F02CFA7D
:10C6780000221B4B51EC100B05F016F802460B4636
:10C688000020184904F05CFE05F0A8FA0546164B90
:10C69800DB6853B1154B1888154B4FF6FF7719888F
:10C6A8000097A2B2ABB2F9F76DF9114B1D600F4BB1
:10C6B8001C60104B1B78022B09D043B14FF6FF7357
:10C6C80000930520DC2132460023FFF70DFB41B023
:10C6D800BDEC068BBDE8F08FB8280020D82E0020CE
:10C6E8000000594000006940200F0020A03A0020B7
:10C6F800403D0020C82E002010B54FF4C770FAF74F
:10C7080089FFDB2805D14FF4C870FAF783FF84B29C
:10C7180019E041F2E104214644F20100FAF76CFF06
:10C7280044F20100FAF776FFA04214BF80244FF4C8
:10C73800007421B24FF4C870FAF75EFF4FF4C77067
:10C74800DB21FAF759FF204610BD024B00221A6080
:10C75800704700BFB438002070EEA10A88B030EEF0
:10C76800010A08B0704770EEE10A88B030EE410A5D
:10C7780008B07047F0EE407A20EEA10A60EE810A18
:10C7880047EEA10A88B017EE810A08B07047D0B505
:10C7980061EEA17A41EE017A2DED048B17EE900A35
:10C7A80088B0B0EE409AF0EE609AF0EE418AB0EEB2
:10C7B800618A04F025FF0022002306460F4605F093
:10C7C800DBF9E8B969EE887A49EE287A29EE088A11
:10C7D80017EE900A04F014FF32463B4605F08EF837
:10C7E80019EEA88A05F042FA044618EE100A04F079
:10C7F80007FF32463B4605F081F805F037FA01E0BD
:10C808000448044600EE900A00EE104A08B0BDEC59
:10C81800048BD0BD0050C347F0B58D4B2DED068B72
:10C8280093ED001AD3ED011A8FB0F0EE408AB0EE06
:10C83800608A8DED060ACDED070A30EE410A70EEEA
:10C84800E10A38EE811A78EE211A8DED0C1ACDED39
:10C858000D1A8DED0A0ACDED0B0AFFF798FF8DED45
:10C86800040ACDED050A04AA92E8030008AB83E8A0
:10C878000300DDED099A9DED08AA69EEA97A4AEE52
:10C888000A7A17EE900A04F0BBFE41EC100B07F091
:10C89800A1F951EC100B05F0E9F909EE100A19EEAF
:10C8A800900A04F0ADFE04461AEE100A0D4604F094
:10C8B800A7FE45EC104B41EC110B07F07DF851EC4D
:10C8C800100B05F0D3F968EE087A48EEA87AB1EEB5
:10C8D80048AAC8EEA79A5F4B5F4D5A691B8B6860E0
:10C8E800EA612B8404468AEE27AA85ED009A19EEA0
:10C8F800100AC5ED028A85ED038AC5ED049A85ED17
:10C9080005AA04F07DFE4CA3D3E9002305F05CF9E9
:10C91800DFED527A002818BFB0EE679AB7EE007ABA
:10C9280079EE077A37EE497A4D4BC7EE877A1B784E
:10C93800033BC5ED067A042B71D8DFE803F0032723
:10C9480038664F0018EE100A04F05AFE044618EE36
:10C95800900A0D4604F054FE06460F4647EC116B4C
:10C9680045EC104B07F028F835A3D3E9002351EC28
:10C97800100BCDE9004504F097FE3246CDE90201DF
:10C988003B463849384809F075FC48E019EE900AEA
:10C9980004F036FE04461AEE100A0D4604F030FE86
:10C9A8002246CDE900012B462F4830492AE019EEEE
:10C9B800100A04F025FE41EC100B07F085F8002260
:10C9C8002B4B51EC100B04F06FFE05F04FF904F0FF
:10C9D80017FE02460B46244826491EE019EE100AA7
:10C9E80004F00EFE064620460F4604F009FE16A384
:10C9F800D3E9002304F058FECDE900011A481E4986
:10CA080032463B4609F036FC09E017EE900A04F07E
:10CA1800F7FD02460B461448184909F02BFC124C46
:10CA280000230220CA212246F9F75AF9002323706D
:10CA38000FB0BDEC068BF0BDAE47E17A14AEEF3F08
:10CA48006666666666A64C40F6285C8FC2A54C40B2
:10CA5800DC3800206C3A0020543C0020A4707D3F54
:10CA6800C82E0020B6E4050878380020D0E4050870
:10CA7800000034C0E0E40508F2E405080EE5050806
:10CA880000B560EEA07A40EE007A2DED028B17EE2D
:10CA9800900A87B0B0EE408AF0EE608A8DED020A07
:10CAA800CDED030A04F0ACFD41EC100B07F092F851
:10CAB80051EC100B05F0DAF8DFED117A07EE100AE9
:10CAC80078EEA78A38EE078A68EEA87A48EE087AE0
:10CAD800C7EE277A17EE900A04F092FD41EC100B8E
:10CAE80007F078F851EC100B05F0C0F800EE900A4A
:10CAF80020EE880A60EEA80A07B0BDEC028B00BDE4
:10CB080000000000F0B52DED028BDFED3A1A3A4B2C
:10CB18008DB030EEA17AF0EE407AB7EE001A8DEDC6
:10CB2800020A83ED001A30EE010AC3ED011A31EE54
:10CB3800671A71EEE01ACDED030AF0EE470A8DEDA3
:10CB4800077A8DED081ACDED091A8DED060AFFF763
:10CB58001EFE8DED000ACDED010A9DE8030004AB31
:10CB680083E803009DED058ADDED048A68EE087A06
:10CB780048EEA87A17EE900A04F042FD41EC100B3B
:10CB880007F028F818EE100A57EC106B04F038FD7F
:10CB9800044618EE900A0D4604F032FD45EC104BA1
:10CBA80041EC110B06F008FF3946304655EC104BA6
:10CBB80005F05CF804F024FD41EC100B06F0FEFED5
:10CBC800002251EC100B0D4B04F06EFD05F04EF8F1
:10CBD80029460646204605F049F800EE900AF6EE8A
:10CBE800007A60EEA70A00EE106A0DB0BDEC028B69
:10CBF800F0BD00BF00000000AC3C00200000E03F9A
:10CC0800F0EE407A86B020EE200A67EE810A06B080
:10CC180070472DE9F04F2DED028B85B0FCF740F9F8
:10CC280010EE105AFCF742F9284610EE104A04F0AC
:10CC3800E7FC80462046894604F0E2FC41EC100BF4
:10CC480041EC180B06F05CFD57EC106BB0EE480A8F
:10CC5800F0EE680A06F054FE32463B464046494626
:10CC68005BEC10AB04F020FD05F000F89FED138A93
:10CC780007EE100ADFED127A57EE087A114C5B4680
:10CC8800C4ED007A52464046494604F00DFD04F0D2
:10CC9800EDFF07EE900A27EE888A04AB84ED018A3F
:10CCA80094E8030003E90300DDED030A9DED020AA1
:10CCB80005B0BDEC028BBDE8F08F00BF0000F0426C
:10CCC80000008C42383D002030B53F4B2DED088BDD
:10CCD800D3ED008AD3ED019A3C4BD3ED00AAD3EDF6
:10CCE80001BA3B4B93ED008A93ED019A394B93EDD2
:10CCF80000AA93ED01BA38EEEA0A79EEEB0A38EEAB
:10CD08004A1A79EE4B1A93B08DED0A0ACDED0B0A4B
:10CD18008DED0C1ACDED0D1AFFF72CFD8DED000AE7
:10CD2800CDED010A9DE803003AEE6A0A7BEE6B0A34
:10CD380004AB38EE681A79EE691A83E803008DEDC2
:10CD4800081ACDED091A8DED0E0ACDED0F0AFFF781
:10CD580011FD8DED000ACDED010A9DE8030006AB3B
:10CD680083E803009DED040ADDED050A9DED061A32
:10CD7800DDED071AFFF70BFD8DED000ACDED010A79
:10CD88009DE8030002AD85E80300134B9DED021AF0
:10CD980093ED000AD3ED010ADDED031AFFF7EAFC73
:10CDA8008DED000ACDED010A9DE8030012AB03E901
:10CDB80003006C46DDED110A85E803009DED100ABD
:10CDC80013B0BDEC088B30BD70380020C838002087
:10CDD8002C3D0020BC3C0020903A0020F7EE007A61
:10CDE80077EEC07A20EE022A20EE210A07EEA00A8A
:10CDF800F0EE420A47EE810A88B008B07047F8B5ED
:10CE0800C400A4B204F58066B0B20F46FAF746FC37
:10CE18001C4D0436B0B285ED000AFAF73FFC04F564
:10CE28008646B0B285ED010AFAF738FC164D04368D
:10CE380085ED000AB0B2FAF731FCA4F5FC4085EDA7
:10CE4800010A80B2FAF72AFC104DA4F5FA40FC3822
:10CE580085ED000A80B2FAF721FC012F85ED010A61
:10CE68000FD1A4F57C5080B2FAF718FC084DA4F550
:10CE78007A547C3C85ED000AA0B2FAF70FFC85EDE8
:10CE8800010AF8BD2C3D0020C8380020BC3C002019
:10CE9800703800202DE9F04F2DED048B8046C1B08D
:10CEA8004FF47670FAF7B6FB04464FF47570FAF74C
:10CEB800B1FB064640F2DE30FAF7D4FB189040F298
:10CEC800E230FAF7CFFB19904FF47F70FAF7A2FB24
:10CED800B8F1030F40F0E480189A199B0090019272
:10CEE80002931EA874493246234609F0C3F9C1B219
:10CEF8001EA8FDF7C7FDD9E001212046FFF77FFFF7
:10CF0800B8F1010F40F091806C4A6D4B10681E68B3
:10CF1800D2ED018A93ED019AF5EEC08A694BF1EEE4
:10CF280010FAD3ED019A54BF4FF0000C4FF0010CEA
:10CF3800B5EEC09A1F68644BBCF1000F0CBF4FF0F0
:10CF48002B094FF02D09F1EE10FA93ED018A54BF29
:10CF58004FF0000E4FF0010EF5EEC09ABEF1000F33
:10CF68000CBF2B252D25F1EE10FA54BF002101210D
:10CF7800B5EEC08A00290CBF4FF02B0A4FF02D0ADE
:10CF8800F1EE10FA54BF00220122D3F800B0002AB3
:10CF98000CBF2B232D23BCF1000F01D0F1EE688AC2
:10CFA800BEF1000F01D0B1EE499A09B1F1EE699ACC
:10CFB8000AB1B1EE488A179304F022FBCDE91A01B1
:10CFC80018EE900ACDF8009004F01AFBCDE90201A2
:10CFD800304604F015FBCDE9040119EE100A069558
:10CFE80004F00EFBCDE90801384604F009FBCDE951
:10CFF8000A0119EE900ACDF830A004F001FBCDE942
:10D008000E01584604F0FCFA179BCDE9100118EE02
:10D01800100A129304F0F4FADDE91A23CDE9140199
:10D028001EA82A4909F026F92FE0B8F1020F2DD1E0
:10D03800FFF74AFE8DED1C0ACDED1D0A1CAB93E8E7
:10D04800030040AB03E903009DED3F8AB5EEC08ABB
:10D05800F1EE10FA03D5B1EE488A2D2600E02B2612
:10D06800199A189B3E9802FB043504F0C9FACDE9D9
:10D07800000118EE100A029604F0C2FA2A46CDE919
:10D0880004011EA8124909F0F5F8C5B21EA82946E0
:10D09800FDF7F8FC01340120FEF704FAA4B200E021
:10D0A80000240C4A1388A342BFF626AF41B0BDEC5A
:10D0B800048BBDE8F08F00BF19E505082C3D002062
:10D0C800C8380020BC3C00207038002036E5050830
:10D0D80068E50508A43C0020F0B52DED028B044658
:10D0E8008DB0002800F0D480714B18890419A4B2BF
:10D0F80022B2002A05DB40F23F139A42C8BF1C4601
:10D1080000E00024F7F750FEA0B24EF29C71F7F74A
:10D118005DFE674B1C81674B186804F071FA5EA3CB
:10D12800D3E9002304F0C0FA04F0A0FD624B1860B4
:10D13800624B1B780A2B054624B23DD107EE104AF4
:10D14800F8EEC77A17EE900A04F05AFA5C4B0646D6
:10D1580018680F4604F042FA02460B4650A1D1E97E
:10D16800000104F0CBFB02460B463046394604F07A
:10D178009BFA064628460F4604F042FA02460B463A
:10D188003046394604F090FA00224E4B04F0B6FBC4
:10D1980004F06CFD04F034FA02460B4604A84A4930
:10D1A80009F068F80020F8F763FD0520D72104AAE4
:10D1B8000023F8F795FD6BE0444B1888604304F0B2
:10D1C8000DFA39A3D3E9002304F098FB04F04EFDCF
:10D1D8003F4B08EE100A1B68FCEEC87A07EE103ABF
:10D1E80017EE905AF8EEC77A3A4B68EE277A1B6822
:10D1F800FDEEE77AADB217EE906A28460121F618DF
:10D20800FFF7FDFDFFF760FD8DED020ACDED030A86
:10D2180002AC94E8030008AB83E80300681C80B202
:10D228000121FFF7ECFDFFF74FFD8DED020ACDED73
:10D23800030A94E803000CAB07EE105A03E9030055
:10D24800B8EEC70ADDED080A38EE400A9DED091A66
:10D25800DDED0A1A9DED0B2AFFF7C0FD8DED020AE0
:10D26800CDED030A94E8030006AB83E803004FF60C
:10D27800FF73009305200023DC213246FEF734FDBE
:10D28800154B9DED060A1878DDED070AFFF7C4FA7D
:10D298000DB0BDEC028BF0BD7B14AE47E17A843F44
:10D2A800000000A0D954BD410000000000F0734008
:10D2B800200F0020D0030020203D00203828002027
:10D2C800D82E00200000F43F7BE50508A43C002090
:10D2D800AC2E0020B8280020C82E00202DE9F843E5
:10D2E800461F8846B6B200250D4F12E008EB040130
:10D2F80089B23046F7F70CFD29F814000A200134EA
:10D30800FBF70CFB062CF1D116350136F22DB6B21F
:10D3180004D06FF0040407EB0509E7E7BDE8F883DC
:10D32800DC3C00202DE9F04F85B00B1A0193431E19
:10D338009BB20293431C441F00F1060901F1FF3A16
:10D3480001F1010B9BB20F461646A4B21FFA89F9E8
:10D358001FFA8AFA1FFA8BFB039380462046514630
:10D368003246F7F70DFD204639463246F7F708FDF5
:10D37800204659463246F7F703FD019B0298E51807
:10D38800ADB229463246F7F7FBFC404629463246FD
:10D39800F7F7F6FC0134039829463246F7F7F0FC14
:10D3A800A4B20A20FBF7BAFA4C45D7D105B0BDE8BC
:10D3B800F08F2DE9F843461F8846B6B200250E4F78
:10D3C80012E008EB040139F8142089B23046F7F767
:10D3D800D7FC01340A20FBF7A1FA062CF1D1163547
:10D3E8000136F22DB6B204D06FF0040407EB05093C
:10D3F800E7E7BDE8F88300BFDC3C00202DE9F043F7
:10D408002DED068B70EE007A8DB017EE900AB0EE17
:10D41800408A10EE904A20EE009A04F0F1F8064691
:10D4280020460F4604F0ECF8F7EE008A41EC100BAA
:10D4380041EC1A0B06F064F979EE287A55EC104B9A
:10D4480017EE900A04F0DCF82246804689462B46FF
:10D458003046394604F028F902460B46404649460C
:10D4680003F06EFF04F002FCB0EE4A0AF0EE6A0A1E
:10D4780009EE900A38EEC99ADFED377A89EE299AD3
:10D4880029EE279A06F03CFA304653EC102B394621
:10D4980004F00AF9044619EE900A0D4604F0B0F8B3
:10D4A80002460B462046294604F028FA00222B4B58
:10D4B80004F0FAF804F0DAFBB4EE688ADFED287AB3
:10D4C800284BF1EE10FA044619EE100A08BFB0EE28
:10D4D800678A1D6804F094F802460B4603A822499F
:10D4E80008F0C8FE204604F08BF802460B4606A852
:10D4F8001E4908F0BFFE78EE287A38EEC88A87EE13
:10D50800888A18EE100A04F07BF802460B4609A830
:10D51800174908F0AFFE0520014603AA0023F8F7D3
:10D52800DFFB0520142106AA0023F8F7D9FBC82041
:10D53800052109AA0023F8F7D3FB4FF6E0730093FF
:10D548000520DC212A460023FEF7CEFB0DB0BDECFA
:10D55800068BBDE8F08300BF000048420000494048
:10D56800A4707D3F883A002084E505088CE505080D
:10D5780094E505082DE9F04F494B2DED048B1D78F6
:10D58800022D85B080467BD1464E348A0121204643
:10D59800FFF735FCFFF798FB8DED000ACDED010A8A
:10D5A8009DE8030004AB03E9030028469DED020A49
:10D5B800DDED030AFFF730F93B4B1A683B4B1B685C
:10D5C80002FB04343A4B1C603A4BDFED3B7A93ED97
:10D5D800008A68EE277A5F6817EE900A04F010F860
:10D5E800824638468B4604F00BF841EC100B41ECB0
:10D5F800190B06F085F8504653EC102B594604F0E9
:10D6080053F823A3D3E9002303F09CFE04F00EFB98
:10D61800B0EE490AF0EE690A054684B206F070F9E0
:10D62800504653EC102B594604F03EF80B46024680
:10D6380019A1D1E9000103F083FE04F0F7FAB37CE5
:10D6480081461FFA80FA1BB9B08AF18AFFF7B1FE4A
:10D65800002320465146B374FFF740FE204651464A
:10D668001F22FFF75FFEB0EE480A00EE907AFFF740
:10D67800C5FE338AB5829844A6F81080A6F816909D
:10D6880005B0BDEC048BBDE8F08F00BFAFF30080A0
:10D698000000000000E063400000000000C05D40A2
:10D6A800C82E0020200F0020AC2E0020B828002013
:10D6B800883A0020543C00200000C842124B1B78D6
:10D6C800022B10B50CD1114B1B78022B08D1104C32
:10D6D8002078C0B140B2FFF74DFF0023237010BD82
:10D6E8000C4C237E23B99F20F7F738FB01232376C0
:10D6F800064B1B78022B06D1054C94F90000FFF766
:10D70800EBFC0023237010BDC82E0020AC3A00208B
:10D71800ED1B0020200F0020034B00201860034B56
:10D728001870FDF7E7BF00BFB4380020AC3A0020FE
:10D73800034B00201860034B02221A70FDF7DABF72
:10D74800B4380020AC3A002037B500242546A0B2F2
:10D7580028213223024601340095F8F713F9B4F56D
:10D76800A07FF4D13EBD2DE9F04F2DED088B0228A6
:10D7780097B080468DED070AB34B05D0032805D036
:10D78800012805D10C2202E0092200E00B221A70C0
:10D798001878F3F7A1F9042103914FF00009F3EE8B
:10D7A8000EAA9FEDAABADFEDAABA7DE1A94B1A68C5
:10D7B800A94B1B6802FB093307EE103A01211FFA37
:10D7C80089F0B8EEC78AFFF71AFBFFF77DFA8DEDEF
:10D7D800080ACDED090A08AD95E803000AAB83E80D
:10D7E80003009E4B1A6802EBC9030EAF19689C4BE5
:10D7F80019600399521812685A60FFF765FA8DED9F
:10D80800080ACDED090A95E803000CAB83E803008C
:10D81800DDED0A9A9DED0BAADDED0C8A9DED0D9AC2
:10D82800B0EE690AF0EE4A0AB0EE681AF0EE491A4C
:10D83800FEF7A0FF8DED080ACDED090A95E8030073
:10D84800B0EE691AF0EE4A1A87E80300B0EE680AEB
:10D85800F0EE490AFEF79BFF8DED080ACDED090AA7
:10D8680095E8030010AB83E803009DED0E0ADDED9B
:10D878000F0AFFF705F98DED080ACDED090A95E8BD
:10D88800030016AA02E903009DED100ADDED110A56
:10D89800149EFFF7F5F88DED080ACDED090A95E815
:10D8A800030087E80300DDED0F0AF5EEC00AF1EE8C
:10D8B80010FA48BFF1EE600A9DED0E0ACDED0F0A91
:10D8C800FFF720F98DED080ACDED090A08AA92E8BC
:10D8D800030012AB83E803000798129D03F090FE43
:10D8E8005D4B139FD3F800B05E4BBDEEC87AD3F8FA
:10D8F80000A0CDE9040117EE102A58465146FEF75C
:10D90800B9F807EE10AAF8EEC77A07EE10BAB4EE27
:10D91800E78AF8EEC77AF1EE10FAB4EEE78A8CBF20
:10D9280000220122504B0690F1EE10FAD4BF0022DB
:10D9380002F00102B8F1020FDA6012D0B8F1030F59
:10D948003ED0B8F1010F68D1304603F059FE36A336
:10D95800D3E9002303F0A8FE0022444B03F0F2FCB5
:10D968002AE0284603F04CFEDDE9042304460D4670
:10D978002FA1D1E9000103F0C1FF02460B46204662
:10D98800294603F091FE2CA3D3E9002303F08CFE73
:10D9980004F06CF907EE900AC7EEAA7A17EE900A1F
:10D9A80003F02EFE41EC100B06F08EF8002251EC2D
:10D9B800100B2F4B03F078FE04F010F904462CE00E
:10D9C80018EE100A03F01CFE044638460D4603F014
:10D9D80017FE17A3D3E9002303F066FEDDE904234D
:10D9E80003F08CFF04F042F903F00AFE14A3D3E914
:10D9F800002303F059FE02460B462046294603F051
:10DA08007DFF04F033F907EE900AB0EE6B7A07EE6B
:10DA18008B7AFDEEC77A17EE904A002C2ADBC72CCA
:10DA2800A8BFC72427E000BF8716D9CEF753F5BF94
:10DA38008FC2F5285CAF43400000000000907040A2
:10DA480000000080DBC48641C82E00200000C8C347
:10DA58000000C843AC2E0020B8280020A0380020C1
:10DA680070380020D82E0020200F002000006940C8
:10DA7800000049C00024114BDB685BB1104B1888CB
:10DA8800104B1988069B4FF6FF759AB2A3B2009502
:10DA9800F7F778FF0B4B039A1C600699084B08327E
:10DAA800196009F101090392074B1B884B45BFF622
:10DAB8007DAE17B0BDEC088BBDE8F08F200F0020BD
:10DAC800A03A0020403D0020A43C0020F0B51E4BA9
:10DAD8001E4F18781E4D1F4E85B0F2F7FDFF1E4BE6
:10DAE8000B221A70002423E01C4B1A68336802FBCF
:10DAF80004336B611A4B20461C840121FFF77FF920
:10DB0800FFF7E2F88DED000ACDED010A9DE803006C
:10DB180004AB03E903000C4B9DED020A1878DDED18
:10DB2800030AFEF779FE6869FEF788F90134A4B2A2
:10DB38003B88A342D8DA0B4B02221A700A4B002208
:10DB48001A7605B0F0BD00BFC82E0020A43C002006
:10DB58006C3A0020B0280020382800203428002003
:10DB6800543C0020AC3A0020200F002030B52D4D49
:10DB780095F9003085B0002B3CD0FDF7D1FB2A4A3F
:10DB88002A4B11682A4C526819605A60608B002130
:10DB9800FFF735F9FFF798F88DED000ACDED010A8A
:10DBA8009DE8030004AB03E90300224B9DED020A44
:10DBB800DDED030A1878FEF72FFE1F4B628B1868FD
:10DBC8001E4B1B6800FB0230FEF738F995F9002060
:10DBD800638BD3181A4A10681A4A12689BB200FB62
:10DBE80003206383FBF7D2FA174B1868FDF75AFC3A
:10DBF80000232B700E4C154B628B1B889A420ED15A
:10DC08004FF08040002102F0AAFD0E4B1868FBF788
:10DC1800BDFA0F4B02221A7000236383237605B0E6
:10DC280030BD00BFB43C00206C3A002070380020A2
:10DC3800200F0020C82E0020AC2E0020B82800207D
:10DC480034280020B028002064280020A43C0020AC
:10DC5800AC3A00207FB54FF08040012102F07FFDF3
:10DC6800FDF75EFB264A274B1168526819605A6017
:10DC7800254C264B22681B68254DD31A06EE903A90
:10DC8800B8EEE67AD5ED006AF8EEE67A0021C7EE3E
:10DC9800277AFCEEE77A17EE906AB0B2FFF7AFF892
:10DCA800FFF712F88DED000ACDED010A9DE803009B
:10DCB80004AB03E9030000209DED020ADDED030A31
:10DCC800FEF7AAFD134B1868134B1B6836B200FB0E
:10DCD8000630124EFEF7B2F81920FDF7E3FB307854
:10DCE80060B12A68236840B202FB0030FBF74EFAA5
:10DCF8000B4B1868FDF7D6FB002333707FBD00BFC0
:10DD08006C3A002070380020A8380020B028002085
:10DD180034280020AC2E0020B8280020B43C002075
:10DD28006428002010B500214FF0804002F017FD54
:10DD3800094B00241C702046F7F7C4FE074B1868EF
:10DD4800FBF724FA064B074801221A70064B1C7091
:10DD5800BDE81040F3F7CBBCB8380020B02800204D
:10DD6800C82E0020081A00203828002007EE100AC4
:10DD7800034BF8EE477A0022C3ED007A5A607047E9
:10DD8800DC38002007EE100A034BF8EE477A002231
:10DD9800C3ED007A5A607047903A00200F4B104943
:10DDA8001A68104B1B68D31A06EE903A0E4B1B6884
:10DDB800B8EEE67A06EE903AF8EEE67AC7EE277AFB
:10DDC800FCEEE77A17EE903A9AB20B80074B188868
:10DDD80090422CBF00200120704700BFD82E0020A1
:10DDE800A43C0020B8280020AC2E0020B428002035
:10DDF80013B502AB011D23ED010A054A89B213F8D8
:10DE0800014B1454013080B28842F8D11CBD00BFC8
:10DE1800EA3900202DE9F8431F4F0740002F044638
:10DE28000D4603DA013F67F00F070137BFB2DFF88D
:10DE380074804FEAC7091FFA89F9484698ED000A25
:10DE480009F10409FFF7D4FF1FFA89F098ED010AD8
:10DE5800FFF7CEFF114B10261B8894FBF6F6F60150
:10DE68009C42B6B20CD1701980B20D498022FAF7E3
:10DE7800F5FD00B1FEE721B24FF47F70F9F7BCFB66
:10DE88000F2F07D17519A8B205498022FAF7E6FDC8
:10DE980000B1FEE7BDE8F8830F000080A43C002035
:10DEA800EA3900206C3A00202DE9F043744B2DED3F
:10DEB800028B1888FF2898BF4FF4807093B0C00079
:10DEC80007F066FE6F4B0546186028B90520B42197
:10DED8006D4A2B46F7F704FF0024694F6B4E4FF04D
:10DEE80000086AE0FDF71CFA20464FF44141FFF7AD
:10DEF80091FF674B1A685B683260002173602046A7
:10DF0800FEF77DFFFEF7E0FE8DED020ACDED030A78
:10DF18000DF1080999E803000AAB83E803005D4B9B
:10DF28009DED0A1A93ED007AD3ED017ADDED0B1A17
:10DF380031EE470A71EEE70A31EE071A71EEA71AB9
:10DF48008DED0E0ACDED0F0A8DED101ACDED111ADB
:10DF5800FEF71DFC8DED020ACDED030A99E80300DA
:10DF68000CAB83E80300FF2C4FEAC4032B4404D90D
:10DF7800C3F80080C3F8048003E00C9A1A600D9A75
:10DF88005A603B8840F23F10604390FBF3F080B248
:10DF98004FF4FC630246282100933223F7F7F2FC82
:10DFA8003D4B18683D4B1B68C018FBF7EFF83C4B1E
:10DFB8001868FDF777FA0134A4B23B88A34291DAD6
:10DFC800012213464FF4807105A804F08BFE354EEC
:10DFD800DFF8F880294605A805F066F908233370AC
:10DFE800314B01241C700020F7F73AF82F48F3F75B
:10DFF8007EFB3078F2F770FD2D4B9FED2E8ADFED1A
:10E008002E8A1C700024D5ED007AB0EE687A07EEEF
:10E01800C87A2046FCEEC77A17EE906A03F0DEFA5B
:10E02800264B002203F040FB03F000FEB6B2A3B279
:10E03800C72E28BFC72687B253B1214BB8F80000B6
:10E0480019884FF6FF7300933A463346F7F79AFC60
:10E058001B4BC8F8007001340835B4F5807F1E608A
:10E06800D1D1184B1868FBF791F8114B02221A709E
:10E07800154B00221A7613B0BDEC028BBDE8F08375
:10E08800A43C0020A03800209CDD05087038002042
:10E098006C3A0020DC380020A83800203428002002
:10E0A80064280020C82E0020E10E002064190020FA
:10E0B800AC3A0020000016430000C8420000F43FBC
:10E0C800403D0020B0280020200F0020A03A00206A
:10E0D800F0B5294B294F2A4D2A4E012285B01A70D6
:10E0E80000243AE0284B1A68336802FB04336B615A
:10E0F800264B1C84FDF714F920464FF44141FFF7E5
:10E1080089FE234B2A681A606A6820465A600021F3
:10E11800FEF775FEFEF7D8FD8DED000ACDED010A7C
:10E128009DE8030004AB03E903001A4B9DED020AC6
:10E138001878DDED030AFEF76FFB6869FDF77EFED0
:10E14800154B1868154B1B68C018FBF71FF8144BC4
:10E158001868FDF7A7F90134A4B23B88A342C1DAD5
:10E16800104B1868FBF712F8034B02221A700E4B7B
:10E1780000221A7605B0F0BDAC3A0020A43C00207D
:10E188006C3A0020B8280020AC2E0020543C002017
:10E1980070380020C82E0020A8380020342800201D
:10E1A80064280020B0280020200F002038B5FDF793
:10E1B800FDFC124B124D9F221A81124B0124187834
:10E1C8002C70F2F789FC104B00221A600F4B1B7859
:10E1D800072B04D00B2B0DD0062B0ED102E0BDE887
:10E1E800384075E74FF0804021462C70BDE8384034
:10E1F80002F0B5BABDE8384068E438BD200F002009
:10E20800AC3A0020C82E0020B4380020382800205E
:10E218002DE9F743002581462C46154E154FDFF8AA
:10E228005C801FE0FDF77CF849462046FFF7F2FDC9
:10E23800D8F800303868C018FAF7A8FF0E4B1868ED
:10E24800FDF730F9308895FBF0F080B24FF4FC63AD
:10E258000093282102463223F7F794FB05F59E75B3
:10E26800013403353388A342DCDABDE8FE8300BFFE
:10E27800A43C0020A838002064280020342800206E
:10E2880010B5104C4FF47570B4F90010F9F7B4F9E3
:10E298000D4B4FF47670B3F90010F9F7ADF940F271
:10E2A800D230F9F7B7F9B02804D040F2D230B02113
:10E2B800F9F7A2F92088FFF759FD034B1888BDE844
:10E2C80010405FE5780200207402002000210A2235
:10E2D80008B509F01FF9D0F1010038BF002008BDCA
:10E2E80073B5041D0E46A4B20C2200234FF6E07548
:10E2F800204601360095F7F7E9FB00230C22B1B25E
:10E3080020460095F7F7E2FB0D4B1B78012B16D141
:10E318000C4E0D4D308829880024043080B20C2220
:10E3280023460094F7F7D2FB3088298800940430FC
:10E33800013180B289B20C222346F7F7C7FB7CBDB6
:10E3480094380020DA3800208C3A002008B54FF6BF
:10E35800FF70F7F78BFB0020F7F78AFC2148FFF7DF
:10E36800B5FF20B11F482049012207F083FF4B2049
:10E3780023211C4A0023F7F7B3FC1C48FFF7A6FF2C
:10E3880020B11A481849012207F074FF4B20462192
:10E39800164A0023F7F7A4FC1548FFF797FF20B1AA
:10E3A80013481149012207F065FF4B206921104AE3
:10E3B8000023F7F795FC0F48FFF788FF20B10D48B9
:10E3C8000949012207F056FF4B208C210023094AF6
:10E3D800F7F786FC084B1888084B1988BDE80840F1
:10E3E8007EE700BF7C28002046D90508A428002025
:10E3F800BA2E002068280020B63C0020843C00206B
:10E4080070B5044600200D461646F7F731FC00208B
:10E41800F7F742FB4FF4FC60F7F728FB2046294644
:10E4280056BB1E4A3346F7F75BFC1D48FFF74EFF05
:10E4380020B11B481B49012207F01CFF04F170069C
:10E44800B6B230462946164A0023F7F749FC164863
:10E45800FFF73CFF20B114481249012207F00AFFD8
:10E468003235ADB220462946104A0023F7F738FC6A
:10E47800304629460C4A07E00D4A0023F7F730FCDE
:10E4880032350B4AA9B220460023F7F729FC094B7D
:10E498001888094B1988BDE8704021E7A0E50508F0
:10E4A800243D002044DD0508983C0020A8E5050827
:10E4B800E7DD0508B63C0020843C002030B5144D4B
:10E4C8009DF80C402C70134D2880134D02FB04005E
:10E4D8002980124D80B22880114D2980114D2A8043
:10E4E800114A1380114B1880114B1980114B124996
:10E4F800E2B21A7000230B7010490A709DF81020C0
:10E508000134013254430E4A14700E4A137030BD60
:10E518003C3E00201C3D00206A3A0020B63C00200A
:10E52800843C0020E8390020483D0020DA380020EB
:10E538008C3A0020863C0020B9380020B83C0020E6
:10E54800953800209438002038B5054600200C4640
:10E55800F7F78EFB0020F7F79FFA4FF4FC60F7F708
:10E5680085FA0B48FFF7B2FE28B1094809490A4B5A
:10E57800002207F07FFE284621460023044AF7F7C9
:10E58800AFFB064B1888064B1988BDE83840A7E64C
:10E59800D0380020A3E205080000F03FB63C002078
:10E5A800843C002038B5054600200C46F7F760FB90
:10E5B8000020F7F771FA4FF4FC60F7F757FA0B48A9
:10E5C800FFF784FE28B1094809490A4B002207F0E1
:10E5D80051FE284621460023044AF7F781FB064BE3
:10E5E8001888064B1988BDE8384079E6AC38002011
:10E5F800A3E205080000F03FB63C0020843C002060
:10E6080038B5C501ADB20024601980B2F9F7CEFF64
:10E618000134C0B2FCF726FAA4B24FF47A70FAF7C4
:10E628007DF9802CF0D138BD73B5104D00240E2033
:10E63800FCF718FA002609E00DF10700FCF723FAA9
:10E6480020B19DF80730AB550136F6B23306F3D545
:10E65800E00180B205498022FAF700FA00B1FEE72E
:10E668000134A4B2B4F5007FE1D17CBDEA390020C1
:10E6780007EE100AF8EE477A7FB517EE900A02F017
:10E68800BFFF02460B4601A8054907F0F3FD0A2023
:10E69800962101AA0023F7F723FB07B000BD00BFAE
:10E6A800B0E50508AFF3008070B5302000210822DE
:10E6B8002A4E2B4CF9F738FE0023337020E0172B35
:10E6C80004D1302000210922F9F72EFE00232370FF
:10E6D800244D0EE0327803214A43D118AA18D318E2
:10E6E800695C93F84B203020F9F71EFE237801333C
:10E6F80023702378194A022BECD91378013313704D
:10E708003378164D182BDAD900232B70144C20E0DF
:10E71800152B04D1302000210A22F9F705FE002329
:10E728002370104E0EE02B78032101FB03639A1827
:10E73800302092F8961092F84B20F9F7F5FD2378DF
:10E74800013323702278054B022AECD91A7801325A
:10E758001A702B78182BDBD970BD00BFE41B002082
:10E768003D3E0020D80300200EB403B070470A28AD
:10E7780010B5044602D10D20FFF7F9FF064A1368C9
:10E788001BB103F8014B136010BD044B1B680BB1A0
:10E798002046984710BD00BF400F0020403E002093
:10E7A80010B5044601E0FFF7E2FF14F8010B00285A
:10E7B800F9D110BD2DE9F04F044685B00D464FF054
:10E7C8000A0A00E035462078002800F0C480252891
:10E7D80001D0013467E06078302803D1A0780123A4
:10E7E800033407E02D2802D00234002302E0A07889
:10E7F800022303344FF0000805E00AFB080814F868
:10E80800010BA8F13008A0F13002D2B2092AF4D9DC
:10E818006C2801D04C2803D114F8010B43F00403F1
:10E82800002800F09880602886BFA0F12002D2B2AC
:10E8380002464F2A3DD006D8432A2DD0442A09D073
:10E84800422A30D133E0552A04D0582A29D0532AF5
:10E8580029D101E00A272DE02E1D2F68002500E0B0
:10E8680001357A5D002AFBD104E02020FFF77FFF05
:10E878004D4601E0980704D4454505F10109F4D354
:10E888004D463846FFF78CFF03E02020FFF76FFF67
:10E8980001354545F9D395E728782E1DFFF767FF21
:10E8A80090E7102706E0FFF762FF2E468AE7022767
:10E8B80000E008272E1D442A296804D1002902DA1D
:10E8C800494243F00803002200E02A46B1FBF7FE64
:10E8D80007FB1E11CDB2092D714607D9782814BF40
:10E8E8004FF0070C4FF0270C6544EDB230350DF8AA
:10E8F8000250551CBEF1000F02D0102DE5D10F2299
:10E90800190705D504A94D192D2105F8101C951CCA
:10E9180013F0010F0CBF4FF0200B4FF0300B9B078B
:10E928002F4604D508E05846FFF721FF4F464745D4
:10E9380007F10109F7D34F46013D1DF80500FFF720
:10E9480016FF002DF8D103E02020FFF710FF013754
:10E958004745F9D336E705B0BDE8F08F70B5064DE9
:10E968000C462E68286001E0FFF701FF14F8010B40
:10E978000028F9D12E6070BD403E00200FB407B5C5
:10E9880004A951F8040B0191FFF714FFBDE80E40EC
:10E9980004B070470EB417B505A9084C51F8043BEC
:10E9A800206018460191FFF705FF226800231370C5
:10E9B8002360BDE81E4003B0704700BF400F002031
:10E9C8000EB433B505A9074C51F8043B25682060FF
:10E9D80018460191FFF7EEFE2560BDE83C4003B004
:10E9E800704700BF403E002070B51E4604461C48D4
:10E9F8001546FFF7C3FF022E1FD0042E25D0012E87
:10EA08002AD105E0A15D1748FFF7B8FF013600E0FD
:10EA18000026AE42F6DB2020FFF7A9FE002609E01B
:10EA2800A05DA0F12003DBB25E2B88BF2E20FFF78C
:10EA38009EFE0136AE42F3DB0EE034F8021B0A48B4
:10EA4800FFF79CFF013DF8D106E054F8041B074886
:10EA5800FFF794FF013DF8D10A20BDE8704086E633
:10EA6800B7E50508BEE50508C4E50508CAE50508D3
:10EA780008B501214FF4807001F07CFA4FF48070E2
:10EA88000021BDE8084001F075BA43680A6823F020
:10EA9800407323F4807313430A7943EA02234360E3
:10EAA800CA680B6930B51A4384688D68084B2A43D5
:10EAB800234013434A7943EA420383600B7DC26AC9
:10EAC800013B22F47002DBB242EA0353C36230BD59
:10EAD800FDF7FFC000230360037143718360C360C7
:10EAE8000361012303757047074A084B516810B545
:10EAF8000B4090E8120021438468C0682143014319
:10EB08000B43536010BD00BF00230140E030FCFF01
:10EB18000023036043608360C3607047836811B15A
:10EB280043F0010301E023F0010383607047436869
:10EB380023F4400323F400730B434360704741629E
:10EB480082627047436823F01F030B43436070479A
:10EB5800044B5A6810B142F4000201E022F40002AA
:10EB68005A60704700230140044B5A6810B142F4C0
:10EB7800800201E022F480025A60704700230140BD
:10EB8800092970B50CB20CD904EB44041E3CC668C4
:10EB98000725A54026EA0505A34045EA0304C46005
:10EBA8000AE0066904EB44040725A54026EA0505A2
:10EBB80013FA04F42C430461062A0CD80523013AFD
:10EBC8005A43446B1F23934024EA0303914043EACA
:10EBD8000102426370BD0C2A12B20CD802EB820209
:10EBE800233A046B1F23934024EA0303914043EA2A
:10EBF8000102026370BD02EB8202413AC46A1F231C
:10EC0800934024EA0303914043EA0102C26270BDC3
:10EC1800836843F08043836070478068C0F3805006
:10EC28007047836811B143F4806301E023F4806383
:10EC380083607047836811B143F0020301E023F059
:10EC48000203836070474368013923F4604343EA51
:10EC5800413343607047436811B143F4006301E0F6
:10EC680023F4006343607047C06C80B27047014B67
:10EC78001868704708230140836811B143F4807312
:10EC880001E023F4807383607047836811B143F413
:10EC9800007301E023F4007383607047044B5A68E3
:10ECA80010B142F4005201E022F400525A60704759
:10ECB80000230140092970B50CB20CD904EB4404B7
:10ECC8001E3CC6680725A54026EA0505A34045EA77
:10ECD8000304C4600AE0066904EB44040725A54060
:10ECE80026EA050513FA04F42C430461836BC3F385
:10ECF8000154121B0232D2B202EB82021F2494404A
:10ED080023EA040391400B43836370BD836B01398D
:10ED180023F4401343EA01538363704782B000230E
:10ED280001930190019BCB180193019B1A6002B0DB
:10ED38007047836823F470230B43836070478368AC
:10ED480023F440130B4383607047836843F48003C4
:10ED5800836070478068C0F380507047436811B182
:10ED680043F4806301E023F48063436070474368A1
:10ED780011B143F4805301E023F48053436070479A
:10ED880082B0002301930190019B28335B18019303
:10ED9800019B186880B202B070470123C9B213FA08
:10EDA80001F143680AB1194301E023EA0101416016
:10EDB8007047036819420CBF002001207047C943FF
:10EDC800016070474368006810EA112007D00122EB
:10EDD800C9B212FA01F119420CBF00200120704794
:10EDE8006FEA112101607047036823F00103036093
:10EDF8000023036043608360C36003612123436190
:10EE08002C4B98421CD02C4B984220D02B4B98422C
:10EE180025D02B4B98422AD02A4B98422FD02A4BE8
:10EE2800984233D0294B984237D0294B984204D185
:10EE38004FF03D5243F8AC2C7047264B984203D113
:10EE48003D2243F8082C7047234B984204D14FF4D5
:10EE5800746243F8202C7047204B984204D14FF439
:10EE6800741243F8382C70471D4B984204D14FF068
:10EE7800746243F8502C70471A4B984203D11A4ACF
:10EE880043F8642C7047194B984203D1184A43F849
:10EE98007C2C7047174B984203D1174A43F8942C9F
:10EEA8007047164B984204BF4FF03D5243F8AC2CC4
:10EEB800704700BF10600240286002404060024076
:10EEC800586002407060024088600240A0600240C2
:10EED800B860024010640240286402404064024066
:10EEE80058640240706402403D000020886402407B
:10EEF800400F0020A064024000003D20B86402409A
:10EF08000268134B10B51340CC680A6822434C6959
:10EF180022438C692243CC6922430C6A22434C6AFF
:10EF280022438C6A22434C6B22438C6B224313434B
:10EF3800036042690C6BCB6A22F007022343134338
:10EF480043610B6943604B6883608B68C36010BD85
:10EF58003F801CF00023036043608360C36003614B
:10EF680043618361C361036243628362C362036373
:10EF7800436383637047036811B143F0010301E001
:10EF880023F0010303607047036811B143F40043A1
:10EF980001E023F4004303607047036811B143F0B4
:10EFA800200301E023F020030360704741607047AD
:10EFB800406880B27047036812B143F4002301E04F
:10EFC80023F40023036001617047036811B143F41F
:10EFD800802301E023F48023036070470AB10161B4
:10EFE8007047C16070470068C0F3C0407047006850
:10EFF80000F001007047406900F0380070470A4A85
:10F008000A4B10B50A4CA04288BF13468A004CBF71
:10F018005B681B6821F0F02121F0821119420CBFB6
:10F028000020012010BD00BF0064024000600240C3
:10F038000F64024010B5084B084A094CA04288BF2B
:10F04800134611F0005F21F0F02121F0821114BF66
:10F05800D960996010BD00BF0060024000640240A2
:10F068000F6402400B0607D5436912B143F08003D1
:10F0780001E023F080034361802909D001F01E01DB
:10F08800036812B119430160704723EA0101016066
:10F098007047124B124A10B5124CA0428CBF14464E
:10F0A8001C4621F0F02323F0C3132BB1026802F0B1
:10F0B8001E0202EAD12202E0426902F080028800C0
:10F0C8004CBF6368236821F0F02121F082101840BA
:10F0D80002D0101C18BF012010BD00BF0060024004
:10F0E800006402400F64024010B5084B084A094CFE
:10F0F800A04288BF134611F0005F21F0F02121F0F3
:10F10800821114BFD960996010BD00BF0060024031
:10F11800006402400F640240044B00221A605A60E7
:10F128009A60DA60024A5A61704700BF003C0140A9
:10F13800FFFF7F00837910B5002B29D01A4B016897
:10F148001C68CA4314401C605C6822405A600279FB
:10F1580002F1804202F59E32146821431160026870
:10F168009C68D1430C409C60DC682140D96041799F
:10F17800102906D1996811439960D9680A43DA6061
:10F1880010BD01F1804303F59E3319680A4308E076
:10F198000379016803F1804303F59E331A6822EA74
:10F1A80001021A6010BD00BF003C014000230C2280
:10F1B80003600371427183717047024B1A690243FD
:10F1C8001A617047003C0140034B5B6918420CBF51
:10F1D80000200120704700BF003C0140014B5861EE
:10F1E800704700BF003C0140054B1A685B6903404B
:10F1F80004D010420CBF0020012070471846704709
:10F20800003C0140014B5861704700BF003C014081
:10F218004FF0204318B943F2DB021A6003E043F2CF
:10F22800D20243F820204FF02042411C6FF0704377
:10F2380042F8213002F5827242F82030704770B5EA
:10F2480084684568C368C16A026825431D43036929
:10F258001D4343691D4383691D43C3691D43036AF5
:10F268001D43436A1D43836A1D43036B0D431D43BE
:10F278004FF02043082C43F8225005D153F8224080
:10F2880044F0400443F82240436B9E691D683543AF
:10F298005E6845EA06159E6845EA0625DE6845EA81
:10F2A80006451E695B6945EA0655541C45EA03652F
:10F2B8004FF02043B1F5804F43F8245010D1836BB1
:10F2C800986919680143586841EA0011986841EA49
:10F2D800002118695B6941EA005141EA036101E0D4
:10F2E8006FF07041014B43F8221070BD040100A07B
:10F2F800022242604FF480524262416B4FF4005246
:10F3080010B5826200230F22FF2403608360C3606C
:10F31800036143618361C3610362C36203630A607B
:10F328004A608C60CA600A614A618B61816B0A60BD
:10F338004A608C60CA600A614A618B6110BD4FF0F7
:10F34800204321B153F8202042F0010203E053F892
:10F358002010024A0A4043F820207047FEFF0F00A1
:10F3680010280CBF064B074B4FF040024FF0180116
:10F3780019605A604FF0FC329A60DA60704700BF3B
:10F38800600000A0800000A030B5836844681C437A
:10F39800C36844F008041C4303691C43436944EAF6
:10F3A8004324836944EA4334C36999685A68090461
:10F3B80041EA02211A68DB68114341EA0361036AE2
:10F3C8009A685D68120442EA05221D68DB682A43D0
:10F3D80042EA03620368102B0CBF034B034B1C600B
:10F3E8009960DA6030BD00BF600000A0800000A016
:10F3F80010230360C269002343608360C360036114
:10F4080043618361FC23136053609360D360026A95
:10F41800136053609360D360704741B110280CBFEC
:10F42800074B084B1A6842F004021A60704710280C
:10F438000CBF034A034A044B11680B401360704722
:10F44800600000A0800000A0FBFF0F0041B1102861
:10F458000CBF084B084B1A6842F040021A6070470C
:10F4680010280CBF034A044A044B11680B40136070
:10F47800704700BF600000A0800000A0BFFF0F0021
:10F48800102802D1024B58697047024B58697047DF
:10F49800600000A0800000A0054B18221A6000221E
:10F4A8005A604FF0FC329A60DA601A61704700BF08
:10F4B800A00000A00268436842F0100242EA43221A
:10F4C800836842EA4332144B10B51A60C2689168E7
:10F4D8005468090441EA04211468D268214341EAC6
:10F4E80002629A60026991685468090441EA042139
:10F4F8001468D268214341EA0262DA60426991687D
:10F508005068090441EA00211068D268014341EAC1
:10F5180002621A6110BD00BFA00000A0C2680023EB
:10F52800036043608360FC23136053609360D3607F
:10F538000269136053609360D3604269136053603B
:10F548009360D3607047054B18B11A6842F0040203
:10F5580002E01968024A0A401A607047A00000A039
:10F56800FBFF0F0062B1102801D10E4B03E0B0F58C
:10F57800807F03D10C4B5A68114311E00B4BFAE71B
:10F58800102804D1074B5A6822EA010108E0B0F5B7
:10F59800807F0CBF044B054B5A686FEA010111408C
:10F5A80059607047600000A0800000A0A00000A083
:10F5B800102801D1064B04E0B0F5807F0CBF054B45
:10F5C800054B5B680B420CBF00200120704700BF51
:10F5D800600000A0800000A0A00000A0102804D1B6
:10F5E800074B5A6822EA010108E0B0F5807F0CBF9A
:10F5F800044B054B5A686FEA010111405960704786
:10F60800600000A0800000A0A00000A0102801D188
:10F61800084B04E0B0F5807F0CBF074B074B5B68D5
:10F6280013EA010004D013EAD1010CBF0020012025
:10F63800704700BF600000A0800000A0A00000A0EC
:10F64800102804D1084B5A6822EAD10109E0B0F524
:10F65800807F0CBF054B064B5A684FEAD10122EA5E
:10F6680001015960704700BF600000A0800000A041
:10F67800A00000A008B52C4B984205D101200146F6
:10F6880000F048FC012048E0284B984205D10220B0
:10F69800012100F03FFC02203FE0254B984205D1B4
:10F6A8000420012100F036FC042036E0214B98426A
:10F6B80005D10820012100F02DFC08202DE01E4B6B
:10F6C800984205D11020012100F024FC102024E0EC
:10F6D8001A4B984205D12020012100F01BFC202064
:10F6E8001BE0174B984205D14020012100F012FC85
:10F6F800402012E0134B984205D18020012100F0F0
:10F7080009FC802009E0104B98420BD14FF480701F
:10F71800012100F0FFFB4FF480700021BDE8084094
:10F7280000F0F8BB08BD00BF000002400004024022
:10F7380000080240000C0240001002400014024081
:10F7480000180240001C0240002002402DE9F0474A
:10F758000023D1F800801A464FF0010C03270CFA59
:10F7680002F404EA0805A5422ED1066817FA03F444
:10F77800E443264006600E79D0F8009006FA03FAB2
:10F78800013E4AEA0909012EC0F8009014D886689B
:10F7980091F8059026408660866809FA03F949EAD7
:10F7A80006068660466826EA050545608D7946683E
:10F7B8009540ADB235434560C5682C40C460CC79EE
:10F7C800C5689C402C43C46001320233102AC6D15C
:10F7D800BDE8F0874FF6FF730360002303714371A0
:10F7E8008371C371704782B04FF480330193019BDA
:10F7F8000B430193019BC361C161019BC361C36951
:10F808000193C369019302B07047036919420CBFA1
:10F81800002001207047006980B27047436919428F
:10F828000CBF002001207047406980B270470183F7
:10F838007047418370470AB101837047418370471D
:10F848004161704743694B404361704701F00703CA
:10F85800C908083130B59B0050F821500F249C404E
:10F8680025EA040440F8214050F8214012FA03F335
:10F878001C4340F8214030BD08B5134B984207D1CE
:10F888004FF40010012100F069FB4FF4001014E060
:10F898000E4B984207D14FF48000012100F05EFB27
:10F8A8004FF4800009E00A4B98420BD14FF4000056
:10F8B800012100F053FB4FF400000021BDE808408F
:10F8C80000F04CBB08BD00BF005400400058004089
:10F8D800005C00407FB50446868868460D4600F007
:10F8E8006DFA02992C482B6826F03F063604B1FBC6
:10F8F800F0F0360C80B20643A680228822F001027E
:10F908001204120C2280254A93420AD85B00B1FBEC
:10F91800F3F301309BB280B22084032B98BF0423F9
:10F9280021E0EE884BF6FF72964205D1032253433D
:10F93800B1FBF3F39BB206E019225343B1FBF3F397
:10F948009BB243F480431A054FF4967208BF43F004
:10F95800010350434FF47A7290FBF2F0013080B209
:10F9680043F400432084A38323886989AA889BB22F
:10F9780043F001032380238823F4816323F00203E7
:10F988001B040A431B0C13439BB223802A89AB89AF
:10F9980013439BB223817FBD40420F00A086010024
:10F9A80041F288330360002383804BF6FF720381A2
:10F9B80043814FF48043C28083817047038819B123
:10F9C8009BB243F0010303E023F001031B041B0C6B
:10F9D80003807047038819B19BB243F4807303E036
:10F9E80023F480731B041B0C03807047038819B130
:10F9F8009BB243F4007303E023F400731B041B0C55
:10FA08000380704712B141F0010101E001F0FE01ED
:10FA180001827047038819B19BB243F4806303E005
:10FA280023F480631B041B0C0380704783899BB2FB
:10FA380001F0FE0123F0FE030B43838170478389A5
:10FA480019B19BB243F0010303E023F001031B0447
:10FA58001B0C83817047038819B19BB243F04003A4
:10FA680003E023F040031B041B0C0380704703884A
:10FA780029B16FEA43436FEA53439BB201E05B0449
:10FA88005B0C03807047038819B99BB243F080036D
:10FA980003E023F080031B041B0C03807047B1F5BF
:10FAA800804F838B04D023F480431B041B0C02E09B
:10FAB8009BB243F4804383837047B1F5006F03889A
:10FAC80003D19BB243F4006303E023F400631B04F7
:10FAD8001B0C03807047B1F5005F038803D19BB20C
:10FAE80043F4005303E023F400531B041B0C03806E
:10FAF8007047038819B19BB243F0100303E023F069
:10FB080010031B041B0C0380704701827047008A96
:10FB1800C0B27047038819B19BB243F4805303E025
:10FB280023F480531B041B0C03807047B1F5006F4E
:10FB3800038803D19BB243F4006303E023F400631A
:10FB48001B041B0C03807047038819B19BB243F058
:10FB5800200303E023F020031B041B0C03807047E1
:10FB6800008BC0F307207047838819B19BB243F418
:10FB7800006303E023F400631B041B0C83807047BD
:10FB8800838819B19BB243F4805303E023F4805374
:10FB98001B041B0C8380704782B0002301930190E3
:10FBA800019BCB180193019B188880B202B0704763
:10FBB80083889BB20AB1194301E023EA01018180DD
:10FBC8007047838A008B9BB243EA0040084020F0CC
:10FBD8007F40431A584240EB03007047838A008BEA
:10FBE8009BB243EA004020F07F40704782B0002378
:10FBF800009301930B0F01900093009B21F07F412C
:10FC080013B1019B143302E0019B090C18330193D3
:10FC1800019B1B6819420CBF0020012002B07047ED
:10FC2800C94389B2818270478388808A80B208403C
:10FC38009BB206D001F0E06113EA11410CBF00202D
:10FC480001207047C94389B2818270470A4B1A68FC
:10FC580042F001021A6000229A60196821F084714A
:10FC680021F48031196005495960196821F480210F
:10FC78001960DA60704700BF003802401030002475
:10FC8800024B00221A701870704700BF02380240F9
:10FC9800034B1A6822F0F80242EAC0021A60704761
:10FCA80000380240014B1860704700BF000047420F
:10FCB800064B002201281A701A7002D0042804D1B9
:10FCC80001E01870704705221A70704770380240BA
:10FCD800014B1860704700BF800E4742014341EA5C
:10FCE800821200995B08013B42EA016141EA034143
:10FCF800014B5960704700BF00380240014B186043
:10FD0800704700BF600047428001034B40EA017121
:10FD1800C3F88410704700BF00380240014B1860D8
:10FD2800704700BF68004742014B1860704700BF2A
:10FD38004C004742034B9A6822F0EC6202430A43A4
:10FD48009A60704700380240034B9A6822F0784264
:10FD580002430A439A60704700380240034B9A688E
:10FD680022F0030202439A60704700BF0038024045
:10FD7800024B986800F00C00704700BF0038024042
:10FD8800034B9A6822F0F00202439A60704700BF62
:10FD980000380240034B9A6822F4E05202439A600A
:10FDA800704700BF00380240034B9A6822F4604253
:10FDB80042EAC0029A607047003802401E4B9A68B7
:10FDC80002F00C02042A10B503D0082A03D01B4BFA
:10FDD80018E01B4B16E059685A6811F4800F5968EF
:10FDE80014BF174B154B02F03F02B3FBF2F3124A54
:10FDF8005268C2F30142C1F3881101324B435200E9
:10FE0800B3FBF2F30C4903608B680E4A0468C3F332
:10FE18000313D35C34FA03F343608C68C4F382247D
:10FE2800145D33FA04F484608968C1F34231525C8A
:10FE3800D340C36010BD00BF003802400024F40066
:10FE480000127A00B904002000F44073B3F5407F33
:10FE5800084B08D1996820F0704221F4F81122F477
:10FE680040720A439A601A6F000542EA10501867F8
:10FE7800704700BF00380240014B1860704700BF50
:10FE88003C0E4742014B1860704700BF400E474286
:10FE9800014B1860704700BF5C014742044B1A6B66
:10FEA80009B1104301E022EA00001863704700BF5F
:10FEB80000380240044B5A6B09B1104301E022EAB2
:10FEC80000005863704700BF00380240044B9A6B2B
:10FED80009B1104301E022EA00009863704700BFAF
:10FEE80000380240044B1A6C09B1104301E022EAC1
:10FEF80000001864704700BF00380240044B5A6C79
:10FF080009B1104301E022EA00005864704700BFBD
:10FF180000380240044B1A6909B1104301E022EA93
:10FF280000001861704700BF00380240044B5A694E
:10FF380009B1104301E022EA00005861704700BF90
:10FF480000380240044B9A6909B1104301E022EAE3
:10FF580000009861704700BF00380240044B1A6ADD
:10FF680009B1104301E022EA00001862704700BF9F
:10FF780000380240044B5A6A09B1104301E022EAF2
:10FF880000005862704700BF00380240044B1A6DE9
:10FF980009B1104301E022EA00001865704700BF6C
:10FFA80000380240044B5A6D09B1104301E022EABF
:10FFB80000005865704700BF00380240044B9A6D36
:10FFC80009B1104301E022EA00009865704700BFBC
:10FFD80000380240044B1A6E09B1104301E022EACE
:10FFE80000001866704700BF00380240044B5A6E84
:08FFF80009B1104301E022EA07
:020000040801F1
:1000000000005866704700BF00380240044B1A7861
:1000100009B1104301E022EA00001870704700BFE8
:100020000D3802404309012B074A01D1136803E050
:10003000022B0CBF136F536F00F01F0033FA00F058
:1000400000F00100704700BF0038024007B50023F0
:1000500001933120FFF7E6FF019B01330193019BE0
:10006000B3F5A06F01D00028F3D03120FFF7DAFFFD
:10007000003018BF01200EBD024B5A6F42F0807253
:100080005A67704700380240034BDB6818420CBFC8
:1000900000200120704700BF00380240014B18705B
:1000A000704700BF0E38024008B5154B98420BD17F
:1000B00001214FF48050FFF761FF4FF48050002181
:1000C000BDE80840FFF75ABF0E4B984207D14FF4E6
:1000D00080400121FFF746FF4FF4804009E00A4BC2
:1000E00098420BD14FF400400121FFF73BFF4FF442
:1000F00000400021BDE80840FFF734BF08BD00BF45
:100100000030014000380040003C00400B8802886D
:1001100010B54C8823438C882343CC8823430C8917
:1001200023434C8923438C892343CC8902F44152D5
:10013000234313439BB20380838B23F400631B048C
:100140001B0C83830B8A038210BD838B23F47B6398
:1001500023F00F031B041B0C8383022303848B688F
:10016000F0B5858B022BADB238D0294A8E889468C1
:10017000002E14BF02260126240203D5946824F41D
:1001800000049460D2F88440D2F884705268DFF89A
:1001900084C002F03F02BCFBF2F2C4F38814544363
:1001A000C7F30272B4FBF2F4CA88B2F5007F4FF0D5
:1001B0000A0201D1240A02E07601B4FBF6F462439C
:1001C000B2FBF3F305330A229BB2B3FBF2F303F065
:1001D00001021202C3F34F0392B200E000229C1E00
:1001E000A4B2FE2C28BF0022CC8828BF02231343D0
:1001F00023439BB203840B884A882B4343F4006358
:1002000013438A8813438A8913439BB28383F0BDC7
:100210000038024000127A0000230380438083806C
:10022000C380038143818381C38107230382704795
:1002300000230222038043808380C3808260838105
:100240007047038819B19BB243F0400303E023F0E9
:1002500040031B041B0C03807047838B19B19BB2B6
:1002600043F4806303E023F480631B041B0C83834B
:100270007047038823F400631B041B0C038003886E
:100280009BB20B4303807047B1F5804F038803D1C5
:100290009BB243F4804303E023F480431B041B0C14
:1002A000038070474FF6FF639942038803D09BB2E7
:1002B00043F4807303E023F480731B041B0C03805E
:1002C0007047838819B19BB243F0040303E023F025
:1002D00004031B041B0C83807047838819B19BB2F5
:1002E00043F0100303E023F010031B041B0C838076
:1002F0007047838B23F47B6323F00F031B041B0CD9
:100300008383022303840B88828BB3F5007F10B5AF
:1003100092B205D0002B0CBF4FF48073002301E094
:100320004FF480734C8822438C88898942F40062A0
:1003300022430A4392B21343838310BD808980B263
:10034000704781817047038819B19BB243F4005311
:1003500003E023F400531B041B0C03807047038845
:100360009BB243F4805303807047012902D0008B75
:1003700080B27047808A80B27047008A80B270472E
:1003800083889BB20AB1194301E023EA010181800D
:100390007047090901238B409BB21AB1828892B23F
:1003A000134303E0828892B222EA030383807047FA
:1003B000038919420CBF002001207047C94389B24C
:1003C0000181704710B584880089012301F00F0274
:1003D00080B213FA02F21040A4B205D009098B4092
:1003E0001C420CBF0020012010BD01F00F010123B1
:1003F0008B40DB439BB20381704700BF08B50121EE
:100400004FF48040FFF7BAFD4FF480400021BDE873
:100410000840FFF7B3BD014B18607047003801403A
:1004200001F0030289080A4B023130B5920053F8FB
:1004300021500F24944025EA040443F8214053F846
:10044000214010FA02F2144343F8214030BD00BFAE
:1004500000380140014B1860704700BFDC002742A4
:10046000014B1860704700BF00042742024B186A16
:10047000C0F30020704700BF0038014030B5048C45
:1004800024F001042404240C0484058B048CADB2F4
:10049000A4B225F0F305154324F00A0445EA031538
:1004A00044F00104ADB20C430583048430BD30B583
:1004B000048C24F010042404240C0484048B058C84
:1004C00024F44074ADB22405240D25F0A00544EABF
:1004D000022445F0100544EA033445EA0115A4B2AC
:1004E000ADB20483058430BD08B5474B984205D1B1
:1004F00001200146FFF742FD01203DE0B0F1804FB1
:1005000005D101200146FFF72DFD012076E03F4B8C
:10051000984205D102200121FFF724FD02206DE061
:100520003B4B984205D104200121FFF71BFD04201D
:1005300064E0384B984205D108200121FFF712FDF5
:1005400008205BE0344B984205D110200121FFF7D1
:1005500009FD102052E0314B984205D120200121A5
:10056000FFF700FD202049E02D4B984209D10220E1
:100570000121FFF703FD02200021BDE80840FFF73D
:10058000FDBC284B984207D14FF480300121FFF782
:10059000F5FC4FF48030EFE7234B984207D14FF43E
:1005A00000300121FFF7EAFC4FF40030E4E71F4B75
:1005B000984207D14FF480200121FFF7DFFC4FF470
:1005C0008020D9E71A4B984205D140200121FFF73E
:1005D000C9FC402012E0174B984205D18020012130
:1005E000FFF7C0FC802009E0134B98420BD14FF479
:1005F00080700121FFF7B6FC4FF480700021BDE848
:100600000840FFF7AFBC08BD0000014000040040F7
:1006100000080040000C00400010004000140040A2
:1006200000040140004001400044014000480140F6
:1006300000180040001C0040002000401C4A0388B5
:1006400090429BB212D002F5806290420ED0B0F17F
:10065000804F0BD0A2F58032904207D002F5806225
:10066000904203D002F58062904203D14A8823F081
:10067000700313430F4A904208D002F58062904203
:1006800004D023F440730A899BB2134303804B6860
:10069000C3620B880385064B984203D003F5806341
:1006A000984201D18B7A038601238382704700BF71
:1006B00000000140001000404FF0FF334360002372
:1006C0000380038143808372704701858282704773
:1006D000038823F070031B041B0C0B43038070473B
:1006E00041627047C1627047406A7047008D80B2B6
:1006F0007047038819B19BB243F0020303E023F073
:1007000002031B041B0C03807047038819B19BB2C2
:1007100043F0040303E023F004031B041B0C0380D9
:100720007047038819B19BB243F0800303E023F0C4
:1007300080031B041B0C03807047038823F008030D
:100740001B041B0C038003889BB20B430380704780
:10075000038823F440731B041B0C038003889BB2A3
:100760000B4303807047038819B19BB243F0010328
:1007700003E023F001031B041B0C03807047038C70
:1007800023F001031B041B0C038470B5038C8488C5
:10079000028B0D884E8822F073021204120C2A4339
:1007A0008D8923F002031B0435431B0CADB22B4390
:1007B0000E4DA842A4B203D005F58065A8420ED123
:1007C000CD894E8A23F008032B438D8823F0040340
:1007D0002B430D8A354324F44074ADB22C438480FE
:1007E00002838A684263038470BD00BF0000014039
:1007F000038C23F010031B041B0C0384038C8288DE
:1008000030B5048B0D8824F4E6442404240C23F032
:10081000200344EA05241B048D891B0C43EA0513BD
:100820004D8843EA0513134DA84292B2A4B29BB27D
:1008300003D005F58065A84215D1CD8923F080034A
:100840009BB243EA05134FF6BF751D408B8845EAFE
:1008500003130D8A22F4406242EA85024D8A42EA7D
:1008600085029BB292B282808A6804838263038489
:1008700030BD00BF00000140038C23F480731B04D3
:100880001B0C0384038C828830B5848B0D8824F084
:1008900073042404240C23F400731B042C438D895B
:1008A0001B0C43EA05234D8843EA0523124DA84259
:1008B00092B29BB203D005F58065A84215D1CD89CF
:1008C00023F400639BB243EA05234FF6FF351D4036
:1008D0008B8845EA03230D8A22F4405242EA05122E
:1008E0004D8A42EA05129BB292B282808A68848362
:1008F000C263038430BD00BF00000140038C23F4B9
:1009000080531B041B0C0384038C30B58488828BBA
:100910000D8822F4E6421204120C23F4005342EA3A
:1009200005221B048D891B0C43EA05334D8843EADD
:1009300005330B4DA842A4B292B29BB203D005F589
:100940008065A84205D10D8A24F4804444EA8514C8
:10095000A4B2848082838A680264038430BD00BFAD
:1009600000000140002303804380838083608381F3
:10097000C38103824382704730B5058C0124ADB238
:100980008C4025EA040400F11803048409B1082905
:1009900007D149084FF68F70CC582040C850C8582E
:1009A0000AE00439C1F34E0148F6FF70CC582040EC
:1009B000C8501202C85892B20243CA5030BD4163B7
:1009C000704781637047C163704701647047038B50
:1009D00023F070031B041B0C0B4303837047038B32
:1009E00023F4E0431B041B0C43EA01239BB2038363
:1009F0007047838B23F070031B041B0C0B43838312
:100A00007047838B23F4E0431B041B0C43EA012350
:100A10009BB283837047038B23F008031B041B0CDA
:100A20000B4303837047038B23F400631B041B0CED
:100A300043EA01239BB203837047838B23F00803AF
:100A40001B041B0C0B4383837047838B23F40063CD
:100A50001B041B0C43EA01239BB283837047038B67
:100A600023F004031B041B0C0B4303837047038B0D
:100A700023F480631B041B0C43EA01239BB2038312
:100A80007047838B23F004031B041B0C0B438383ED
:100A90007047838B23F480631B041B0C43EA012300
:100AA0009BB283837047038B23F080031B041B0CD2
:100AB0000B4303837047038B09025B0441EA5343F2
:100AC0009BB203837047838B23F080031B041B0CB2
:100AD0000B4383837047838B09025B0441EA5343D2
:100AE0009BB283837047038C23F002031B041B0C0F
:100AF0000B4303847047038C23F008031B041B0C77
:100B00000B4303847047038C23F020031B041B0C4E
:100B100043EA01139BB203847047038C23F08003E4
:100B20001B041B0C43EA01139BB203847047038C24
:100B300023F400731B041B0C43EA01239BB20384C0
:100B40007047038C23F400631B041B0C43EA01234E
:100B50009BB203847047038C23F400531B041B0CCB
:100B600043EA01339BB20384704710B5048C012320
:100B70008B40A4B224EA03030384038C12FA01F12C
:100B80000B439BB2038410BD10B5048C04238B402F
:100B9000A4B224EA03030384038C12FA01F10B4389
:100BA0009BB2038410BD0023012203804380828016
:100BB000C38003817047406B7047806B7047C06B88
:100BC0007047006C7047038B23F00C031B041B0C55
:100BD0000383038B9BB20B4303837047038B23F484
:100BE00040631B041B0C0383038B9BB243EA01236A
:100BF0009BB203837047F8B50C464988A288B4F8C5
:100C000000E02389054600290CBF02270027012A9E
:100C100014BF01260226BEF1000F10D1FFF72EFCF3
:100C20002846E188FFF7CFFF284639463246238918
:100C3000FFF73DFCE1882846BDE8F840CEE7FFF726
:100C400036FC2846E188FFF7C9FF28463946324678
:100C50002389FFF713FCE1882846BDE8F840B2E796
:100C6000838B23F00C031B041B0C8383838B9BB2AD
:100C70000B4383837047838B23F440631B041B0C5B
:100C80008383838B9BB243EA01239BB283837047A8
:100C9000F8B50D460B88AA88498804463BB92B89CC
:100CA000FFF7ECFBE9882046BDE8F8408BE7042B12
:100CB00007D12B89FFF7FBFBE9882046BDE8F84008
:100CC0008CE7082BB5F808C0078C1DD127F4807776
:100CD0003F043F0C0784868B038CB6B29BB226F090
:100CE000F30623F4206346EA0C1C43EA01211FFAB1
:100CF0008CFC89B24CEA020241F480718283018447
:100D0000E988BDE8F840ABE727F480573F043F0C83
:100D10000784868B038C26F4407623F40053360533
:100D20005B04360D5B0C46EA022243EA013342EAD9
:100D30000C329BB2E98892B243F4805382830384DD
:100D4000BDE8F84097E74A880B8813438A88134325
:100D5000CA8813430A8913434A8913438A89134370
:100D60009BB2A0F844307047002303804380838007
:100D7000C3800381438183817047B0F8443029B137
:100D80006FEA43436FEA53439BB201E05B045B0CA1
:100D9000A0F844307047838819B19BB243F0040334
:100DA00003E023F004031B041B0C8380704783883B
:100DB00019B19BB243F0010303E023F001031B04CC
:100DC0001B0C8380704783899BB20AB1194301E0F1
:100DD00023EA01018181704781827047038A1942A9
:100DE0000CBF002001207047C94389B201827047BF
:100DF000038A828911EA030092B203D011420CBF28
:100E0000002001207047C94389B2018270470A431C
:100E1000A0F84820704783899BB20AB1194301E0CA
:100E200023EA010181817047838819B19BB243F0A5
:100E3000080303E023F008031B041B0C83807047A6
:100E4000038923F007031B041B0C038170470389EC
:100E500023F070031B041B0C0B43038103899BB21B
:100E600043F007030381704738B50D461146012250
:100E7000602D044602D1FFF71AFB01E0FFF7FEFAEE
:100E8000238923F070031B041B0C1D432581238938
:100E90009BB243F00703238138BD038923F070031D
:100EA0001B041B0C0B4303817047838823F07003E2
:100EB0001B041B0C838083889BB20B438380704789
:100EC000038923F007031B041B0C038103899BB2D6
:100ED0000B4303817047038923F080031B041B0C21
:100EE000038103899BB20B430381704710B50489CA
:100EF000E4B20C43144344EA0324A4B2048110BDB9
:100F000010B50446FFF7F2FF23899BB243F48043F8
:100F1000238110BD10B50446FFF7E8FF238923F0B5
:100F200077031B041B0C43F07703238110BD70B5BE
:100F30000489068B058C26F44076ADB226F00306B4
:100F400024F00704360425F022052404360C15434A
:100F5000240C46F4807645EA0315214346F0010649
:100F6000ADB201810683058470BD838819B19BB23F
:100F700043F0800303E023F080031B041B0C8380F9
:100F80007047A0F85010704708B5234B984205D120
:100F900010200121FEF7F2FF102037E01F4B98428E
:100FA00007D14FF400300121FEF7DCFF4FF4003091
:100FB00009E01B4B98420BD14FF480200121FEF732
:100FC000D1FF4FF480200021BDE80840FEF7CABFE2
:100FD000144B984207D14FF400200121FEF7C2FFC5
:100FE0004FF40020EFE7104B984207D14FF48010E8
:100FF0000121FEF7B7FF4FF48010E4E70B4B984256
:1010000009D120200121FEF7B9FF20200021BDE8F1
:101010000840FEF7B3BF08BD001001400044004087
:1010200000480040004C00400050004000140140C7
:10103000038ACA889BB223F4405330B513430D464C
:10104000038283890989AA8823F4B0530A436989F2
:1010500023F00C031B040A431B0C92B2134383813D
:10106000838AAA899BB223F44073134385B0838299
:1010700004466846FEF7A6FE1A4B9C4203D003F5D1
:1010800080639C4201D1039B00E0029BA28912B2C3
:10109000002A4FF019012A6801FB03F101DA52001E
:1010A00000E092006423B1FBF2F1B1FBF3F2120114
:1010B000100903FB1011A08900B2002806DAC9004C
:1010C0003231B1FBF3F303F0070305E009013231DC
:1010D000B1FBF3F303F00F031A4392B2228105B080
:1010E00030BD00BF001001404FF4165303600C22C6
:1010F00000238380C38003814281838170470B88F2
:10110000028A10B54C8823438C88C988234392B245
:101110000B4322F470629BB21343038210BD002381
:10112000038043808380C3807047838919B19BB259
:1011300043F4005303E023F400531B041B0C83818E
:101140007047038B03F47F430383038B9BB20B43F2
:1011500003837047838929B16FEA43436FEA53439E
:101160009BB201E05B045B0C83817047838A19B1F9
:101170009BB243F4006303E023F400631B041B0CE5
:1011800083827047C905C90D818070478088C0057A
:10119000C00D7047038A23F00F031B041B0C03824E
:1011A000038A9BB20B4303827047838919B19BB2B8
:1011B00043F0020303E023F002031B041B0C8381B2
:1011C0007047838923F400631B041B0C838183898C
:1011D0009BB20B4383817047038A23F020031B04D7
:1011E0001B0C0382038A9BB20B4303827047038A62
:1011F00019B19BB243F4804303E023F480431B0402
:101200001B0C0382704783899BB243F001038381E7
:101210007047838A19B19BB243F0080303E023F0BF
:1012200008031B041B0C83827047038BDBB2038310
:10123000038B9BB243EA012303837047838A19B16E
:101240009BB243F0200303E023F020031B041B0C9C
:1012500083827047838A19B19BB243F0100303E085
:1012600023F010031B041B0C83827047838A23F036
:1012700004031B041B0C8382838A9BB20B4383826F
:101280007047838A19B19BB243F0020303E023F055
:1012900002031B041B0C83827047838A9BB20AB132
:1012A000194301E023EA010181827047C1F342132F
:1012B00010B501F01F01012414FA01F1A34201D17C
:1012C0000C3004E0022B01D1103000E01430036830
:1012D0000AB1194301E023EA0101016010BD03884E
:1012E00019420CBF002001207047C94389B2018018
:1012F0007047012210B501F01F03C1F342149A4058
:10130000012C01D1838903E0022C0CBF038A838A5C
:101310009BB21340028892B243B1090A012313FA27
:1013200001F111420CBF0020012010BD184610BD74
:10133000090A01238B40DB439BB20380704700BF47
:1013400081F0004102E000BF83F0004330B54FEA76
:1013500041044FEA430594EA050F08BF90EA020FE3
:101360001FBF54EA000C55EA020C7FEA645C7FEA76
:10137000655C00F0E2804FEA5454D4EB5555B8BF99
:101380006D420CDD2C4480EA020281EA030382EA0A
:10139000000083EA010180EA020281EA0303362D9C
:1013A00088BF30BD11F0004F4FEA01314FF4801C6F
:1013B0004CEA113102D0404261EB410113F0004F81
:1013C0004FEA03334CEA133302D0524263EB430338
:1013D00094EA050F00F0A780A4F10104D5F1200ED6
:1013E0000DDB02FA0EFC22FA05F2801841F1000131
:1013F00003FA0EF2801843FA05F359410EE0A5F105
:1014000020050EF1200E012A03FA0EFC28BF4CF035
:10141000020C43FA05F3C01851EBE37101F00045EB
:1014200007D54FF0000EDCF1000C7EEB00006EEBF8
:101430000101B1F5801F1BD3B1F5001F0CD3490882
:101440005FEA30004FEA3C0C04F101044FEA4452D9
:1014500012F5800F80F09A80BCF1004F08BF5FEA60
:10146000500C50F1000041EB045141EA050130BD40
:101470005FEA4C0C404141EB010111F4801FA4F1E3
:101480000104E9D191F0000F04BF01460020B1FA38
:1014900081F308BF2033A3F10B03B3F120020CDA70
:1014A0000C3208DD02F1140CC2F10C0201FA0CF04E
:1014B00021FA02F10CE002F11402D8BFC2F1200CB3
:1014C00001FA02F120FA0CFCDCBF41EA0C01904069
:1014D000E41AA2BF01EB0451294330BD6FEA0404B2
:1014E0001F3C1CDA0C340EDC04F11404C4F120029D
:1014F00020FA04F001FA02F340EA030021FA04F3AF
:1015000045EA030130BDC4F10C04C4F1200220FA05
:1015100002F001FA04F340EA0300294630BD21FA43
:1015200004F0294630BD94F0000F83F4801306BF09
:1015300081F480110134013D4EE77FEA645C18BFFD
:101540007FEA655C29D094EA050F08BF90EA020F94
:1015500005D054EA000C04BF1946104630BD91EA8C
:10156000030F1EBF0021002030BD5FEA545C05D18F
:101570004000494128BF41F0004130BD14F58004CE
:101580003CBF01F5801130BD01F0004545F0FE4142
:1015900041F470014FF0000030BD7FEA645C1ABF77
:1015A000194610467FEA655C1CBF0B46024650EAAE
:1015B000013406BF52EA033591EA030F41F40021DA
:1015C00030BD00BF90F0000F04BF0021704730B560
:1015D0004FF4806404F132044FF000054FF0000135
:1015E00050E700BF90F0000F04BF0021704730B5F6
:1015F0004FF4806404F1320410F0004548BF4042CB
:101600004FF000013EE700BF42004FEAE2014FEA1F
:1016100031014FEA02701FBF12F07F4393F07F4FFA
:1016200081F06051704792F0000F14BF93F07F4F2C
:10163000704730B54FF4607401F0004521F000416F
:1016400020E700BF50EA010208BF704730B54FF0F5
:1016500000050AE050EA010208BF704730B511F0FA
:10166000004502D5404261EB41014FF4806404F132
:1016700032045FEA915C3FF4DCAE4FF003025FEAB4
:10168000DC0C18BF03325FEADC0C18BF033202EB3C
:10169000DC02C2F1200300FA03FC20FA02F001FA96
:1016A00003FE40EA0E0021FA02F11444C1E600BF35
:1016B00070B54FF0FF0C4CF4E06C1CEA11541DBFE8
:1016C0001CEA135594EA0C0F95EA0C0F00F0DEF8B3
:1016D0002C4481EA030621EA4C5123EA4C5350EA98
:1016E000013518BF52EA033541F4801143F48013E9
:1016F00038D0A0FB02CE4FF00005E1FB02E506F07A
:101700000042E0FB03E54FF00006E1FB03569CF0CE
:10171000000F18BF4EF0010EA4F1FF04B6F5007FD4
:1017200064F5407404D25FEA4E0E6D4146EB060646
:1017300042EAC62141EA55514FEAC52040EA5E50CF
:101740004FEACE2EB4F1FD0C88BFBCF5E06F1ED879
:10175000BEF1004F08BF5FEA500E50F1000041EBB0
:10176000045170BD06F0004646EA010140EA02005D
:1017700081EA0301B4EB5C04C2BFD4EB0C0541EA7F
:10178000045170BD41F480114FF0000E013C00F394
:10179000AB8014F1360FDEBF002001F0004170BDB8
:1017A000C4F10004203C35DA0C341BDC04F11404D1
:1017B000C4F1200500FA05F320FA04F001FA05F25D
:1017C00040EA020001F0004221F0004110EBD3702A
:1017D00021FA04F642EB06015EEA430E08BF20EA56
:1017E000D37070BDC4F10C04C4F1200500FA04F3F9
:1017F00020FA05F001FA04F240EA020001F000418B
:1018000010EBD37041F100015EEA430E08BF20EAFD
:10181000D37070BDC4F1200500FA05F24EEA020E45
:1018200020FA04F301FA05F243EA020321FA04F074
:1018300001F0004121FA04F220EA020000EBD3702B
:101840005EEA430E08BF20EAD37070BD94F0000F2B
:101850000FD101F00046400041EB010111F4801F5F
:1018600008BF013CF7D041EA060195F0000F18BF10
:10187000704703F00046520043EB030313F4801F4C
:1018800008BF013DF7D043EA0603704794EA0C0F06
:101890000CEA135518BF95EA0C0F0CD050EA41061C
:1018A00018BF52EA4306D1D181EA030101F0004199
:1018B0004FF0000070BD50EA410606BF10461946C1
:1018C00052EA430619D094EA0C0F02D150EA0136CD
:1018D00013D195EA0C0F05D152EA03361CBF10460E
:1018E00019460AD181EA030101F0004141F0FE41AD
:1018F00041F470014FF0000070BD41F0FE4141F431
:10190000780170BD70B54FF0FF0C4CF4E06C1CEA30
:1019100011541DBF1CEA135594EA0C0F95EA0C0FE5
:1019200000F0A7F8A4EB050481EA030E52EA0335A0
:101930004FEA013100F088804FEA03334FF08055C1
:1019400045EA131343EA12634FEA022245EA1115EE
:1019500045EA10654FEA00260EF000419D4208BF9F
:10196000964244F1FD0404F5407402D25B084FEA4C
:101970003202B61A65EB03055B084FEA32024FF4F8
:1019800080104FF4002CB6EB020E75EB030E22BF55
:10199000B61A754640EA0C005B084FEA3202B6EB15
:1019A000020E75EB030E22BFB61A754640EA5C00C4
:1019B0005B084FEA3202B6EB020E75EB030E22BF54
:1019C000B61A754640EA9C005B084FEA3202B6EB55
:1019D000020E75EB030E22BFB61A754640EADC0014
:1019E00055EA060E18D04FEA051545EA16754FEA76
:1019F00006164FEAC30343EA52734FEAC2025FEA94
:101A00001C1CC0D111F4801F0BD141EA00014FF022
:101A100000004FF0004CB6E711F4801F04BF0143F3
:101A20000020B4F1FD0C88BFBCF5E06F3FF6AFAE0F
:101A3000B5EB030C04BFB6EB020C5FEA500C50F19F
:101A4000000041EB045170BD0EF0004E4EEA113122
:101A500014EB5C04C2BFD4EB0C0541EA045170BD29
:101A600041F480114FF0000E013C90E645EA060E6D
:101A70008DE60CEA135594EA0C0F08BF95EA0C0F9B
:101A80003FF43BAF94EA0C0F0AD150EA01347FF4E3
:101A900034AF95EA0C0F7FF425AF104619462CE7BA
:101AA00095EA0C0F06D152EA03353FF4FDAE10461D
:101AB000194622E750EA410618BF52EA43067FF46E
:101AC000C5AE50EA41047FF40DAF52EA43057FF4FE
:101AD000EBAE12E74FF0FF3C06E000BF4FF0010C09
:101AE00002E000BF4FF0010C4DF804CD4FEA410C6D
:101AF0007FEA6C5C4FEA430C18BF7FEA6C5C1BD03A
:101B000001B050EA410C0CBF52EA430C91EA030FBA
:101B100002BF90EA020F0020704710F1000F91EA17
:101B2000030F58BF994208BF90422CBFD8176FEAE5
:101B3000E37040F0010070474FEA410C7FEA6C5CB3
:101B400002D150EA013C07D14FEA430C7FEA6C5CBA
:101B5000D6D152EA033CD3D05DF8040B704700BFE6
:101B60008446104662468C461946634600E000BF34
:101B700001B5FFF7B7FF002848BF10F1000F01BD06
:101B80004DF808EDFFF7F4FF0CBF012000205DF8D1
:101B900008FB00BF4DF808EDFFF7EAFF34BF012056
:101BA00000205DF808FB00BF4DF808EDFFF7E0FFEF
:101BB00094BF012000205DF808FB00BF4DF808ED40
:101BC000FFF7CEFF94BF012000205DF808FB00BFA7
:101BD0004DF808EDFFF7C4FF34BF012000205DF889
:101BE00008FB00BF4FEA410212F5001215D211D5D1
:101BF0006FF47873B3EB625212D94FEAC12343F00A
